:020000040800F2
:100000009437002017050008850400081D09000822
:10001000890400088B0400088D040008000000001B
:100020000000000000000000000000008F04000835
:1000300091040008000000009304000895040008E3
:1000400097040008990400089B0400089D04000818
:100050009F040008A1040008A3040008A5040008E8
:10006000A7040008A9040008AB040008AD040008B8
:10007000AF040008B1040008B3040008B504000888
:10008000B7040008B9040008BB040008BD04000858
:10009000BF040008C1040008C3040008C504000828
:1000A000C7040008C9040008CB040008CD040008F8
:1000B000CF040008D1040008D3040008D5040008C8
:1000C000D7040008D9040008DB040008DD04000898
:1000D000DF040008E1040008E3040008E504000868
:1000E000E7040008E9040008EB040008ED04000838
:1000F000EF040008F1040008000000000000000008
:100100000000000000000000F3040008F5040008EF
:100110000000000000000000F7040008F9040008D7
:10012000FB040008FD040008FF04000801050008A6
:100130000305000805050008070500080905000873
:100140000B05000800000000000000000000000097
:10015000000000000000000000000000000000009F
:1001600000000000000000000D0500080F05000859
:100170001105000800000000130500080000000041
:08018000000000001505000855
:10020000DECEA5ED02003078463337320000000024
:100210000000000000004452385F313430390000E3
:100220000000000000004170706C69636174696FC8
:100230006E00000000000000000000000000000050
:100240000000000000000406FE00DAF7DECEA5ED97
:100250000200307846333732000000000000000012
:10026000000053504C6174436F6E74726F6C6C6518
:1002700072004170706C69636174696F6E00000098
:10028000000000000000000000000000000000006E
:0802900000000000FE00DAF797
:100298007105000817000000BD07000803000000F2
:1002A800F90D000806000000A11000080900000070
:1002B8009912000802000000791300080F000000DE
:1002C80035150008FF0000002D1900080B0000007C
:1002D800411C000800000000751D00080500000012
:1002E800DD39000811000000053D00080A00000083
:1002F800B93F00080A000000694700081300000021
:10030800894B000808000000A152000807000000FF
:10031800495900080F000000315D00081200000074
:10032800D16E0008120000007DE6000815000000EC
:1003380061F0000816000000AD1D0108150000005E
:10034800D11E010816000000692C010814000000E5
:100358002F49072291438D462E492F480A1A06D065
:100368000722914381F30988022282F314882B48DB
:100378002B492C4A00F039F82B482C492C4A00F01C
:1003880034F82C482C492D4A00F02FF82C482D49D8
:100398002D4A00F02AF82D482D492E4A00F025F85C
:1003A8002D482E492E4A00F020F82E482E490022CA
:1003B80000F026F82D482E49091A082903DB0022E7
:1003C8000260043001601F481F49884205D0026856
:1003D800043003B4904703BCF7E700208646EC4698
:1003E80000200021234A9047FEE7884207D0521A8E
:1003F80005D0037801300B700131013AF9D170470B
:10040800884202D002700130FAE770471A487047F4
:1004180094370020943F002094370020A0870108DB
:1004280088010020080200207005000870050008F7
:10043800185E010820880108943F0020943F00209E
:1004480070050008700500087005000870050008B0
:100458007005000870050008185E0108185E01089C
:10046800A0870108080200204834002094340020A6
:1004780094340020E5290008FFFFFFFFFEE7FEE7B0
:10048800FEE7FEE7FEE7FEE7FEE7FEE7FEE7FEE73C
:10049800FEE7FEE7FEE7FEE7FEE7FEE7FEE7FEE72C
:1004A800FEE7FEE7FEE7FEE7FEE7FEE7FEE7FEE71C
:1004B800FEE7FEE7FEE7FEE7FEE7FEE7FEE7FEE70C
:1004C800FEE7FEE7FEE7FEE7FEE7FEE7FEE7FEE7FC
:1004D800FEE7FEE7FEE7FEE7FEE7FEE7FEE7FEE7EC
:1004E800FEE7FEE7FEE7FEE7FEE7FEE7FEE7FEE7DC
:1004F800FEE7FEE7FEE7FEE7FEE7FEE7FEE7FEE7CC
:10050800FEE7FEE7FEE7FEE7FEE7FEE7FEE7134845
:10051800854600F022F84EF68850CEF200000168B9
:1005280051F47001016000BF00BF00BFF1EE100A76
:1005380050F04070E1EE100A4FF0000080F314888C
:100548004EF63C71CEF20001086850F04070086029
:10055800034804490160FFF7FBBE70470080002094
:0805680008ED00E000000008AE
:1005700010B582B04FF003004FF0000140F20D6261
:10058000C0F6000202F074FD4FF0010040F21D6160
:10059000C0F6000140F2FD52C0F6000202F068FD14
:1005A0004FF008004FF0090102460EF083FC4FF0B7
:1005B000070300934FF00004019420464EF6853166
:1005C000C3F6D16141F6B862C3F68562234610F0E6
:1005D0004BFD00944FF0FF00019020464FF00A01C0
:1005E0004FF00B024FF0010301F044FD45F6386077
:1005F000C0F6010005F028FE02B010BD08B519B91B
:100600004FF0030012F0FAFA08BD00BF08B5012947
:1006100003D14FF0010012F0F1FA08BD08B54FF018
:100620000A0000F0B7FD08BD08B501464FF00B0009
:1006300000F0B0FD08BD00BF45F65463C0F60103ED
:100640001A684EF60C50CEF200000260FEE700BFC2
:1006500008B5FFF7F1FF00BF51E8002FBFF35F8F30
:1006600041E80003012B3FF4F7AF1046704700BF8D
:1006700013461A462DE9F00F092AC0F00980B1E8A7
:10068000F80FA0E8F80FA2F10902092ABFF4F7AFAA
:100690004FF00C0303FB02F21D4B1A44974600F087
:1006A00032B800BF00BF00BF00BF0B68036000F09E
:1006B0002AB800BF00BF91E8180080E8180000F0D9
:1006C00022B891E8380080E8380000F01CB891E8C2
:1006D000780080E8780000F016B891E8F80080E82B
:1006E000F80000F010B891E8F80180E8F80100F097
:1006F0000AB891E8F80380E8F80300F004B891E83C
:10070000F80780E8F807BDE8F00F704713460000CF
:100710009E06000813461A462DE9F00F0B460C46BC
:100720000D460E460F46884689468A468B46092A5C
:10073000C0F00780A0E8F80FA2F10902092ABFF46F
:10074000F9AF4FF0080303FB02F2144B1A4497462B
:1007500000F020B800BF00BF046000F01BB800BF6D
:1007600080E8300000F016B880E8700000F012B8A1
:1007700080E8F00000F00EB880E8F00100F00AB860
:1007800080E8F00300F006B880E8F00700F002B857
:1007900080E8F00FBDE8F00F7047134650070008DF
:1007A000EFF311804FF0800181F3118870474FF013
:1007B000000000BF80F31188704700BF30B440F2E2
:1007C0000003C0F6000340F28812C0F60002D01AFF
:1007D0004FEAA001B1F5C47F04D81346264A9A42D5
:1007E00001D324E0FEE7254D254C601B20F00305D6
:1007F0004FF0000340F20002C2F2000240F200019A
:10080000C0F6000105F10400C5F380045D589D5059
:1008100003F10403834226D109E05C589C5003F1A4
:1008200004035C58D45003F104038342F5D14EF61F
:100830000853CEF2000340F20002C2F200021A6036
:100840004FF0B501CBF26B1143F29440C2F20000BD
:1008500001604EF61453CEF200031A6842F0100104
:10086000196030BC7047002CD7D05C589C5003F105
:1008700004038342D1D1DAE7000000080400000835
:100880008B01000830B4034600283FD002F1100469
:1008900040F20000C2F2000040F82430002A0ADAD8
:1008A00012F10C0F36DB02F10C024EF61850CEF2AC
:1008B000000011542EE04EF20015CEF200054CB2AD
:1008C00011EA240438BF80244EF20041CEF2000128
:1008D00054541346002AB8BF02F11F034FEA6310B5
:1008E00005EB80014FF01F03C8F200031340002BFB
:1008F00005DA03F1FF3262F01F0303F1010358B27E
:100900004FF0010202FA00F30B6003E0002AC7DB9C
:10091000014DD4E730BC704780E100E01EF0040FC9
:100920000CBFEFF30880EFF3098020E9F00F00F02F
:1009300001B800BF10B5026843F24843C2F2000399
:100940001A604168596082689A60C168D96002691A
:100950001A614169596182699A61C169D961026A02
:100960001A62416A5962826A9A62C16AD962026BEA
:100970001A63416B5963826B9A63C16BD96300F14F
:10098000400018644EF62850CEF2000002685A6407
:1009900015F002FA002800F0FB8145F65860C0F619
:1009A000010015F0FFF94EF62C54CEF20004236836
:1009B000002B05DA45F66860C0F6010015F0F2F983
:1009C0004EF62C51CEF20001086810F0020F05D04F
:1009D00045F67860C0F6010015F0E4F94EF62852AD
:1009E000CEF200025478002C72D045F69060C0F62A
:1009F000010015F0D7F94EF62853CEF200035978CE
:100A000011F0010F05D045F6A060C0F6010015F009
:100A1000C9F94EF62850CEF20000427802F00204E6
:100A2000E3B22BB145F6C060C0F6010015F0BAF98B
:100A30004EF62851CEF20001487800F00402D4B2FC
:100A40002CB145F6E460C0F6010015F0ABF94EF6A6
:100A50002853CEF20003597801F00800C2B22AB13F
:100A600045F60870C0F6010015F09CF94EF62854C2
:100A7000CEF20004637803F01001C8B228B145F645
:100A80002870C0F6010015F08DF94EF62852CEF20E
:100A90000002547804F02003D9B229B145F6487019
:100AA000C0F6010015F07EF94EF62850CEF2000097
:100AB000427802F08004E3B253B14EF63851CEF2E0
:100AC0000001096845F66870C0F6010015F06AF982
:100AD0004EF62850CEF20000428894B2002C5ED030
:100AE00045F68870C0F6010015F05CF94EF6285303
:100AF000CEF20003598811F0010F05D045F6987029
:100B0000C0F6010015F04EF94EF62850CEF2000066
:100B1000428802F00204A3B22BB145F6C470C0F6BD
:100B2000010015F03FF94EF62851CEF20001488839
:100B300000F0040294B22CB145F6E870C0F6010052
:100B400015F030F94EF62853CEF20003598801F023
:100B5000080082B22AB146F22800C0F6010015F062
:100B600021F94EF62854CEF20004638803F4807114
:100B700088B228B146F25800C0F6010015F012F90B
:100B80004EF62852CEF20002548804F4007399B253
:100B900029B146F27400C0F6010015F003F94EF6D3
:100BA0002850CEF200000278002A63D046F28C0072
:100BB000C0F6010015F0F6F84EF62854CEF2000407
:100BC000237813F0010F05D046F29C00C0F6010017
:100BD00015F0E8F84EF62851CEF20001087800F042
:100BE0000202D4B22CB146F2BC00C0F6010015F0EE
:100BF000D9F84EF62853CEF20003197801F0080018
:100C0000C2B22AB146F2D400C0F6010015F0CAF80B
:100C10004EF62854CEF20004237803F01001C8B237
:100C200028B146F2F800C0F6010015F0BBF84EF608
:100C30002852CEF20002147804F02003D9B229B170
:100C400046F21C10C0F6010015F0ACF84EF6285024
:100C5000CEF20000027802F08004E3B253B14EF607
:100C60003451CEF20001096846F23C10C0F6010092
:100C700015F098F843F24844C2F20004216A46F2A3
:100C80006810C0F6010015F08DF8616A46F27C101C
:100C9000C0F6010015F086F8A16A46F29010C0F681
:100CA000010015F07FF8E16A46F2A410C0F60100D9
:100CB00015F078F8216846F2B810C0F6010015F07A
:100CC00071F8616846F2CC10C0F6010015F06AF8C0
:100CD000A16846F2E010C0F6010015F063F8E16883
:100CE00046F2F410C0F6010015F05CF8216946F2F6
:100CF0000820C0F6010015F055F8616946F21C2085
:100D0000C0F6010015F04EF8A16946F23020C0F699
:100D1000010015F047F8E16946F24420C0F60100F1
:100D200015F040F8216B46F25820C0F6010015F08E
:100D300039F8216C46F26C20C0F6010015F032F84B
:100D4000616B46F28020C0F6010015F02BF8A16B14
:100D500046F2A420C0F6010015F024F843F29040BA
:100D6000C2F20000026846F2C820C0F60100114637
:100D7000126815F017F840F61C03C2F200031A6857
:100D800046F2E020C0F601001146126815F00AF89C
:100D9000FFF75EFC10BD00BF00B504F09BFC00280F
:100DA00008BF5DF804FBEFF30981EFF3118221E93D
:100DB000F40F5DF804EB1EF0100F08BF21ED108A50
:100DC00041F804ED0B4C2268002A18BF516004F072
:100DD000F3FC2268516851F804EB1EF0100F08BFB5
:100DE000B1EC108AB1E8F40F82F3118881F309881D
:100DF000704700009034002008B540F69950C0F6C6
:100E000000004FF0FF016FF00102FFF73BFD08BD4E
:100E1000F8B507460C461E460799089D14F0030FC7
:100E200000D0FEE722B1A4EB8500A0F1480401E068
:100E300004F14800012D01D8A16205E02A46FFF720
:100E400017FCA7EB8507A7624FF0000363604FF024
:100E50001130E0624FF0223121634FF03332626390
:100E60004FF04433A3604FF05530E0604FF06631EF
:100E700021614FF0773262614FF08833A3614FF008
:100E80009930E0614FF0AA3121624FF0BB326262CB
:100E90004FF0CC33A363E663069820644FF0807173
:100EA00061646FF00202226005F11200F8BD00BF1C
:100EB00062B64EF60453CEF200031A6842F0805038
:100EC000186000BF10B540F20403C4F600031C68AC
:100ED00046F25C31C0F601010A6824EA020446F2D7
:100EE0004432C0F60102106804431C6040F204431F
:100EF000C4F600031868496820EA0100526840EA15
:100F000002041C6040F60403C4F60003186818606D
:100F100040F60441C4F600010A680A6041F2040484
:100F2000C4F600042368236041F20440C4F60000C4
:100F30000168016040F20C01C4F600010C6846F241
:100F40004C42C0F60102136824EA030446F27433EB
:100F5000C0F60103186804430C6040F20C41C4F66B
:100F600000010C68506824EA0004586804430C60CF
:100F700040F60C01C4F600010C68906824EA0004F5
:100F8000986804430C6040F60C41C4F600010C68FC
:100F9000D06824EA0004D86804430C6041F20C01D4
:100FA000C4F600010868126920EA02001B6940EAE1
:100FB00003040C6041F20C41C4F6000108680860AB
:100FC00046F22C33C0F601031A6840F21404C4F64A
:100FD00000042260596840F21440C4F60000016029
:100FE0004FF0000340F61402C4F60002136040F60E
:100FF0001444C4F60004236041F21401C4F6000155
:101000000B6041F21440C4F60000036040F200019E
:10101000C4F600010C6846F28C32C0F60102136877
:1010200024EA030446F26443C0F60103186804434B
:101030000C6040F20041C4F600010C68506824EADC
:101040000004586804430C6040F60001C4F6000137
:101050000C68906824EA0004986804430C6040F629
:101060000041C4F600010C68D06824EA0004D86886
:101070002043086041F20001C4F6000108681269CB
:1010800020EA02001B691843086041F20041C4F6DF
:1010900000010A680A604FF0010002F067FD10BD10
:1010A00008B541F21403C4F202031A6842F4FC00CA
:1010B0001860FFF707FF08BD2DE9F00146F2A434E0
:1010C000C0F6010454F820004FEAD106C7684FEA81
:1010D00041044FF0030505FA04F56FEA050546F2F1
:1010E0007C4CC0F6010C9DF814805CF828C00CFA0A
:1010F00004FC2F404CEA0707C760476846F2004CE3
:10110000C0F6010C5CF8233003FA01F34FF0010C38
:101110000CFA01FC27EA0C073B434360836846F264
:101120003C47C0F601079DF818C057F82C7007FA25
:1011300004F72B403B43836006F1080350F823700B
:1011400001F007014FEA8101079E06F00F0606FA3B
:1011500001F64FF00F0C0CFA01F127EA01013143BF
:1011600040F8231003681D4046F2F031C0F601013B
:1011700051F8222002FA04F425430560BDE8F0018D
:10118000704700BF46F2A433C0F6010353F82000B5
:101190000069704746F20843C0F6010353F8203057
:1011A0007BB139B146F2BC31C0F6010151F82020C3
:1011B0001360704746F2F822C0F6010252F8200090
:1011C0000360704708B540F20C23C2F200031968AF
:1011D000A1B1B0B9FFF7E4FA40F20C22C2F200026A
:1011E00011684FF000034B6240F20822C2F2000285
:1011F0001370FFF7DFFA4FF0010008BD4FF0000059
:1012000008BD4FF0000008BD10B50C4640F20C239D
:10121000C2F200031968A9B1B8B9FFF7C1FA40F2E8
:101220000C22C2F200021368596A40F20822C2F28C
:101230000002137841EA03412160FFF7BBFA4FF047
:10124000010010BD4FF0000010BD4FF0000010BDB8
:1012500010B50C4640F20C23C2F200031968A1B18C
:10126000B0B9FFF79DFA40F20C22C2F200021368F7
:101270005C624FEA144440F20821C2F200010C7093
:10128000FFF798FA4FF0010010BD4FF0000010BDBD
:101290004FF0000010BD00BF41F22403C4F202036E
:1012A0001B6847F20402C4F20002126840F21021E7
:1012B000C2F200014FF000000870C2F3400242EA9F
:1012C000D36010F0010F04D008464FF08001017088
:1012D00023E04FEA136303F01001CAB23AB140F2BF
:1012E0001023C2F200034FF001021A7015E003F060
:1012F0000400C1B239B140F21020C2F200004FF038
:101300004001017009E013F0600F06D040F2102395
:10131000C2F200034FF020021A7041F22403C4F21B
:1013200002031A6842F08070186047F20001C4F2AC
:1013300000010B6843F008020A6043F29040C2F2D9
:101340000000016840F21423C2F2000319607047E4
:1013500040F21023C2F200031878704708B54FF22C
:10136000AC71C1F6FF714FF00C0212F035FF4FF077
:101370000C0008BD0000000010B542F20803CEF2D8
:1013800004031A6842F01000186041F23140C0F6C0
:1013900000004FF00F014FF03602FFF773FA41F2F1
:1013A0001C01C4F202010C6844F010030B6046F209
:1013B0008842C0F60102106841F20004C4F2000441
:1013C000206046F6E001C0F60101886911F0C2FC18
:1013D00015A3D3E9002311F001FF4FF000024FF0F5
:1013E0000003C3F6F07311F0B3FD11F01FFD41F2DD
:1013F0002C03C4F20003188041F22800C4F200005C
:101400004FF00002028046F28C41C0F601010868EC
:1014100041F20C03C4F200031860228842F001017B
:10142000218010BDAFF300802D431CEBE2362A3F34
:10143000684620F007018D4601B541F21003C4F261
:1014400000034FF000021A6004F054FCBDE80140B4
:101450008546704770B50446B0F5CC7F2FD940F271
:101460003233984216D940F26560844215D940F66D
:10147000CB418C4214D941F69712944213D943F2CE
:101480002F36B44212D946F25F639C4298BF0625BC
:101490000ED90FE04FF001050AE04FF0020507E01A
:1014A0004FF0030504E04FF0040501E04FF005059F
:1014B000072D06D1FFF7CCF84FF0070501E04FF0FC
:1014C0000005FFF76DF9064604EB84044FEAC400FB
:1014D00046F29041C0F6010151F83520B0FBF2F31D
:1014E0009CB2012C05D9B4F5805F04D3FFF7B0F8A6
:1014F00001E04FF0020443F20000C4F2000045F2A4
:101500005551016046F29042C0F6010202EBC5055A
:101510006B6843F20401C4F200010B6043F208025D
:10152000C4F2000214604AF6AA2303603046FFF7B3
:1015300041F970BD08B543F20003C4F200034CF654
:10154000CC421A604FF0C800FFF784FF08BD00BF0F
:1015500043F20003C4F200034AF6AA221A6070475D
:1015600010B5044643F20C03C4F20003186810F0EF
:10157000010F74D04FF0320005F066FE43F20C010B
:10158000C4F200010A6812F0010F68D04FF0320077
:1015900005F05AFE43F20C03C4F20003186810F081
:1015A000010F5CD04FF0320005F04EFE43F20C010B
:1015B000C4F200010A6812F0010F50D04FF032005F
:1015C00005F042FE43F20C03C4F20003186810F069
:1015D000010F44D04FF0320005F036FE43F20C010B
:1015E000C4F200010A6812F0010F38D04FF0320047
:1015F00005F02AFE43F20C03C4F20003186810F051
:10160000010F2CD04FF0320005F01EFE43F20C010A
:10161000C4F200010A6812F0010F20D04FF032002E
:1016200005F012FE43F20C03C4F20003186810F038
:10163000010F14D04FF0320005F006FE43F20C010A
:10164000C4F200010A6812F0010F08D04FF0320016
:1016500005F0FAFD43F20C03C4F200031B682046B8
:10166000FFF7F8FE10BD00BF02469CF8043043B1FE
:10167000DCF8000040B140F24021C2F2000141F824
:101680002200DCF8000050B940F24023C2F200030F
:1016900053F8220049F64042002808BF1046704720
:1016A00038B50D460446F0B1132801D9FEF7D0FF36
:1016B00046F6E003C0F6010353F82400B0FBF5F250
:1016C0004FEA124202F10101B0FBF1F3B3FBF5F571
:1016D00046F69000C0F6010050F824108A62CD62F0
:1016E0004FF000024A6238BDF0B583B000918DF82A
:1016F000042008281ED10CE007FA05F1314232D04F
:10170000EC462846FFF7B0FF01462846FFF7C8FF22
:1017100029E04FF0010749F20806C0F208063C46EE
:1017200007FA07F0304215D104F101042546142CC4
:10173000E2D10DE046F22473C0F601031C5C3CB11B
:10174000EC462046FFF790FF01462046FFF7A8FF32
:1017500003B0F0BDEC463846FFF786FF0146384639
:10176000FFF79EFFE0E704F1010407FA04F23242BA
:10177000DAD0EC462046FFF777FF01462046FFF718
:101780008FFFD1E710B507EE901A46F26064C0F6FD
:10179000010404EB0014B7EE007AF4EEC77AF1EE20
:1017A00010FA09DCF5EE407AF1EE10FA9FED1C0A12
:1017B00048BFF0EE407A01E0F7EE007A2378012B83
:1017C00017D16068D0ED001AB8EE612A62EE272AC0
:1017D00012EE900A11F064FB4FF000024FF000038C
:1017E000C3F6E07311F0B6FB11F020FBA2681060A5
:1017F00010BD022B13D1DFED0B0A27EEA01A11EE5C
:10180000100A11F04DFB4FF000024FF00003C3F639
:10181000E07311F09FFB11F009FBA168086010BD97
:101820000000000000F07F4510B54FF000044FF0BD
:1018300000002146FFF7A6FF4FF001002146FFF709
:10184000A1FF4FF002002146FFF79CFF4FF003007D
:101850002146FFF797FF4FF004002146FFF792FF64
:101860004FF005002146FFF78DFF4FF0060021469F
:10187000FFF788FF4FF007002146FFF783FF40F294
:101880000C03C4F600031A6846F23471C0F6010175
:10189000086822EA000246F21071C0F601010868E9
:1018A00002431A6040F20C43C4F600031A681A603F
:1018B00040F60C01C4F600010868086040F60C43CD
:1018C000C4F600031A681A6041F20C01C4F6000164
:1018D0000868086040F20003C4F600031A6846F284
:1018E000F451C0F60101086822EA000246F2E06104
:1018F000C0F60101086802431A6040F20043C4F6D2
:1019000000031A681A6040F60001C4F60001086876
:10191000086040F60043C4F600031A681A6041F2FA
:101920000001C4F600010868086010BDF0B585B07C
:1019300040F21820C2F2000046F2F861C0F6010140
:1019400003F046F941F20403C4F202031A684FF0AF
:10195000020161F38F321A6041F21800C4F20200F2
:10196000046844F40075056042F20446C4F20106BE
:101970004FF00007376046F20863C0F601031A68AB
:1019800042F20C41C4F201010A6046F2F460C0F672
:101990000100046842F21045C4F201052C6046F2D1
:1019A0000476C0F60106376842F22C43C4F2010304
:1019B0001F6046F22C72C0F60102116842F2084024
:1019C000C4F201000160046844F0040505600646A5
:1019D000376817F0040FFBD141F21C03C4F2020375
:1019E0001C6846F20871C0F601010A6824EA020484
:1019F00046F2FC65C0F60105286844EA00061E6050
:101A000041F21807C4F202073B684C6823EA04015C
:101A10006A6841EA02053D60694B03F58C7400E099
:101A20003B461E4653F8147C77B153F80C0C00B1BA
:101A3000386056F8081C11B156F8142C516056F84D
:101A4000105C56F8046C2E6003F11407A342E7D330
:101A500046F23073C0F601031C6844F24400C4F23D
:101A6000010004604FF008004FF000010A46FFF744
:101A70003BFE4FF0000400944FF0020501954FF03B
:101A80000A06029620464FF004014FF00302234657
:101A9000FFF712FB009401954FF00B0102912046D5
:101AA0004FF003010A462346FFF706FB0094019519
:101AB000029620464FF005014FF003022346FFF740
:101AC000FBFA00940195029520464FF006014FF075
:101AD00003022346FFF7F0FA0094019502954FF0B8
:101AE000010021464FF003022346FFF7E5FA009478
:101AF00001954FF00107029738464FF00E014FF065
:101B000003022346FFF7D8FA00940195029738465E
:101B10004FF00F014FF003022346FFF7CDFA009478
:101B200001950295384639464FF003022346FFF7E8
:101B3000C3FA4FF0000620463146FFF723FE384631
:101B40003146FFF71FFE28463146FFF71BFE4FF0D8
:101B500003003146FFF716FE4FF004003146FFF751
:101B600011FE4FF005003146FFF70CFE4FF0060066
:101B70003146FFF707FE4FF007003146FFF702FE40
:101B800046F25C62C0F60102116846F20C60C0F6D3
:101B90000100A0F1040300F14C0003F104025B68B2
:101BA00003B1196002F10403526822B904E0FFF79F
:101BB0003BFE05B0F0BD11608342EED1F7E700BFF8
:101BC000DC64010810B5012888BF4FF0FF3425D828
:101BD00040F21820C2F200004FF0000103F010F8AC
:101BE00042F20043C4F201035A6B6FF304025A63DA
:101BF000DA6C986840F4800199601C46236813F001
:101C0000020FFBD042F20042C4F20102D46C40F257
:101C10001820C2F2000003F001F9FFE7204610BDD2
:101C200008B5FFF7CFFF07EE900AB8EE677A9FED91
:101C3000030AC7EE000A10EE900A08BD00F07F45C7
:101C400008B572B646F26073C0F601031A684EF624
:101C50003470CEF20000026046F25471C0F6010109
:101C60000A684EF68853CEF200031A6046F25070AE
:101C7000C0F60100016842F20802CEF204021160CF
:101C800046F25C73C0F60103186842F20C01CEF212
:101C90000401086041F20003C4F202031A6842F42E
:101CA0008030186019460B6813F4003FFBD046F2F1
:101CB0005872C0F60102106841F20401C4F2020138
:101CC000086046F24C73C0F601031A6842F2000045
:101CD000C4F20200026041F20001C4F202010B688A
:101CE00043F080720A600846016811F0007FFBD063
:101CF00041F20403C4F202031A684FF0020060F3D9
:101D000001021A6019460B6803F00C02082AFAD186
:101D100041F21800C4F20200016841F001030360BF
:101D200042F21C02C4F20202106845F61861C0F6C5
:101D300001010A6846F24873C0F601031B6850406F
:101D4000184215D045F61861C0F60101087800F078
:101D50000401C8B260B942F21C01C4F20201086871
:101D600020EA0300134018434FF0FF3100F082FDDA
:101D700008BD00BF41F21403C4F202031A6842F026
:101D800001001860704700BF70B41646002A47D0A3
:101D900040F20802C4F20202146814F0010F06D0E7
:101DA00040F20C05C4F202052A68002AFCD140F278
:101DB0000804C4F202044FF00005256046F2687280
:101DC000C0F60102156840F20402C4F20202156076
:101DD00040F21002C4F20202116040F21401C4F297
:101DE0000201086040F20C00C4F20200066046F2F4
:101DF0006472C0F6010211682160206840F001029F
:101E000022606BB140F20C01C4F202010B68002B9E
:101E1000FCD140F20800C4F202004FF00002026060
:101E200070BC704740F29023C2F2000318687047FC
:101E300070B48568C668446806FB0540411819609F
:101E400040F29020C2F20000006881420CD2521889
:101E500090420CD340F29420C2F20000026889182C
:101E600019604FF0010004E04FF0000001E04FF076
:101E7000000070BC704700BFF8B50446FFF768FB70
:101E800003F02EFF064640F29825C2F200054FF0FF
:101E900000072B689869042C17D8DFE804F00306C4
:101EA00009101300C0F3400210E0C0F380120DE0EF
:101EB00000F01102012A14BF0022012206E0C0F343
:101EC000800203E0C0F3401200E03A46A2B9C0F33A
:101ED000072111F0010F12D100F01003D8B288B918
:101EE00001F00202D1B281B903F0FAFE831B052B87
:101EF000CFD94FF00000F8BD4FF00100F8BD4FF012
:101F00000000F8BD4FF00000F8BD4FF00000F8BD34
:101F1000F8B540F29824C2F2000425684FF0FF366D
:101F2000EE61FF2B34BF1E46FF264FF000044FF03A
:101F3000A00767F3090461F38A2466F31744FF2BB3
:101F400094BF0023012363F3186462F359646C6047
:101F500060F34D346C60002914BF03200020FFF7AC
:101F60008BFF002814BF30460020F8BD2DE9F0415A
:101F700080460F4616461D46FFF7CAFF0446002856
:101F800074D14FF0050003F031FA4046394632462D
:101F90002B46FFF7BDFF0446002867D14FF0050030
:101FA00003F024FA4046394632462B46FFF7B0FF8D
:101FB000044600285AD14FF0050003F017FA4046B6
:101FC000394632462B46FFF7A3FF044600284DD181
:101FD0004FF0050003F00AFA4046394632462B46D8
:101FE000FFF796FF0446002840D14FF0050003F0AC
:101FF000FDF94046394632462B46FFF789FF044635
:10200000002833D14FF0050003F0F0F9404639467F
:1020100032462B46FFF77CFF044638BB4FF00500E5
:1020200003F0E4F94046394632462B46FFF770FF8D
:102030000446D8B94FF0050003F0D8F940463946B8
:1020400032462B46FFF764FF044678B94FF005008F
:1020500003F0CCF94046394632462B46FFF758FF8D
:10206000044618B94FF0050003F0C0F92046BDE85A
:10207000F08100BF2DE9F04184B014461D460B29C4
:1020800000F29F800B2A00F29F8001EB810246F252
:102090008873C0F6010303EB8202137C002B40F02F
:1020A000968004EB840246F28873C0F6010303EBCA
:1020B0008202137C012B40F08D8046F28873C0F6BB
:1020C000010301EB810653F8262004EB840653F844
:1020D00026309A4240F0818040F29C27C2F20007ED
:1020E0003870012A02D0022A23D111E041F21C00EB
:1020F000C4F20200066846F40012026040F298231F
:10210000C2F2000345F20047C4F200071F6010E06E
:1021100041F21C00C4F20200066846F4800202602C
:1021200040F29823C2F2000345F60007C4F200070C
:102130001F6046F28878C0F6010801EB810108EBC8
:102140008102107991684FF0000700974FF0010667
:102150000196D36802934FF003023346FEF7ACFFBB
:1021600004EB840408EB84042079A16800970196AD
:10217000E26802924FF003023346FEF79DFF40F201
:102180009820C2F2000001680F6046F28473C0F626
:1021900001031A680A611DB340F29420C2F20000E4
:1021A0000A99016040F29022C2F200020B9B136078
:1021B00040F28810C2F20000294606F0FDFC3046CD
:1021C00010E04FF000000DE04FF000000AE04FF08B
:1021D000000007E04FF0000004E04FF0000001E0D5
:1021E0004FF0010004B0BDE8F08100BF2DE9F04FD1
:1021F00083B091460D46002900F09C8040F2982360
:10220000C2F2000319680A6842F001040C60044637
:1022100040F29C2AC2F2000A46F2787BC0F6010B1B
:1022200040F29827C2F200079AF800005BF820609D
:1022300006F1FF3309EA0301731A00F1FF3202F0DD
:10224000FF0001288CBF012602264FF001004FF04D
:1022500000010246AB4294BFF3187319FFF786FEE4
:102260000646002852D09AF8001001F1FF33DAB286
:10227000012A0BD83868C9F30721816206F1FF36BD
:102280004FF00200FFF7F8FD002842D03B685FFAEC
:1022900089F29A62013E26D04FF0020806F1FF3023
:1022A00000F0010101914046FFF7E6FD002846D10C
:1022B00032E04046FFF7E0FD70B334B1386814F8FF
:1022C000012B6FEA0201816203E039684FF0FF03DE
:1022D0008B6206F1FF3605F1FF354046FFF7CCFD76
:1022E000002855D118E09AF800005BF820108944C6
:1022F000C1F1000209EA02094FF00400FFF7BCFD3A
:1023000068B1002D90D14FF001000AE04FF00000BD
:1023100007E04FF0000004E04FF0000001E04FF054
:10232000000040F29823C2F2000319684FF0000247
:102330000A6001E04FF0010003B0BDE8F08F24B95E
:102340003B684FF0FF029A6205E0386814F8011B01
:102350006FEA0103836205F1FF35013EC3D0019AA4
:10236000002AA6D04046FFF787FD0028D4D024B924
:1023700038684FF0FF01816205E03B6814F8012BDB
:102380006FEA0200986205F1FF35013E91D1AAE79C
:1023900024B93B684FF0FF00986205E0396814F8F3
:1023A000012B6FEA02038B6205F1FF35013E80D1FC
:1023B00099E700BF30B583B015461C461A4601ABFD
:1023C000FFF736FD48B128462146019AFFF70EFF78
:1023D00000280CBF1820002001E04FF01F0003B0C0
:1023E00030BD00BF2DE9F04F83B004468946164644
:1023F000002A00F09E8040F29C23C2F2000318786D
:1024000000F1FF3101F0FF0340F29822C2F2000216
:102410001168086840F001020A604FF001004FF0B7
:1024200000010A4683428CBF03460223FFF79EFD4C
:10243000002864D040F29C23C2F20003197801F115
:10244000FF30C2B2012A0DD840F29823C2F2000335
:102450001968C4F3072088624FF00200FFF70CFDF3
:1024600000284FD040F29822C2F200021368E4B272
:102470009C624FF00100FFF7FFFC002845D04FF0B1
:1024800001004FF0030740F29828C2F2000800E074
:102490002E464FF001010A463346FFF739FD8246CA
:1024A000002835D0CB46354600F1FF3101F0010060
:1024B00001903846FFF7E0FC00283FD12BE038467A
:1024C000FFF7DAFC38B3D8F80020536A6FEA03014B
:1024D000A14609F8011B05F1FF353846FFF7CCFC92
:1024E000002854D117E04FF00400FFF7C5FCA8B155
:1024F0004FF00000002DCBD14FF0010010E04FF065
:1025000000000DE04FF000000AE04FF0000007E08F
:102510004FF0000004E04FF0000001E04FF0000039
:1025200040F29822C2F2000213684FF000011960D5
:1025300001E04FF0010003B0BDE8F08FD8F8004093
:10254000626A6FEA020389F8003009F10104A146CA
:1025500006F1FF350AEB0501B142C4D0019800280D
:10256000ADD03846FFF788FC0028D4D0D8F800203A
:10257000536A6FEA03018BF8011004F10104A146CC
:1025800005F1FF350AEB0500B04298D1ABE7D8F86A
:102590000000426A6FEA0203637009F10104A14678
:1025A00005F1FF350AEB0501B14288D19BE700BF79
:1025B00030B583B015461C461A4601ABFFF738FC10
:1025C00048B1019829462246FFF70CFF00280CBFAE
:1025D0001820002001E04FF01F0003B030BD00BF05
:1025E00042F21003C4F20203186810F0800F0DD0FD
:1025F00042F20401C4F2020140F22312C4F2675213
:102600000A6048F6AB13CCF6EF530B6042F21000B1
:10261000C4F20200016801F08002002A14BF022007
:102620000020704742F21003C4F20203186810F051
:10263000800F07D142F21001C4F202010A6842F091
:1026400080030B60704700BF40F20003C0F6000338
:10265000984208D340F20001C0F6040188422CBF22
:102660000020012070474FF0000070472DE9F0472F
:1026700006460D46FFF7E8FF002855D02846FFF72D
:10268000E3FF002853D0AE4254D8FEF789F88246C3
:10269000FFF7A6FF0446B8BB41F28830FEF760FFA3
:1026A00046F67803C0F601031A6842F21000C4F23D
:1026B0000200026042F21409C4F20209804642F2AA
:1026C0000C07C4F20207FEF743FFC9F80060D8F810
:1026D000001041F04003C8F8003006F500663A6883
:1026E00012F0010FFBD1386810F0200F0AD03968C2
:1026F00041F020033B60B542E5D24FF06400FEF7A5
:102700002FFF01E04FF0020446F67C02C0F6010202
:10271000106842F21001C4F202010860FFF782FF64
:102720005046FEF747F807E04FF0020404E04FF090
:10273000020401E04FF002042046BDE8F08700BF2C
:10274000F8B507460C4616460846FFF77DFF0028F9
:1027500000F0898006F1FF302018FFF775FF002890
:1027600000F0848040F62C03C2F2000353E8002FEF
:1027700002F1010243E800210129F7D0FFF730FF01
:10278000054600284BD146F68001C0F601010A68D3
:1027900042F21000C4F20200026014F0010F09D0EE
:1027A00037F8013C24F8013C04F1010407F101076A
:1027B00006F1FF36012E25D904F1020207F10200CD
:1027C000A6F1020C4FEA5C0C04F1040E0EEB4C0E69
:1027D00042F20C01C4F202010B6813F0010FFBD1AD
:1027E00030F8023C22F8023C02F1020200F1020041
:1027F0007245F1D10CF101024FEA420024183F1852
:1028000006F001060EB13978218046F68404C0F640
:102810000104226842F21003C4F202031A60FFF7B7
:1028200001FF40F62C03C2F2000353E8002FA2F18F
:10283000010243E80024012CF7D053E8002FB2F145
:10284000004F0DD14FF0000243E80024012CF4D0DA
:102850004EF60450CEF20000016841F08051016054
:10286000BFF32F8F04E04FF0020501E04FF00205A7
:102870002846F8BD30B585B004460D4668464FF091
:10288000FF014FF0100211F0CBFCE3B203F00402A1
:10289000D0B2002840F0A28003F00201CBB223B1F5
:1028A0004FF011008DF8000003E06FF055028DF835
:1028B0000020C4F307218DF80210C4F307438DF8FC
:1028C00004304FEA14648DF806408DF80850FDF787
:1028D00067FF0546FFF784FE002873D142F2080027
:1028E000C4F2020040F22312C4F26752026048F6BA
:1028F000AB11CCF6EF51016042F21003C4F20203B7
:102900001C6814F4007F5DD046F68800C0F6010014
:10291000026842F21001C4F202010A600B6843F03F
:1029200040040C6042F20C00C4F20200026812F093
:10293000010FFBD142F21003C4F202034FF0000179
:10294000196042F20804C4F2020440F22310C4F2F7
:102950006750206048F6AB12CCF6EF5222601B683D
:1029600013F4007F2ED046F68C01C0F601010C68EE
:1029700042F21000C4F2020004604FF60003C1F6F8
:10298000FF7303F11002934213D24FF010044FF083
:102990000001184642F20C02C4F202023DF8013076
:1029A0000B52136813F0010FFBD101F10201A14298
:1029B000F4D142F21004C4F202044FF0000121608D
:1029C000FFF730FE4FF0000442F21000C4F20200A4
:1029D00004602846FDF7EEFE204601E04FF00200BD
:1029E00005B030BD08B543F29440C2F2000043F296
:1029F0009472C2F20002131A4FF0FF314FEAA302A1
:102A0000FDF788FE01F04AFDFEF752FA4FF0000094
:102A100008BD00BFBFF36F8F704700BF46F630138D
:102A2000C0F60103185C00EB400146F64C22C0F6EC
:102A3000010252F821305B6A704700BF38B546F694
:102A40003013C0F601031B5C03EBC30440F2A02269
:102A5000C2F2000202EB840282F8211014693CB138
:102A600040F2A025C2F200051346D2699B69A04737
:102A700038BD00BFF8B506460F4646F63013C0F61F
:102A800001031D5C05EBC50040F2A024C2F2000466
:102A900004EB8004D4F810C0BCF1000F07D0E26949
:102AA0008A4204D030464FF00001A369E047E76155
:102AB00063695BB105EBC50040F2A022C2F20002DF
:102AC00002EB8002304639469269984794F820100C
:102AD00079B127696FB105EBC50540F2A023C2F2B9
:102AE000000303EB8505304694F82110E269AB69D9
:102AF000B847F8BD46F63013C0F60103185C00EB8A
:102B0000400146F64C22C0F6010252F82130186806
:102B100040F080011960704746F63013C0F601039B
:102B2000185C00EB400146F64C22C0F6010252F858
:102B30002130986940F0020199611A6842F08000E2
:102B40001860704746F63013C0F601031A5C02EBBA
:102B5000420346F64C22C0F6010252F82330DA69ED
:102B600012F0800F1ABF996201200020196841F00D
:102B700080021A60704700BF46F63013C0F60103AA
:102B8000185C00EB400346F64C22C0F6010252F8F6
:102B90002300C36913F0800FFBD08162704700BF30
:102BA000F8B5044600EB400246F64C23C0F601039C
:102BB00053F82260F569356205F0010215F0020F45
:102BC0001CBF42F00202D2B215F0040F18BF42F04F
:102BD000080215F0080F18BF42F0040215F4807FB8
:102BE00005D0706810F4804F18BF42F0100215F045
:102BF000200F00D1E2B104EBC40140F2A027C2F2E1
:102C0000000707EB81039F688FB1716A04EBC40072
:102C100040F2A023C2F2000303EB800346F6242017
:102C2000C0F60100005DC9B29B69B84700E0736A55
:102C3000326812F0800F1CD015F0800F19D0316867
:102C40006FF3C711316004EBC40040F2A023C2F25D
:102C5000000353F8203063B140F2A022C2F2000218
:102C600002EB800246F62420C0F60100005D916967
:102C7000984715F0400F17D004EBC40140F2A02391
:102C8000C2F2000303EB810253686BB1084640F2C5
:102C9000A021C2F2000101EB800246F62420C0F61A
:102CA0000100005D91699847F8BD00BF684620F0BB
:102CB00007018D4601B54FF00300FFF771FFBDE836
:102CC00001408546704700BF684620F007018D46E9
:102CD00001B54FF00200FFF763FFBDE801408546F4
:102CE000704700BF684620F007018D4601B54FF0E0
:102CF0000100FFF755FFBDE801408546704700BF62
:102D00002DE9F04385B016461F4646F63013C0F64F
:102D100001031C5C04EB440246F64C25C0F6010599
:102D200055F8224046F64823C0F60103185C00EB34
:102D3000400246F63415C0F6010505EBC20588468B
:102D4000002956D0002E57D0287B29699DF83420C1
:102D500000924FF0010301936A6902924FF003025F
:102D60003B46FEF7A9F940F62C03C2F2000353E8F4
:102D7000002F02F1010243E800210129F7D0216868
:102D80004FF000002060012E14BF0026012662686B
:102D900066F3CF32626046F63020C0F6010002686A
:102DA000B8F1010F14BF4FF000084FF0010868F3AD
:102DB000C302A260216053E8002FA2F1010243E8A0
:102DC0000024012CF7D053E8002FB2F1004F0DD1B1
:102DD0004FF0000243E80024012CF4D04EF60450DA
:102DE000CEF20000016841F080510160BFF32F8FE7
:102DF00017E04FF0010901E04FF0000928786968F9
:102E00009DF8303000934FF001020192AB680293BD
:102E10004FF003023B46FEF74FF9B9F1000FA2D085
:102E200092E705B0BDE8F0832DE9F84F81468B4667
:102E300090461E469DF828A046F63013C0F60103C2
:102E40001D5C05EB450246F64C20C0F6010050F82B
:102E500022409DF82C70012F14BF00270127082E57
:102E600006D0072E02D1B8F1000F01D1FDF7F0FB1B
:102E70000AF1FF31CBB2012B01D9FDF7E9FB46F690
:102E80000C22C0F6010252F82500B0FBFBF1E16014
:102E90004FF0200267F38612BAF1010F04D0002F21
:102EA0000CBF0223002301E04FF0000363F30D3257
:102EB00067F38E326068C0F3C03363F3CF32626071
:102EC0004FF06D01B8F1020F14BF0023012363F32B
:102ED000492118F1000818BF4FF0010868F38A2152
:102EE000082E18BF4FF0000868F30C3121604846E7
:102EF000FFF794FDBDE8F88F2DE9F843054646F647
:102F00003013C0F60103185C00EBC00240F2A024AD
:102F1000C2F2000404EB820446F64C21C0F6010123
:102F200000EB40064FEA860301EB030851F80390DB
:102F3000FDF736FC064694F82000B8B14FF00007C4
:102F4000C9F800703846394698F90420FDF79AFC14
:102F500028463946FFF772FDE3681BB12846E16950
:102F6000A26998474FF0000284F820203046FDF710
:102F700021FCBDE8F88300BF2DE9F04F85B0054680
:102F80008B469246994646F63013C0F601031E5C06
:102F900040F2A028C2F2000806EBC6074FEA8707F6
:102FA00008EB070406EB460046F64C21C0F601018B
:102FB00001EB8006FDF7F4FB039041F21C03C4F221
:102FC0000203186846F61C21C0F601010A6820EACF
:102FD000020E46F62822C0F6010210684EEA0000F2
:102FE000186041F21803C4F202031868496820EA25
:102FF000010052681043186046F63421C0F6010102
:1030000005EB8503C818C95C4278837890F803C043
:10301000CDF800C0007901902846FFF771FE9DF8B9
:10302000382000929DF83C1001912846594652469E
:103030004B46FFF7F9FE109B48F807301298A06046
:10304000119A62601399E160149BA361B0684FF01C
:103050000F0196F90420FDF715FC4FF0010084F8EC
:1030600020000398FDF7A6FB05B0BDE8F08F00BF78
:1030700046F63013C0F60103185C00EBC00340F2C3
:10308000A020C2F2000000EB830319615A6170476F
:1030900046F64823C0F60103185C00EB400146F6F3
:1030A0007C12C0F6010202EB01107047F8B54FF038
:1030B0004C0404FB00F440F66C31C2F200016218CB
:1030C00046F20003C4F2000303EB001345F600458B
:1030D000C4F2000505EB80006558002D6BD09468A4
:1030E0000CB1968801E04FF000061F6866F30F07E9
:1030F0001F6059686FF309015960D16819B15668AA
:10310000A719BFB201E04FF000079E6867F30F06F2
:103110009E603E2994BF00270127DE6867F3CF3603
:10312000DE60DE6816F4004F1DBF4F0907F1FF3760
:1031300007F01F07C1F34407DE6867F38E26DE60E1
:103140000368166A66F303032E7A46F69C25C0F6DA
:10315000010555F8265065F34A236FF30823C3F39E
:103160000115002C14BF022400246C4064F30513E5
:10317000C3F30134002914BF03210021614061F32E
:103180000D336FF3CF336FF3C713036040F6543042
:10319000C2F200000378191F18BF012151624FF0DD
:1031A000010090624FF00003D3621363536302F196
:1031B000100000F0BBFCF8BDF8B545F64443C4F27E
:1031C00000031C6814F4004F52D040F65430C2F291
:1031D0000000017801294BD945F64442C4F20002AF
:1031E000156805F00F0640F66C37C2F200074FF085
:1031F0004C0303FB067545F60040C4F2000000EBEB
:10320000860750F82660C6F3C031EA6A0A43EA62CC
:10321000C6F3C0202B6B03432B63C6F3C0116A6B4C
:103220000A436A63C6F3072000F00803D9B219B154
:103230004FF00001E9630BE0EA6B4AB126F07F0032
:10324000C3B22BB14FF000016963286A03F060FA42
:10325000EA6A0AB9686B18B105F1100000F066FC63
:1032600046F68423C0F60103196826EA01063E608B
:1032700014F4806F0DD040F66130C2F200004FF0C0
:103280000102027040F62833C2F20003186801F010
:1032900017FF14F4006F1CD045F64041C4F2000142
:1032A000086840F008020A6040F66033C2F200038A
:1032B0004FF00101197040F6CC50C2F200004FF0FF
:1032C0000002027040F62833C2F20003186801F0D1
:1032D000F7FE14F4805F1CD045F64041C4F20001B3
:1032E00008686FF3C300086040F66033C2F2000361
:1032F0004FF000021A7040F6CC51C2F200014FF0BC
:103300000100087040F62833C2F20003186801F08B
:10331000D7FE6FEA040445F64442C4F2000214608A
:10332000F8BD00BF684620F007018D4689B500AFA3
:10333000FFF742FFBD46BDE889408546704700BFA4
:1033400045F64043C4F200031A6860F3CF321A60B6
:10335000704700BF40F6D053C2F200031A5C45F636
:103360000040C4F2000049B150F82200C0F301113E
:1033700046F68023C0F60103585C704750F82210CF
:10338000C1F3013346F68022C0F60102D05C7047DB
:1033900040F6D053C2F200031A7845F60043C4F257
:1033A000000353F8221046F69020C0F60100006892
:1033B00021EA000181F0100141F4807043F82200FD
:1033C000704700BF2DE9F00340F6D053C2F200036E
:1033D000185C45F6004CC4F2000C0CEB800C4FEA74
:1033E000001346F20007C4F2000703EB0708D859A0
:1033F00083B207EB4307012A31D901F10204A2F19C
:1034000002094FEA590901F1040606EB4906351B8A
:10341000A5F10205C5F3400534F8024C384620F802
:10342000044B01F10403B34238D10FE033F8025CDE
:10343000044624F8045B03F1020333F8025C858040
:1034400004F1040003F10203B342EFD102F00100E2
:1034500009F1010901EB490107EB890700E010467A
:1034600008B109783980D8F8040062F30900C8F877
:103470000400DCF8003046F67C22C0F60102116838
:1034800023EA01000346C0F3011282F0030161F355
:103490000513CCF80030BDE8F0037047002DC5D00F
:1034A00033F8024C20F8044B03F10203B342BDD1C0
:1034B000CCE700BF2DE9F00140F6D053C2F2000383
:1034C0001C5C45F6004CC4F2000C0CEB840C46F27C
:1034D0000000C4F2000000EB0414A3689BB200EBF0
:1034E0004300E3684FEA83534FEA9353934204D275
:1034F000E2684FEA82534FEA9352012A31D901F12F
:103500000203A2F102084FEA580801F1040707EB91
:103510004807FD1AA5F10205C5F34006044634F834
:10352000045B23F8025C01F10403BB4233D10FE0DA
:10353000254635F8046B23F8026C03F10203A488D6
:1035400023F8024C05F1040403F10203BB42EFD15E
:1035500002F0010308F1010801EB480100EB8800CB
:1035600000E013460BB103880B70DCF8000046F650
:103570009421C0F601010B6820EA03000346C0F362
:10358000013181F0030060F30D33CCF800301046B8
:10359000BDE8F0017047002ECAD034F8045B23F870
:1035A000025C03F10203BB42C2D1D1E708B545F684
:1035B0004043C4F200031A686FF3C3021A604FF06D
:1035C0000000FFF773FD4FF00100FFF76FFD4FF0B4
:1035D0000200FFF76BFD4FF00300FFF767FD4FF0B0
:1035E0000400FFF763FD4FF00500FFF75FFD4FF0AC
:1035F0000600FFF75BFD4FF00700FFF757FD46F6AB
:103600009820C0F60100016845F64C43C4F200035F
:10361000196008BD2DE9F041074640F66C33C2F24F
:1036200000031868002800F0118140F66C31C2F2E6
:1036300000014A683F2A08D940F66C34C2F20004FF
:10364000A5685619E368F51801E04FF0400540F60B
:103650006C30C2F20000C16C002900F0008140F61D
:103660006C32C2F20002146DA54207D840F66C36E7
:10367000C2F20006756D6019B36DC51840F66C3165
:10368000C2F20001D1F89820002A00F0EC8040F648
:103690006C34C2F20004D4F89C60B54209D840F6FC
:1036A0006C30C2F20000D0F8A0507119D0F8A430EC
:1036B000CD1840F66C32C2F20002D2F8E440002C81
:1036C00000F0D58040F66C36C2F20006D6F8E8006D
:1036D000854209D840F66C31C2F20001D1F8EC50B5
:1036E0004219D1F8F030D51840F66C34C2F200041B
:1036F000D4F83061002E00F0BE8040F66C30C2F28B
:103700000000D0F834118D4209D840F66C32C2F274
:103710000002D2F838514C19D2F83C31E51840F685
:103720006C36C2F20006D6F87C01002800F0A780B3
:1037300040F66C31C2F20001D1F88021954209D8DF
:1037400040F66C34C2F20004D4F884515619D4F80F
:103750008831F51840F66C30C2F20000D0F8C8117C
:10376000002900F0908040F66C32C2F20002D2F8DC
:10377000CC41A54209D840F66C36C2F20006D6F814
:10378000D0516019D6F8D431C51840F66C31C2F268
:103790000001D1F81422002A79D040F66C34C2F22C
:1037A0000004D4F81862B54209D840F66C30C2F271
:1037B0000000D0F81C527119D0F82032CD1840F614
:1037C0006C32C2F20002D2F86042002C63D0454E47
:1037D0004FF00808FCF73CFF387A88B140F23031EE
:1037E000C2F200010A8812F0020F0CD04FF001045F
:1037F00004F1010442FA04F313F0010FF8D104E0DC
:103800004FF0000401E04FF0010440F23030C2F20A
:1038100000004FF0010202FA04F201880A4302801C
:103820007889B060BB89F3603F2B99BF013323F0E7
:1038300001031F3323F01F03F360F2688118481956
:10384000B0F5E07F2ED9FCF703FF2BE040F66C3695
:10385000C2F200064FF000084FF040051EE0224E75
:103860004FF001081AE0214E4FF0020816E0204EFA
:103870004FF0030812E01F4E4FF004080EE01E4EFA
:103880004FF005080AE01D4E4FF0060806E01C4EFA
:103890004FF0070802E0134E4FF00808B8F1070F89
:1038A0009AD997E740F6D053C2F2000303F8048098
:1038B0003760756006F1200528464FF000014FF093
:1038C0001C0210F0ADFC34627A68B26306F110009D
:1038D0004FF006013A682B4600F008F92046BDE893
:1038E000F08100BFCC0D0020B80B0020040C00209C
:1038F000500C00209C0C0020E80C0020340D00200F
:10390000800D0020032907D145F64C43C4F2000383
:103910001A6860F306021A60704700BFF0B585B000
:103920000646002842D041F21C01C4F202010C6894
:1039300044F400050D604FF0000400944FF00305BF
:1039400001954FF00E07029720464FF00B012A46D3
:103950002346FDF7B1FB00940195029720464FF0F6
:103960000C012A462346FDF7A7FB46F68C23C0F63A
:1039700001031A6845F64047C4F200073A6028463A
:1039800003F062FC3C6043F22530C0F600004FF0CB
:103990000F014FF04B02FCF775FF45F64440C4F2AF
:1039A000000004604FF41C41396011E04FF000004A
:1039B0004FF00F014FF04B02FCF764FF46F68823EF
:1039C000C0F601031A6845F64040C4F200000260E8
:1039D0003046FCF729FE05B0F0BD00BF2DE9F041EF
:1039E00082B046F6AC27C0F6010743F6BD26C0F606
:1039F000000640F29415C2F200054FF00408CDF81D
:103A0000008038464FF0800132462B4601F0A4FC7E
:103A100040F23434C2F200042060CDF80080384611
:103A20004FF08101324605EB080301F095FC606020
:103A3000CDF8008038464FF08201324605F1080388
:103A400001F08AFCA060CDF8008038464FF0830179
:103A5000324605F10C0301F07FFCE060CDF80080F8
:103A600038464FF08401324605F1100301F074FC32
:103A70002061CDF8008038464FF08501324605F1CF
:103A8000140301F069FC6061CDF8008038464FF006
:103A90008601324605F1180301F05EFCA061CDF805
:103AA000008038464FF08701324605F11C0301F0D3
:103AB00053FCE06102B0BDE8F08100BF08B50546E7
:103AC0004FF000060BE0FCF76BFE2C686168296084
:103AD0006660FCF76FFE22680AB1A06890472B6809
:103AE000B3F1FF3FEFD101F0B9FAF8E70260B3F1AB
:103AF000FF3F18BF8360FF290ED143F29043C2F20B
:103B000000031A6822B192F829304FEA530101E00C
:103B10004FF007010173704701F07F010173704797
:103B200010B14FF000020260704700BF38B5044684
:103B3000FCF736FE0546A4B1636893B9227B40F2D8
:103B40009410C2F2000050F82210616040F8224048
:103B5000227B40F23433C2F2000353F8220001F01A
:103B6000AFFA2846FCF726FE38BD00BF10B5044664
:103B700040F20850C2F200004FF000014FF018026E
:103B800010F04EFBD4B140F28430C2F200004FF08E
:103B900000014FF0300210F043FB40F2E830C2F277
:103BA00000004FF000014FF0180210F039FB40F216
:103BB000E033C2F200034FF002021A7010BD00BFE2
:103BC00038B546F6F023C0F6010353F8205040F212
:103BD000B431C2F2000151F8204046F62032C0F65E
:103BE0000102105CFDF7CEFA2840A04214BF00206D
:103BF000012038BD46F62033C0F601031A5C40F2BE
:103C0000E831C2F2000151F8222046F6F023C0F656
:103C1000010353F8200002420CBF0020012070472E
:103C200070B440F62C03C2F2000353E8002F02F1F7
:103C3000010243E800210129F7D046F62032C0F600
:103C40000102155C40F20851C2F2000151F8254012
:103C500046F6F026C0F6010656F8202024EA0200B7
:103C600041F8250053E8005FA5F1010543E800563F
:103C7000012EF7D053E8005FB5F1004F0DD14FF0A2
:103C8000000543E80056012EF4D04EF60450CEF263
:103C90000000016841F080510160BFF32F8F144292
:103CA0000CBF0020012070BC704700BF46F62C33CB
:103CB000C0F60103185C704710B50446FDF762FAC0
:103CC00040F2B413C2F2000353F82410484010BD70
:103CD00010B504464FF00100FFF748FF46F6B82341
:103CE000C0F6010353F8342040F2E431C2F200017F
:103CF0000A6003EBC404606840F20043C2F20003B0
:103D0000186010BD00B585B04FF00000FFF7E0FF70
:103D10004FF00003009340F20442C2F2000201920D
:103D20004FF04000029046F61430C0F601004FF00C
:103D3000020143F6D952C0F6000201F0F9F940F24F
:103D40000453C2F20003186005B000BD2DE9F00174
:103D5000804600283CD04FF000034FEA83020868F9
:103D600050F823404D6855F8236086EA04078868B8
:103D700050F8235084EA050C4CEA07076FEA070C59
:103D8000C86850F8235026EA050707EA0C0705EA39
:103D90000C0C66EA0C06354040F82350CD6855F807
:103DA0002300384345F823000D6955F823003843B4
:103DB00045F823004D690DB145F8237048688558D2
:103DC000886885504868845003F101034345C4D195
:103DD000BDE8F001704700BF2DE9F84340F2E43838
:103DE000C2F2000840F2D836C2F2000640F2543463
:103DF000C2F200044FF0000540F20047C2F2000793
:103E0000D8F8000000EB800001F0F0FA3368002BD6
:103E100040F09380204629464FF0180210F000FA37
:103E20008BE04FF0060046F6D821C0F60101FFF7FF
:103E30008DFF40F2E031C2F200010B783BB103F19B
:103E4000FF32D3B240F20850C2F20000056040F2E7
:103E5000DC31C2F200010A6822B940F2DC30C2F261
:103E6000000005603BB103F1FF33DBB240F20851C3
:103E7000C2F200014D6040F2DC32C2F20002106872
:103E800020B940F2DC31C2F200010D603BB103F118
:103E9000FF33DBB240F20852C2F20002956040F2FA
:103EA000DC30C2F20000016821B940F2DC32C2F21B
:103EB000000215603BB103F1FF33DBB240F2085062
:103EC000C2F20000C56040F2DC31C2F200010A68B3
:103ED00022B940F2DC30C2F2000005603BB103F1D0
:103EE000FF33DBB240F20851C2F200010D6140F233
:103EF000DC32C2F20002106820B940F2DC31C2F2BA
:103F000000010D603BB103F1FF33DBB240F2085218
:103F1000C2F20002556140F2DC30C2F200000168DA
:103F200021B940F2DC32C2F20002156040F2E0300A
:103F3000C2F200000370356062E7D4F800902846B2
:103F4000FFF7BAFE40EA09012160D4F804904FF06F
:103F50000100FFF7B1FE40EA09026260D4F8089060
:103F60004FF00200FFF7A8FE40EA0900A060D4F875
:103F70000C904FF00300FFF79FFE40EA0903E36057
:103F8000D4F810904FF00400FFF796FE40EA0901C4
:103F90002161D4F814904FF00500FFF78DFE40EA40
:103FA00009026261306800F1010030603B689842AC
:103FB000FFF426AF35E700BF00B585B04FF0000332
:103FC000009340F24C52C2F2000201924FF0800086
:103FD000029046F63840C0F601004FF0060143F665
:103FE000F972C0F6000201F0A3F840F22053C2F2C9
:103FF0000003186005B000BD2DE9F04F85B040F218
:1040000098731F46C2F2000740F268700646C2F27B
:10401000000640F23451C2F20001029101F01EF894
:104020003A68002AFAD014E1A359002B51D028464F
:10403000FFF742FE029962586050904349D0A3595D
:1040400010EA030245D0039991F800E046F6404992
:10405000C0F601094FEA451840F22451C2F20001AE
:104060004FF6FF7C46F6383AC0F6010A40F2507B24
:10407000C2F2000B204674468646C2F1000313408C
:1040800022EA03021CB95EF80B0003421ED1180E8F
:1040900004D01AF8003003F118030DE0180C04D016
:1040A0001AF8003003F1100306E0180A1ABF1AF8D4
:1040B000003008331AF80330434419F8033031F85C
:1040C000130060451CBF013021F81300002AD4D131
:1040D000744605F1010504F10404062DA4D1019DE7
:1040E0006A1E019240F0AC8003990C7804F101043F
:1040F000E3B20B700B2B03D14FF000050D7002E003
:10410000002B40F09A8040F28072C2F200021168E7
:1041100091B16FEA010433682340336040F250707C
:10412000C2F2000005682C40046040F28071C2F2C7
:1041300000014FF000020A6040F28074C2F20004F5
:10414000636893B16FEA030075680540756040F2DB
:104150005072C2F2000251680840506040F2807410
:10416000C2F200044FF00003636040F28070C2F2BC
:104170000000856895B16FEA0504B2682240B2601C
:1041800040F25073C2F2000399680C409C6040F208
:104190008070C2F200004FF00005856040F280742C
:1041A000C2F20004E26892B16FEA0203F1681940BA
:1041B000F16040F25070C2F20000C5682B40C3604D
:1041C00040F28074C2F200044FF00002E26040F25C
:1041D0008073C2F20003196991B16FEA0100356979
:1041E0000540356140F25074C2F20004226910406B
:1041F000206140F28073C2F200034FF000011961A8
:1042000040F28070C2F20000456995B16FEA050482
:1042100072692240726140F25073C2F20003596920
:104220000C405C6140F28070C2F200004FF000056B
:1042300045614FF4FA74019402E04FF4FA70019072
:104240004FF0010001F0D2F83A68002A3FF4E6AEE0
:1042500007E04FF4FA74019440F24C75C2F2000585
:1042600003954FF000042546DEE600BF10B54FF081
:10427000000440F29873C2F200031C6040F25070D8
:10428000C2F2000021464FF00602FCF743FA40F26A
:104290006870C2F2000021464FF00602FCF73AFABD
:1042A00040F28070C2F2000021464FF00602FCF797
:1042B00031FA40F23450C2F2000021464FF00602BB
:1042C000FCF728FA40F22450C2F2000021464FF0D9
:1042D00010020FF0A5FF40F24C70C2F20000047013
:1042E00010BD00BF70B546F62033C0F601031B5C5D
:1042F00046F6F022C0F6010252F8202040F29870F3
:10430000C2F20000046840F26875C2F2000555F878
:104310002300104206D104F1010640F29875C2F262
:1043200000052E6049B140F25071C2F2000151F80F
:104330002350154341F8235009E040F25071C2F276
:10434000000151F8235025EA020541F8235010439B
:1043500040F26871C2F2000141F8230040F280711E
:10436000C2F2000151F8230020EA020241F82320A2
:1043700034B940F22053C2F20003186800F0A0FEE6
:1043800070BD00BF30B446F62033C0F601031B5C9D
:1043900046F6F022C0F6010252F8202040F2687082
:1043A000C2F2000050F82300104229D040F2987465
:1043B000C2F20004256805F10105256071B140F2E3
:1043C0008071C2F2000151F82340144341F82340A8
:1043D00040F24C71C2F20001097889B96FEA020219
:1043E00040F25071C2F2000151F82340144041F8EC
:1043F0002340024040F26870C2F2000040F82320DF
:1044000030BC704730B4034640F62C02C2F20002C2
:1044100052E8000F00F1010042E80004012CF7D03F
:1044200040F22450C2F2000030F8132039B140F2BB
:104430002451C2F200014FF0000421F8134040F66D
:104440002C03C2F2000353E8004FA4F1010443E837
:104450000045012DF7D053E8004FB4F1004F0DD1C6
:104460004FF0000443E80045012DF4D04EF604500F
:10447000CEF20000016841F080510160BFF32F8F40
:10448000104630BC704700BF40F24C73C2F20003CC
:104490001878D0F1010038BF002070472DE9F84F9F
:1044A000DFF834814B4FC8EB07004FEAD00707F124
:1044B00001074FF0000540F2982AC0F6000A40F2CA
:1044C0005839C0F6000931E044464FF000066FEA63
:1044D000060B0BEB070101F0010B58F8043CAB4253
:1044E00029D135E054F8043CAB4205D154F8080C0E
:1044F0008047FDF72DF80BE0FF2B09D9FF2D07D1E1
:1045000054F8040C4FF0070154F8082C00F030FF69
:1045100006F1010604F1080454F8041CA94240D134
:104520004CE005F10105B5F5807F02D0CA45CBD33B
:10453000F7E7BDE8F88FFF2B0FD9FF2D0DD158F805
:10454000040C4FF0070158F8082C00F011FF04E0AC
:1045500058F8082C9047FCF7FBFF06F1010604F120
:104560000804BE42DDD0BBF1000FBBD054F8040CF0
:10457000A8420AD0FF280DD9FF2D0BD14FF007011B
:1045800054F8082C00F0F4FE04E054F8081C8847A6
:10459000FCF7DEFF06F1010604F10804BE42A1D1DA
:1045A000BFE7FF290FD9FF2D0DD154F8040C4FF0B0
:1045B000070154F8082C00F0DBFE04E054F8082C46
:1045C0009047FCF7C5FF06F1010604F10804BE425E
:1045D00088D1A6E75F030008A0020008027840F631
:1045E0000003C2F200031B789A4206D34FF0000288
:1045F0000270087800F1010008700A7840F60103A3
:10460000C2F200031878824224BF0020087070476D
:1046100010B5A0F10803052B3DD8DFE803F01F3CDF
:104620002C3C038340F2A070C2F200004FF0200146
:104630004FF054020FF0F4FD40F2F470C2F20000AB
:104640004FF0FF314FF00C020FF0EAFD40F604008E
:10465000C2F20000026802F1010202604FF00001A4
:1046600040F29C73C2F20003197040F29D70C2F2D6
:104670000000017056E040F29C71C2F200014FF060
:1046800000030B7040F29D70C2F20000027802F14C
:10469000010202703CE040F29C72C2F20002127809
:1046A00040F29D71C2F200010B7840F60001C2F2A7
:1046B0000001097801FB032340F2A071C2F200015E
:1046C000C95C81421DD040F2A074C2F20004E054E3
:1046D0004FEA531040F2F471C2F2000103F01F03DD
:1046E0004FF0010404FA03F351F820401C4341F851
:1046F000204040F60400C2F20000016801F101010F
:10470000016002F1010240F29C73C2F200031A70D0
:1047100040F29C70C2F2000040F29D71C2F20001B2
:10472000FFF75CFF4FF0000010BD00BF062818D84F
:10473000002808BF052046F60053C0F6010313F811
:10474000101040F60002C2F20002117003EB4000AC
:10475000417840F60103C2F2000319704FF00100E6
:1047600070474FF00000704708B54FF00500FFF7A5
:10477000DDFF4FF00C004FF00001FFF749FF08BDCF
:1047800008B540F29C72C2F20002107040F29D73B4
:10479000C2F20003197010461946FFF71FFF08BD4B
:1047A000034628B140F60000C2F2000000781870FD
:1047B00029B140F60103C2F20003187808702AB14B
:1047C00040F60401C2F200010B68136040F2A070D1
:1047D000C2F20000704700BF2DE9F00140F2A0775F
:1047E000C2F200073F1853284BD8002A49D03B4655
:1047F00007F1010702F1FF3257FA82F74FF0000686
:1048000040F2F474C2F200044FF001056FEA030CA9
:104810000CEB070202EA050C13F8018B01F1FF31E2
:1048200011F8012F90452FD13DE013F801CB01F194
:10483000010049788C450ED003F8011C4FEA521153
:1048400002F01F0605FA06FC54F821604CEA060641
:1048500044F821602E4602F10102D2B2542A07D058
:1048600013F801CB00F101014078844542D150E0BA
:104870003EB140F60403C2F20003196801F10101E0
:104880001960BDE8F001704703F8012C4FEA50169B
:1048900000F01F0805FA08F854F8262048EA02023A
:1048A00044F826202E4600F10100C2B2542ADFD07F
:1048B000BB42DDD0BCF1000FB7D013F801CB11F82B
:1048C000010F84450ED003F8010C4FEA521002F09C
:1048D0001F0605FA06FC54F820604CEA060644F868
:1048E00020602E4602F10102D2B2542AC0D0BB424F
:1048F0009BD1BDE703F8010C4FEA521002F01F06EE
:1049000005FA06FC54F820604CEA060644F82060DC
:104910002E4602F10102D2B2542AA9D0BB4284D160
:10492000A6E700BF034628B10868834214BF0020F1
:10493000012070474FF00000704700BF10B440F6F0
:104940002C03C2F2000353E8002F02F1010243E8F6
:1049500000210129F7D00468C4B16268824202D103
:104960009268626002E043688168996023688342CC
:1049700002D15B68236002E0826841685160A268EE
:1049800002F1FF31A1604FF00004046040F62C03F7
:10499000C2F2000353E8002FA2F1010243E8002411
:1049A000012CF7D053E8002FB2F1004F0DD14FF09A
:1049B000000243E80024012CF4D04EF60450CEF25D
:1049C0000000016841F080510160BFF32F8F10BCDF
:1049D000704700BF38B504460D464FF000014FF058
:1049E00010020FF01DFCE56038BD00BFF8B50446AD
:1049F0000F46C6688D192946FFF794FF00283CD161
:104A000040F62C03C2F2000353E8002F02F101022A
:104A100043E800210129F7D04FF000006860616889
:104A2000A96001B14D60226802B925606560BC5182
:104A3000A36803F10103A36040F62C03C2F2000354
:104A400053E8002FA2F1010243E80024012CF7D023
:104A500053E8002FB2F1004F0DD14FF0000243E8B0
:104A60000024012CF4D04EF60450CEF20000016870
:104A700041F080510160BFF32F8FF8BD2DE9F04167
:104A800004468846C6688D199719C2B940F62C03AA
:104A9000C2F2000353E8002F02F1010243E80021B3
:104AA0000129F7D002686A6005604FF00000A86035
:104AB000616809B9656020E06B689D601DE039465A
:104AC000FFF730FF00283FD02846FFF737FF40F6BA
:104AD0002C03C2F2000353E8002F02F1010243E865
:104AE00000210129F7D0B868A8606F60BD60216817
:104AF000B9420EBF2560A9684D6048F80640A2681B
:104B000002F10102A26040F62C03C2F2000353E856
:104B1000002FA2F1010243E80024012CF7D053E852
:104B2000002FB2F1004F0DD14FF0000243E80024F6
:104B3000012CF4D04EF60450CEF20000016841F092
:104B400080510160BFF32F8FBDE8F081C368C918A1
:104B5000486808B1C01A70474FF00000704700BFA6
:104B6000036813B1C068181A70474FF0000070470F
:104B700008B5C368C918FFF7D5FE08BD08B5C068F9
:104B80000818FFF7DBFE08BD08B540F60800C2F2C2
:104B900000004FF01C01FFF71DFF08BD70B5054672
:104BA00000F108063046FFF7DBFF0446686050B1AD
:104BB00030462146FFF7E2FF4FF00100A861204692
:104BC00000F07EFA70BD4FF00003AB6170BD00BF16
:104BD00038B504460D464FF000014FF028020FF0A3
:104BE0001FFB204640F8085B4FF01C01FFF7F2FE68
:104BF00040F60800C2F200002146FFF7F7FE38BD7C
:104C00002DE9F0410746884643F29043C2F2000383
:104C10001868002800F0FE8040F62C04C2F2000460
:104C200054E8002F02F1010244E800210129F7D0E5
:104C3000796831B143F29042C2F20002136899429E
:104C40002ED143F29040C2F2000004687C60B96942
:104C500001F10101B96140F62C03C2F2000353E8EF
:104C6000002FA2F1010243E80024012CF7D053E801
:104C7000002FB2F1004F0DD14FF0000243E80024A5
:104C8000012CF4D04EF60450CEF20000016841F041
:104C900080510160BFF32F8F4FF00100BDE8F0811C
:104CA000B8F1FF3F24D140F62C03C2F2000353E8D1
:104CB000002FA2F1010243E80024012CF7D053E8B1
:104CC000002FB2F1004F0DD14FF0000243E8002455
:104CD000012CF4D04EF60450CEF20000016841F0F1
:104CE00080510160BFF32F8F4FF00000BDE8F081CD
:104CF00007F108052846FFF733FF0246F0B143F2FB
:104D00009046C2F20006306892F8294090F82910C7
:104D10008C4208D912E0336892F8290093F82940B0
:104D2000A04204D90AE043F29046C2F200062846A7
:104D30001146FFF70BFF02460028ECD1284643F24C
:104D40009041C2F200010968FFF798FE40F62C0678
:104D5000C2F2000656E8002FA2F1010246E8002444
:104D6000012CF7D056E8002FB2F1004F0DD14FF0D3
:104D7000000246E80024012CF4D04EF60450CEF296
:104D80000000016841F080510160BFF32F8FB8F13E
:104D9000000F04D008EB880000F028FB01E000F0D1
:104DA0005DF940F62C04C2F2000454E8003F03F120
:104DB000010344E80032012AF7D043F29046C2F2E0
:104DC000000628463168FFF7D9FE54E8003FA3F1FA
:104DD000010344E80032012AF7D054E8003FB3F160
:104DE000004F0DD14FF0000344E80032012AF4D007
:104DF0004EF60450CEF20000016841F0805101608F
:104E0000BFF32F8F78683268904214BF00200120D2
:104E1000BDE8F0814FF00100BDE8F08110B5044617
:104E200043F29043C2F200031868002860D0626821
:104E3000904201D0FBF70CFC40F62C03C2F20003B9
:104E400053E8002F02F1010243E800210129F7D0C5
:104E5000A16901F1FF30A06118B340F62C03C2F242
:104E6000000353E8002FA2F1010243E80024012CC3
:104E7000F7D053E8002FB2F1004F0DD14FF00002F0
:104E800043E80024012CF4D04EF60450CEF200008A
:104E9000016841F080510160BFF32F8F4FF0000097
:104EA00010BD2046FFF77AFE40F62C03C2F2000345
:104EB00053E8002FA2F1010243E80024012CF7D0AF
:104EC00053E8002FB2F1004F0DD14FF0000243E83C
:104ED0000024012CF4D04EF60450CEF200000168FC
:104EE00041F080510160BFF32F8F4FF0010010BDE2
:104EF0004FF0010010BD00BFF8B5054640F62C0389
:104F0000C2F2000353E8002F02F1010243E800213E
:104F10000129F7D040F60800C2F20000FFF720FE9A
:104F20000446E0B140F60807C2F200076068A842F4
:104F300003D12046FFF732FE0AE004F108063046AE
:104F40002946FFF715FE18B130462946FFF716FE31
:104F500038462146FFF7FAFD04460028E6D140F620
:104F60002C03C2F2000353E8002FA2F1010243E830
:104F70000024012CF7D053E8002FB2F1004F0DD1DF
:104F80004FF0000243E80024012CF4D04EF6045008
:104F9000CEF20000016841F080510160BFF32F8F15
:104FA000F8BD00BF08B546F60C53C0F60103195C06
:104FB000012906D011B102290BD105E0FEF768F8EE
:104FC00008BD02F001F908BDFBF742FB4FF00000FD
:104FD00008BD4FF0000008BD4EF60453CEF20003AA
:104FE0001A6842F080501860704700BF4FF001020D
:104FF00080F8282040F62803C2F2000390F8291018
:1050000002FA01F2188802431A80704710B440F681
:105010002403C2F200031A68C2B1904213D104E023
:1050200088420FD102F1140203E040F62402C2F2DA
:10503000000243691BB19C698169611899614369E8
:10504000136003E00A4651690029E9D14FF00002DC
:1050500082614FF0FF31416110BC704710B5FBF722
:105060009FFB044643F29043C2F20003186890F895
:105070002820032A1BD0FBF793FB43F29043C2F294
:10508000000319684FF0000281F8282091F82920C8
:10509000096940F61813C2F2000343F82210FBF727
:1050A00089FB2046FBF786FBFFF796FF10BD4FF00C
:1050B000020180F828102046FBF77CFB10BD00BFE2
:1050C00038B5044690B3036883B3FBF769FB054624
:1050D00094F8280010BB2046FFF788FF43F2904168
:1050E000C2F200010B6843B194F8292093F829001B
:1050F00020F00101531A002B15DA40F62C02C2F2FF
:105100000002106838B140F0004140F62C03C2F2B2
:105110000003196007E0FFF75FFF04E0022804BF07
:10512000032084F828002846FBF744FB38BD00BF65
:105130002DE9F04F85B006460F46934698460F9DE1
:10514000DDF84090FBF72CFB824640F67003C2F27C
:1051500000031968504881420FD248F20002C2F29F
:10516000000252F82C4C54B14C4B1C468B4207D9D0
:1051700053F82C090028F8D102E0474C00E0464CD7
:10518000A14206D1A1F12C0140F67002C2F2000248
:10519000116020464FF000014FF02C020FF040F854
:1051A0004FF0FF3161611EB946F61066C0F6010688
:1051B0002660B8F1000F08D00E9B042B08D91846C2
:1051C00000F103004FEA900604E04FF0000601E012
:1051D0004FF000060DBB43F69479C2F2000940F689
:1051E0001805C2F20005296845F24D60C0F60000BE
:1051F0000090CDF80480029648464FF000025B46CE
:10520000FBF706FE2A68A260E0604FEA80015318AF
:105210002B60C1EB0900606020E028464FF0FF31B1
:105220004A46FBF777FA4AF2ED52CDF6CE622A6093
:10523000E56005EB8905656045F24D61C0F600014A
:105240000091CDF804800296284629464FF00102CD
:105250005B46FBF7DDFDA5EB800363606FEA0702A9
:10526000C2F3C01101EB470707F0FF0784F829706C
:1052700040F63003C2F2000353F82700206143F8E0
:1052800027405046FBF796FA2046FFF719FF2046C5
:1052900005B0BDE8F08F00BFD47F0020A87F0020BC
:1052A00030B585B04FF0000143F29043C2F20003E5
:1052B0001960284C48F20005C2F200052A1B20465E
:1052C0004FEAA202FBF726FA40F61800C2F20000ED
:1052D0000460A5F12C0540F67001C2F200010D60DA
:1052E00043F29473C2F200034FF0B504CBF26B1497
:1052F0001C6003F14C004FF0FF3243F8042F43F8D9
:10530000042F43F8042F8342F9D14FF00004009496
:1053100040F67401C2F2000101914FF0280302939C
:1053200046F61C60C0F601004FF0070145F2CD3291
:10533000C0F600022346FFF7FBFE40F61412C2F24D
:105340000002106040F63000C2F20000C46305B0F5
:1053500030BD00BF983F002010B584B0069C00947B
:105360004FF0000401940294FFF7E2FE04B010BD78
:1053700000B585B04FF00003009301930293FFF74F
:10538000D7FE05B000BD00BF38B543F29043C2F26E
:1053900000031868C0B1FBF703FA054643F29044D6
:1053A000C2F200042068FFF721FE216891F829204D
:1053B000086940F61813C2F2000343F82200284699
:1053C000FBF7F8F9FFF708FE38BD00BF38B543F228
:1053D0009045C2F2000540F63004C2F200042B688A
:1053E00022681A61FFF7D0FFF9E700BF38B543F232
:1053F0009043C2F200031968002900F0918020B99F
:10540000FFF7C2FF4FF001029AE0B0F1FF3F04D175
:10541000FFF724FE4FF0000292E040F62C04C2F2A7
:10542000000454E8002F02F1010244E800210129A0
:10543000F7D040F62402C2F200021568002D7AD09F
:10544000AB6998426FD3C01A05F114016D691DB1A3
:10545000AB698342F7D96AE043F29045C2F2000596
:105460002B689861086858611846FBF7F5F840F614
:105470002C04C2F2000454E8003FA3F1010344E805
:105480000032012AF7D054E8003FB3F1004F0DD1AC
:105490004FF0000344E80032012AF4D04EF60450E5
:1054A000CEF20000016841F080510160BFF32F8F00
:1054B000FFF7D4FD54E8003F03F1010344E8003254
:1054C000012AF7D028684169B1F1FF3F04D0FFF706
:1054D0009DFD4FF0000201E04FF0010240F62C0369
:1054E000C2F2000353E8004FA4F1010443E8004571
:1054F000012DF7D053E8004FB4F1004F0DD14FF01C
:10550000000443E80045012DF4D04EF60450CEF2DD
:105510000000016841F080510160BFF32F8F0FE060
:105520004FF001020CE040F62401C2F20001AC6928
:10553000221AAA6190E740F62401C2F200018BE72B
:10554000104638BDF8B5044600287AD0FBF728F994
:10555000064640F67003C2F20003196839488142DA
:1055600011D248F20002C2F2000252F81C5CA542BD
:1055700063D0354B1D468B4205D9A3F12C03D86B64
:10558000A042F7D15AE094F8293040F63002C2F236
:10559000000252F82300A04206D1016940F6300211
:1055A000C2F2000242F823102046FFF72FFD2046EA
:1055B000FFF7A2FC94F82900236940F61811C2F203
:1055C000000141F8203043F29042C2F2000210681C
:1055D000A04229D0A06838B3E76800EB870540F601
:1055E0001807C2F200073B685A1B29464FEAA2027D
:1055F0004FF00003FCF7C8FBE1683868A0EB8103BB
:105600003B6040F67002C2F2000211680D4B9942F5
:105610000AD29A68954203D8E068A2EB80029A60A9
:10562000A3F12C038B42F4D84FF00001216084F8E1
:1056300028103046FBF7BEF8F8BD024D21692961FC
:10564000A1E7F8BDD47F0020A87F002000BFF0476D
:1056500072B643F29044C2F200042068FFF772FF72
:105660004FF000032360FBF723FC00BF40F6240348
:10567000C2F20003196849B1886950B100F1FF32E4
:105680008A61D2F1010038BF002070474FF000005E
:1056900070474FF00000704770B540F62403C2F227
:1056A00000031C68A4B1A06990B940F62405C2F2B9
:1056B00000054FF0FF3660692946FAF7CDFF6661B5
:1056C0002046FFF7FDFC2C6814B1A1690029F2D037
:1056D00070BD00BFF0B472B640F62803C2F20003FA
:1056E0001C882CB940F61413C2F2000318685FE05E
:1056F00046F6105CC0F6010C40F61815C2F2000523
:1057000040F63006C2F20006C4F1000323401A0A34
:105710001ABF1CF8021008311CF8031011F0010F19
:105720000AD141F0010055F8200038B190F8282046
:10573000012A38D81F4602E01F4600E01F4655F8F0
:105740002120B2B192F828307BB140F62800C2F295
:105750000000048010462BE090F8283033B140F66A
:105760002802C2F20002148022E0104600690028DC
:10577000F2D156F82100824207D1BC43C4D140F691
:105780002801C2F200010C80ACE745F8210011F0BD
:10579000010FD4D114EA4703D1D04FEA4707BFB273
:1057A00041F00101CBE740F62801C2F200010C8074
:1057B00062B6F0BC704700BF70B543F29043C2F2CE
:1057C00000031B6883420FD193F82820012A9CBF55
:1057D000022283F8282093F8291040F61810C2F20C
:1057E000000040F8213070BD40F61C02C2F20002F9
:1057F000136043F29041C2F20001086090F8292042
:1058000040F61813C2F2000343F8220090F8281063
:1058100001299CBF022180F828108268AAB9C168BA
:105820004AF2ED53CDF6CE630868984201D0FAF7FC
:105830000FFF43F29042C2F2000211684868CB6841
:1058400098427ED2FAF704FF70BD40F62003C2F200
:1058500000031B68984274D093B3586843F694745D
:10586000C2F20004251A4FEAA501D96043F29472EE
:10587000C2F2000290420AD34FF0B503CBF26B1391
:1058800043F29470C2F2000004689C4201D0FAF71F
:10589000DFFE40F62005C2F200052A6840F6180433
:1058A000C2F2000420685168D2684FF00003FCF790
:1058B0006BFA296823688B60C86803EB800222605A
:1058C00043F29041C2F200010B6840F62000C2F2A0
:1058D00000000360DA68002A33D0586899684FF0F6
:1058E0000103FCF751FA43F29046C2F20006356814
:1058F000A868EC6800EB840440F61806C2F20006C3
:105900003268131B21464FEAA3024FF00003FCF755
:105910003BFAE9683068A0EB8102326040F6700320
:10592000C2F200031968074B99420AD29A6894425E
:1059300003D8E868A2EB80029A60A3F12C038B42A3
:10594000F4D870BDD47F002000B585B040F6B420F7
:10595000C2F200004FF00001FFF73CF840F65C1087
:10596000C2F200004FF00001FFF734F84FF00003DF
:10597000009340F67412C2F2000201924FF0500000
:10598000029046F62460C0F60100194645F69D4295
:10599000C0F60002FFF7CCFB40F65813C2F200033A
:1059A000186005B000BD00BF08B5FFF7D9F8034681
:1059B00048B1C06850B100F1FF31D960D1F10100A8
:1059C00038BF002008BD4FF0000008BD4FF00000B8
:1059D00008BD00BF70B505460E46144640F62C03C0
:1059E000C2F2000353E8002F02F1010243E8002154
:1059F0000129F7D0FFF7B4F80246002839D0C06873
:105A000084422DD3241A28461146FFF79FF80246F8
:105A100000282ED0C068A042F4D921E040F62C0323
:105A2000C2F2000353E8002FA2F1010243E8002470
:105A3000012CF7D053E8002FB2F1004F0DD14FF0F9
:105A4000000243E80024012CF4D04EF60450CEF2BC
:105A50000000016841F080510160BFF32F8F70BDDD
:105A6000F460D1680B1BD36028463146FFF706F877
:105A7000D4E7F46028463146FEF7B8FFCEE700BF12
:105A8000F8B50646FFF76CF80446F8B1C368EBB901
:105A900030462146FFF75AF80546FAF781FE0746D9
:105AA00030462146FFF76AF83846FAF783FE226946
:105AB0001AB130462146FFF78DFF04F11400FEF7BE
:105AC00035F81DB12C46E8680028E1D0F8BD00BFCC
:105AD00008B540F67013C2F200031A6802F1010221
:105AE0001A6040F65C10C2F20000FFF75DFF28B1BB
:105AF00040F65C10C2F20000FFF7C2FF08BD00BF15
:105B000008B5014640F6B420C2F20000FFF730F8B5
:105B100020B140F6B420C2F2000008BD40F65C108F
:105B2000C2F2000008BD00BF70B5044640F62C0369
:105B3000C2F2000353E8002F02F1010243E8002102
:105B40000129F7D0FFF7DCFF05462146FFF710F8E3
:105B5000002845D040F62C00C2F2000050E8002F8B
:105B600002F1010240E800210129F7D02846214630
:105B7000FEF7ECFF18B1C168E2688B18C360FAF752
:105B80000FFE064628462146FEF7F8FF3046FAF794
:105B900011FE4FF0FF35E56040F62C03C2F2000322
:105BA00053E8002FA2F1010243E80025012DF7D0B0
:105BB00053E8002FB2F1004F0DD14FF0000243E83F
:105BC0000025012DF4D04EF60450CEF200000168FD
:105BD00041F080510160BFF32F8F4FF0010501E0CC
:105BE0004FF0000504F11400FDF79AFF40F62C0376
:105BF000C2F2000353E8002FA2F1010243E800249F
:105C0000012CF7D053E8002FB2F1004F0DD14FF027
:105C1000000243E80024012CF4D04EF60450CEF2EA
:105C20000000016841F080510160BFF32F8F2846CA
:105C300070BD00BF2DE9F04105460F461446984659
:105C4000FFF772FF064694B19DF82030002B14BF79
:105C500020460020286105F114004146069A079B62
:105C6000FDF744FF384629462246FFF7B3FE30468B
:105C7000BDE8F08170B584B00E4615460093089CCF
:105C800001949DF82430029340F6B421C2F2000141
:105C900032462B46FFF7CEFF04B070BD00B583B08F
:105CA0004FF0000300934FF00100019040F6C42034
:105CB000C2F2000041F288314FF0FF0245F6D123D5
:105CC000C0F60003FFF7D6FF40F6B424C2F200048A
:105CD000FFF7E2FC2046FFF7D3FEFFF7BFF9F7E737
:105CE00040F66C13C2F2000318681A689042FBD1A8
:105CF000704700BF10B540F66C13C2F200031A687B
:105D000002F101021A60FFF7B1FC044640F6B4202C
:105D1000C2F20000FFF748FE204310F0FF0F06D04C
:105D200040F65810C2F200000068FFF7C9F910BD34
:105D300008B546F64860C0F601004FF0060146F28D
:105D40006D12C0F60002FFF713FB40F62833C2F2D3
:105D50000003186008BD00BF38B504460D4640F684
:105D60006C33C2F20003586AA0420AD040F66C318C
:105D7000C2F200014C620A681AB115B14948FDF738
:105D8000D5FE40F66C33C2F20003186F84420AD08D
:105D900040F66C31C2F200010C67CA6C1AB115B141
:105DA0004148FDF7C3FE40F66C33C2F20003D3F85E
:105DB000BC0084420CD040F66C31C2F20001C1F844
:105DC000BC40D1F898201AB115B13848FDF7AEFEA5
:105DD00040F66C33C2F20003D3F8080184420CD0C1
:105DE00040F66C31C2F20001C1F80841D1F8E4205C
:105DF0001AB115B12E48FDF799FE40F66C33C2F288
:105E00000003D3F8540184420CD040F66C31C2F246
:105E10000001C1F85441D1F830211AB115B125481B
:105E2000FDF784FE40F66C33C2F20003D3F8A00104
:105E300084420CD040F66C31C2F20001C1F8A0419E
:105E4000D1F87C211AB115B11B48FDF76FFE40F661
:105E50006C33C2F20003D3F8EC0184420CD040F65C
:105E60006C31C2F20001C1F8EC41D1F8C8211AB17D
:105E700015B11248FDF75AFE40F66C33C2F200032A
:105E8000D3F83802A0420CD040F66C31C2F20001C7
:105E9000C1F83842D1F814221AB115B10848FDF7FB
:105EA00045FE38BD7C0B0020C80B0020140C0020E0
:105EB000600C0020AC0C0020F80C0020440D0020E9
:105EC000900D00202DE9F04707460D4691460898B1
:105ED000DDF828800C683E68D8F800108A199442D2
:105EE00002D80219964203D304192C60BDE8F0874A
:105EF000341B061BB14234BF8A46B246099931B100
:105F0000D9F800000818191952460EF065F9D8F8AA
:105F10000030CAEB0302C8F800203E6806EB0A0115
:105F20003960D9F8000000EB0A03C9F800302E6888
:105F3000A41954442C60BDE8F08700BF70B584B04C
:105F40009CF81960157A947B4FF007038CF8103099
:105F50004FF005028CF8112006F00F0260F3C71213
:105F60008CF812204FF0000065F301008CF813004C
:105F70004FF0000261F30A02ACF814208CF81640CE
:105F8000DCF80C100093DCF804300193CDF808C065
:105F900001F104000CF108020CF11003FFF792FF6D
:105FA00004B070BD2DE9F04F8FB00746059114463F
:105FB0004FF000030793136012896068131A8B4235
:105FC00038BF05930599002900F0AA8040F6643592
:105FD000C2F200052D6815B34FEAC5054FF0000267
:105FE0004FF0FF01134640F6E450C2F20000A5F165
:105FF0000806C6F3C00E1658F6798E4240F095801A
:1060000096E01658F6798E421CBF0133314602F1F4
:1060100008028658F6798E4240F09F80A0E04FF04B
:10602000000303EB43024FEAC20000F110000890A6
:106030004FF48071ADF824104FF00402ADF8262023
:106040008DF828300DF129004FF000014FF00702C4
:106050000EF0E6F804F1040B04944FF010030093E3
:10606000019705A802905846214607AA08ABFFF7FA
:1060700029FF0599002951D04FF001028DF8212008
:106080000DF132004FF000014FF006020EF0C8F89B
:1060900040F66433C2F20003186800283ED04FF087
:1060A000FF014FF0000440F6E459C2F2000946F641
:1060B0006868C0F6010840F6643AC2F2000A59F86E
:1060C0003450ED798D4223D08DF820404FEA0516EB
:1060D0000DF1220008EB06014FF008020EF07CF8EB
:1060E00006F108010DF12A0041444FF008020EF0BC
:1060F00073F84FF018020092019705AB02935846CF
:10610000049907AA08ABFFF7DDFE059830B12946D0
:1061100004F10104DAF80020A242D0D8079801E087
:106120004FF0FF300FB0BDE8F08F03F101033146AF
:1061300002F10802AA423FF474AFBEF1000F3FF42F
:1061400060AF1658F6798E421CBF0133314602F11A
:106150000802AA427FF455AF63E703F10103314619
:1061600002F10802AA427FF44CAF5AE72DE9F04150
:106170004FF00100FDF7D2FB46F65860C0F6010073
:10618000FDF748FA40F65433C2F200034FF0010223
:106190001A7040F65030C2F20000016841B940F672
:1061A0005034C2F20004FEF759FF2568002DFAD0E2
:1061B00040F66137C2F2000740F65434C2F20004E0
:1061C00040F66036C2F2000640F6CC55C2F2000539
:1061D00040F6E058C2F200083B783BB14FF00002B5
:1061E0003A704FF002002070FDF7E0F9317859B1B4
:1061F0004FF000033370227862F07F0020704FF080
:1062000001000146FFF7A8FD297851B14FF00000C9
:106210002870237803F07F0222704FF00101FFF70E
:106220009BFD98F8000010B9FEF718FFD4E740F680
:106230005431C2F200014FF002030B704FF0000026
:10624000FDF76CFBBDE8F08108B540F65033C2F2B3
:106250000003186040F62830C2F200000068FEF724
:106260002FFF08BD70B505460E4640F66833C2F2F2
:1062700000031868032801D9FAF7EAF940F66832F2
:10628000C2F20002116840F63034C2F2000444F851
:10629000316004EBC104656001F10101116070BD62
:1062A00070B505460C461646032801D9FAF7D0F911
:1062B00040F6E453C2F2000353F8350008B1FAF790
:1062C000C7F940F6E451C2F2000141F8354001EB54
:1062D000C5056E6040F66433C2F200031A6802F12D
:1062E00001021A60206930B1FDF794F904F1040449
:1062F00020690028F8D170BD08B540F66C33C2F2B1
:106300000003196881425AD040F66C32C2F2000292
:10631000D36C834234D040F66C31C2F20001D1F824
:10632000982082422FD040F66C33C2F20003D3F89B
:10633000E41081422AD040F66C32C2F20002D2F858
:106340003031834225D040F66C31C2F20001D1F8E1
:106350007C21824220D040F66C33C2F20003D3F895
:10636000C81181421BD040F66C32C2F20002D2F852
:106370001432834216D0FAF76BF94FF0080013E09D
:106380004FF0010010E04FF002000DE04FF003006D
:106390000AE04FF0040007E04FF0050004E04FF082
:1063A000060001E04FF0070040F66C31C2F2000138
:1063B0004FF04C0202FB001090F8200008BD4FF097
:1063C0000000F1E72DE9F04F8FB0089007910A9295
:1063D0004FF0000309931360546813891B1B8B4211
:1063E00038BF07930799002900F04A81082C69D823
:1063F00040F66434C2F20004D4F800E040F6683598
:10640000C2F200052E680EEBCE0707EBC60404F1BE
:1064100009044FF0000140F6E457C2F20007CB59DF
:106420008BB1DD68641903F110051B695BB15E89EE
:106430000EB104F107049B890BB104F1070455F870
:10644000043F002BF3D101F108012029E7D140F6E8
:106450005031C2F200010D682F7E6E7EEB8A03F18F
:106460000103C3F347054FF000010C914FF00903FE
:106470008DF82C304FF002018DF82D10ADF82E4024
:106480008DF830E04FF001018DF831104FF0000130
:1064900067F3451166F3861161F07F018DF83310C3
:1064A0008DF834500093019007A8029002F1040087
:1064B000114609AA0BABFFF705FD079A002A00F069
:1064C000DD80E0E04FF009001060DCE05BF8364072
:1064D000002C00F0CE80059D286800284BD07A68FB
:1064E000B2420CD04FF0000310F0010F3ED1DFE0BC
:1064F00007EBC3025268B24240F0E38001E04FF084
:10650000000357F83300D2B290F8048090F805C029
:1065100090F806E0C579016819B143F01000C3B2E4
:1065200001E04FF000034FF008008DF82C004FF011
:106530000B018DF82D108DF82E208DF82F808DF801
:1065400030C08DF831E08DF832508DF833300A9933
:106550000090089A019207AB029301F1040009AA86
:106560000BABFFF7AFFC079828B987E003F10105F3
:106570002B468542BCD104F1100523697BB1294625
:106580004FF00002588908B102F101029B890BB15A
:1065900002F1010251F8043F002BF3D101E04FF06A
:1065A00000025FFA86FCD2B294F804E06079A17927
:1065B00023681BB146F02003DBB201E04FF000037B
:1065C0008DF82CA04FF004088DF82D808DF82EC08A
:1065D0004FF0000C8DF82FC08DF830208DF831E091
:1065E0008DF832008DF833108DF834300A99CDF8DB
:1065F00000A0089A019207A8029001EB080009AADE
:106600000BABFFF75FFC0799002937D0A3686BB18C
:106610000A99E26800920898019007AA029201EB99
:10662000080009AAFFF74EFC079B3BB3246904B39B
:106630004FF001084FF000092046FFF75DFE8DF88E
:106640003500618939B10DF11C0C40462246FFF737
:1066500075FC079991B1A18939B10DF11C0C48461F
:106660002246FFF76BFC079840B155F8044F002C09
:10667000E2D106F10106042E7FF428AF099814E058
:106680004FF0FF3011E04FF0000640F6E45BC2F23D
:10669000000B40F66834C2F2000405944FF0090A7A
:1066A00040F63037C2F2000710E70FB0BDE8F08FB8
:1066B00003F1010307EBC3014A68B2427FF456AF0E
:1066C0001FE705F1010307EBC3014A68B2427FF4FB
:1066D0004DAF16E708B540F6D053C2F200031A5C7E
:1066E00040F66C31C2F200014FF04C0000FB02108A
:1066F000436AD3F1010238BF002242634FF0000128
:10670000C1630164416400F11000FDF70FFA08BD98
:106710002DE9F04790B081468A4640F6D053C2F248
:1067200000031A5C40F66C30C2F200004FF04C04DB
:1067300004FB020404F148064FF001084FF0000783
:10674000354640463146F9F787FF28B14FF0020041
:106750003146F9F781FF36E0BAF1000F05D148461E
:106760004146FCF7F7FD032827D0256C75B1684634
:10677000A168E26BA8470546B0F1FF3F14D0606402
:10678000484669462A46FCF71DFE0EE0616CA56886
:106790008D4228BF0D464846E16B2A46FCF712FEA3
:1067A000E36B5A19E26300E03D46606CA1688842E1
:1067B0003CBFE7632764451B656438463146F9F7FB
:1067C0004BFF0228BCD010B0BDE8F087F8B50546F5
:1067D0000E46174640F6D053C2F200031A5C40F64C
:1067E0006C30C2F200004FF04C0404FB02044FF086
:1067F0000000FCF7A5FDE76326644FF0000161642B
:1068000028464FF00101FFF783FF4FF00100FCF72E
:1068100097FDF8BDF8B505460F46164640F6D0532D
:10682000C2F200031A5C40F66C30C2F200004FF076
:106830004C0404FB0204A168B1420DD243F29473EC
:10684000C2F200039F4207D343F69472C2F20002E1
:10685000974201D2F9F7FCFE4FF00000FCF770FD03
:10686000E7634FF000002064666428464FF00101A2
:10687000FFF74EFF4FF00100FCF762FDF8BD00BFCF
:1068800008B5FCF717FE08BD70B586B005460C4686
:10689000164602A8FAF762FD01462EB102A82A4662
:1068A000234600F09BFD07E04FF00103009302A890
:1068B0002A46234600F044FE06B070BD70B58AB08B
:1068C0000378212B00F0938004D86BB1012B40F0AA
:1068D000D88186E0A12B00F0A781C02B00F0B48105
:1068E000802B40F0CE8195E04178052903D009291D
:1068F00040F0CA8146E0408840F65432C2F20002BD
:106900001378022B02D0032B33D118E000F1FF31B2
:106910008AB27E2A30D8C0B240F6E153C2F20003F8
:1069200018704FF00201FCF7EDFF40F65430C2F250
:1069300000004FF0030101704FF00100C3E170B996
:1069400040F6E152C2F20002107040F65430C2F23A
:1069500000004FF0020303704FF00100B3E17F2805
:106960000DD840F6E151C2F2000108704FF001006D
:10697000A9E14FF00200A6E14FF00200A3E14FF0C1
:106980000200A0E1827840F65433C2F20003197885
:10699000022923D972B940F65433C2F200034FF0F2
:1069A000030119704FF001000146FFF7D5F94FF0D0
:1069B000010088E1012A18BF022040F0848140F6DE
:1069C0005430C2F200004FF0040202704FF0000099
:1069D0000146FFF7C1F94FF0010074E14FF00200EA
:1069E00071E140780B280CBF012002206BE1838805
:1069F000032B00F24C8140F6E454C2F2000404EB95
:106A0000C3035B68002B00F045819847002808BF4E
:106A1000022058E142781AB1062A40F03E8121E076
:106A2000C18802291BD14FF00000ADF8040040F6E8
:106A30005032C2F2000212680346517E61F3000335
:106A4000ADF80430127E62F341030AA921F8243D17
:106A50004FF00202FFF7DEFE4FF0030033E14FF08C
:106A6000020030E18278C1888CB2C378022B2ED02C
:106A7000032B3DD0012B40F0D48040F6E825C2F234
:106A80000005284646F63461C0F601014FF01202B7
:106A90000DF0A2FB40F65030C2F2000001688A8976
:106AA0002A81CB896B81088AA8818A7C2A71CB7C58
:106AB0006B71097DA9714FF000002946122C34BF7B
:106AC00022461222FFF7A6FE4FF00300FBE040F63D
:106AD0000462C2F2000211814FF00000506046F2E1
:106AE000C531C0F60001FFF771FE4FF00300EAE088
:106AF000D2B940F6E824C2F2000404F1020046F6DE
:106B00003061C0F601014FF002020DF065FB4FF05D
:106B1000040222704FF0030565704FF0000021461B
:106B2000FFF778FE2846CEE0012A06D140F6503322
:106B3000C2F20003196809682FE0022A06D140F664
:106B40005032C2F200021068416826E0032A06D1E2
:106B500040F65033C2F20003196889681DE002F064
:106B60000F0022F00F03102B08D15A4B19688842EE
:106B70000EDA594A52F8300001680EE0202B07D196
:106B8000032805D8554951F8300008B1016804E0E0
:106B9000EE2A04D04FF0020095E009B93EE05049DA
:106BA000B1F1FF3F40F0888001A84FF020014FF085
:106BB0000102FFF769FE0AAD2A184FF0000002F843
:106BC000240C01A978E000F10206428003F10102E1
:106BD000134611F8015F5DB100F10400758002F108
:106BE000010311F8012F002A6FD101E04FF00003DB
:106BF00040F6E821C2F200014FF003054D7003F1A9
:106C000001034FEA4303DAB20A704FF00000A242D8
:106C100028BF2246FFF7FEFD284654E04FF0020051
:106C200051E04FF002004EE08388032B38D840F645
:106C3000E454C2F2000404EBC3035B689BB39847BF
:106C4000002808BF02203EE04378212B2ED1C188C6
:106C500040F60463C2F2000319814FF000025A604B
:106C60008088042825D1104645F6A571C0F600019C
:106C700040F60462C2F20002FFF7A8FD4FF00300E5
:106C800021E04FF002001EE04FF002001BE04FF049
:106C9000020018E04FF0020015E04FF0020012E091
:106CA0004FF002000FE04FF002000CE04FF0020046
:106CB00009E04FF0020006E00A78002A96D0094861
:106CC0004FF000037FE70AB070BD1E2B7FF47BAF4F
:106CD0008EE700BF680B0020300B0020E40D002081
:106CE0004C6E0108E80A002010B50446436993B1D0
:106CF0004FF00000606140F65431C2F200010A78A2
:106D0000032A08D140F6E153C2F2000318784FF08D
:106D10000301FCF7F7FD206958B34FF00000206134
:106D2000E06040F62C31C2F20001087040F65831A4
:106D3000C2F200014FF00802FFF7A2FD082853D16C
:106D400040F65832C2F20002137813F0800F06D1D9
:106D500040F65830C2F20000C188002944D140F604
:106D60005830C2F200004FF000010A46FFF7A6FDBE
:106D70002DE0E168002937D04FF00000E06040F6D8
:106D80002C32C2F20002137840F6E821C2F2000170
:106D9000C3F14002FFF774FD034628B340F62C30E0
:106DA000C2F2000001785A18D2B2027040F658338D
:106DB000C2F20003D888904216D140F65830C2F291
:106DC000000040F6E821C2F20001FFF777FD01283C
:106DD00004D0022808D1FCF7DBFA10BD4FF0000008
:106DE00001460246FFF716FD10BD00BF08B540F68C
:106DF0001063C2F200031B693BB14FF0000140F683
:106E00001062C2F200025269984740F61060C2F266
:106E100000004FF00001017041608160C1600161BC
:106E2000416108BD40F61060C2F20000816146F683
:106E30003871C0F601018A5C42778377037F6FF374
:106E4000070303774FF000014162704730B583B00C
:106E500040F61064C2F200042070089D6560099D30
:106E6000A5600A9DE5600B9D25610C9D65619DF8FF
:106E7000184000949DF81C400194FFF7D3FF03B025
:106E800030BD00BF40F61063C2F200035B6AB3F18D
:106E9000FF3F09D140F61061C2F200014FF000033C
:106EA0004B624FF0010070473F2B0BD840F6106249
:106EB000C2F20002106AC15403F1010353624FF0A1
:106EC000010070474FF00000704700BF704700BFDF
:106ED00070B540F61064C2F2000404F1180046F6E2
:106EE0005471C0F601014FF007020DF075F94FF033
:106EF000000046F69471C0F60101FFF7B3F947F2BE
:106F00002D16C0F600064FF0000046F63C71C0F6A4
:106F100001013246FFF7C4F946F69C75C0F601053B
:106F20004FF0010029463246FFF7BAF92869FFF70A
:106F3000E3F984F8280040F63C60C2F200004FF00C
:106F4000070146F65572C0F600024FF00003FCF749
:106F5000CDFD70BD38B540F67063C2F200034FF04E
:106F600001021A7040F61064C2F2000494F828007E
:106F70004FF000010A46FFF74DFC606868B140F62B
:106F80001064C2F200044FF0FF3565626368207838
:106F900061699847616A0029F7D040F61060C2F233
:106FA00000004FF000024262836833B140F6106186
:106FB000C2F2000108784969984738BD2DE9F047C9
:106FC000A2B0804643680BB9806828B14FF0000139
:106FD000C8F80810FFF7BEFFD8F80C20002A3ED0F2
:106FE0004FF00007C8F80C70D8F8000012A94FF055
:106FF0004002FFF745FC074640F61063C2F200036B
:10700000D86860B35FB340F61064C2F200044FF07A
:10701000000507F1FF3606F0010A20789DF84810B8
:107020002A466369E668B0474FF001094F456CD1C5
:1070300015E0E668207812AA12F809102A4663695A
:10704000B04709F10109E668207812AB13F809107E
:107050002A466369B04709F101094F45E9D1D8F8DB
:10706000140000284ED04FF0000440F67061C2F2C8
:1070700000010C70C8F8144040F64C60C2F20000E9
:10708000FEF752FD40F61062C2F2000254625368ED
:10709000002B30D040F61065C2F2000502AC2C6225
:1070A0002C46656A6268207861699047606A85420B
:1070B000F7D105B3D8F8000002A92A46FFF7AAFBCA
:1070C0004FF000010091019140F64C60C2F20000C7
:1070D0004FF04B014FF0FF0246F65573C0F6000328
:1070E000FEF7C8FD0EE040F61062C2F20002107812
:1070F0005169984706E040F61063C2F200039B68AE
:10710000002BF0D122B0BDE8F087BAF1000F90D08B
:10711000E668207812A911F809102A466369B04779
:1071200009F101094F4584D199E700BF10B54478B2
:107130000378212B02D0A12B19D10CE0202C02D0F6
:10714000222C08D119E0072A1AD10F480DF044F873
:107150004FF0010010BD212C0CD14FF000000A4966
:107160004FF00702FFF756FB4FF0030010BD4FF042
:10717000000010BD4FF0000010BD4FF0010010BD29
:107180004FF0020010BD00BF280E002008B540F6E9
:107190007063C2F20003187870B940F61061C2F251
:1071A00000014A6A72B940F61063C2F2000393F814
:1071B0002800FFF78FFA08BD40F63C60C2F20000DD
:1071C000FCF7B4FC08BD00BF46F60870C0F601002D
:1071D000704700BF70B4037801298CBF4478002445
:1071E00002298CBF85780025DCF8000048B34FEAFF
:1071F000930647F2C800C0F60100365C16704FEAED
:10720000031343EA141303F03F031B5C537001297B
:1072100007D94FEA840444EA951303F03F04205C45
:1072200001E04FF03D009070022907D905F03F05BD
:1072300047F2C803C0F60103E95C01E04FF03D01ED
:10724000D17070BC704700BF82B04FF009010CE0F4
:107250000191019B03F1FF32019233B100BF019B09
:1072600003F1FF320192002BF8D100F1FF30B0F1B1
:10727000FF3FEDD102B0704770B4C4B24FEA1020A6
:1072800046F6C876C0F6010647F25C15C0F6010561
:1072900011F8013B1AB94BB944EA00200BE06340F6
:1072A000F45C4440E85C013AF2D1F5E76340F45CF9
:1072B0004440E85CECE770BC704700BF10B444F693
:1072C000FB43C0F2861311F8014B02B9ACB380EA5C
:1072D00004404FEA400010F0807F18BF58404FEA4A
:1072E000400010F0807F18BF58404FEA400010F077
:1072F000807F18BF58404FEA400010F0807F18BFD1
:1073000058404FEA400010F0807F18BF58404FEAC5
:10731000400010F0807F18BF58404FEA400010F046
:10732000807F18BF58404FEA400010F0807F18BFA0
:107330005840002AC7D0013AC5D120F07F4010BC88
:10734000704700BF82B001909DF806304FF00000FA
:1073500063F307009DF8052062F30F209DF80420D9
:1073600062F317409DF8072012F0800F14BF63F0FE
:107370007F0103F07F0161F307004FEA4201CAB2C7
:1073800062F31F6013F0800F18BF42F0010262F336
:107390001F6002B0704700BF84B0C0F307438DF890
:1073A0000C30C0F307228DF80D20C3B24FEA1060F5
:1073B0004FEA500210F0010F14BF63F07F0103F099
:1073C0007F018DF80E1013F0800F18BF62F07F025E
:1073D0008DF80F20039804B0704700BF2DE9F04FDF
:1073E00083B005460F4614461E46019201F1FF3355
:1073F00013F1050F44D8032E43D9A6F10400C0F3BE
:1074000080080DF1040C2846FFF7E4FE05F10305A2
:10741000A7F1030104F10404A6F10406A7F104078F
:1074200017F1050F67D92CE00DF1040C28463946F9
:107430002246FFF7CFFE05F1030B5D46A7F10301DE
:1074400004F1040A5446A6F104094E46A7F10407C4
:1074500017F1050F15D80F460DF1040C584652468A
:10746000FFF7B8FE0BF10305A7F103010AF10404CD
:10747000A9F10406A7F1040818F1050F59D900E095
:10748000FFE799B396B30DF1040C28466A46FFF75F
:10749000A1FE022E11D0032E02D0012E26D11AE019
:1074A000019929B19DF8002022704FF0010301E0FD
:1074B0004FF0000304F1010401E04FF000030198D4
:1074C00030B102A9CA1812F8080C207003F10103A8
:1074D00004F1010401E04FF00003019921B102AA77
:1074E000D31813F8080C207004F101040199601AF4
:1074F00003B0BDE8F08F0F46032EC2D9B8F1000FDC
:1075000092D00DF1040C28462246FFF763FE05F1E8
:107510000305A7F1030104F10404A6F10406A7F191
:10752000040717F1050FACD80F46032E3FF67CAFCA
:10753000A7E7A7F10307032E3FF676AFA1E700BF49
:10754000F0B49DF81040ECB14FEA41079F421CD2C5
:10755000DD1B1DD056194FF030046FEA0203F318FB
:1075600003F0010302F8014BB24240F0928007E0C1
:10757000134603F8014B547003F10102B242F7D1F4
:107580003B4607E04FF0000504E04FF0000501E046
:107590004FF0000500293CD003F1FF34002B3AD016
:1075A00000F1010341182846521B04F1FF3515F084
:1075B000020F10D032E0A4F1020603F101031F46CE
:1075C000012C29D03446B44613F8016C4FEA161644
:1075D000092E42D944E01E4613F8015C4FEA151506
:1075E000092D8CBF37353035155414B900F1010021
:1075F00012E013F8016C06F00F05092D8CBF37352A
:1076000030351618757000F1020528468B42D2D12C
:1076100002E0284600E02846F0BC70471E4613F8FA
:10762000015C4FEA1515092D94BF303537351554D7
:10763000002CDBD013F8016C06F00F05092D94BF68
:10764000303537351618757000F102008B42E3D0E3
:1076500003F10103A4F10204BDE706F1300601E0E5
:1076600006F137065655BCF1000FBFD013F8016C78
:1076700006F00F06092E94BF3036373610184670C4
:1076800005F102008F42C7D003F10103A4F1020407
:10769000A1E7002B3FF46CAF02F8014BB2427FF43C
:1076A00067AF6DE7DCF8143093F8452083F8442089
:1076B000DCF8141091F8463081F84530DCF81410ED
:1076C00091F8472081F84620DCF8143083F8470011
:1076D000704700BFDCF8143093F8470093F8462059
:1076E00083F84720DCF8141091F8453081F84630D3
:1076F000DCF8141091F8442081F84520704700BF51
:1077000042F61C72C2F2000213684AF20001C0F68F
:107710000101C85CC918497803F10203136041EA0A
:1077200000207047DCF80430DCF8082002EBD300BE
:10773000CCF8080003F007014FF0010303FA01F24F
:10774000CCF80420704700BF2DE9F04F83B0044609
:107750008A4693461E46CDF804C04FF00007B8464F
:10776000B9463DE025463046D047034600283DD087
:10777000B9F1000F0CD1202829D0092829D00A28D6
:1077800029D00D2829D0022D4FF0010988BF0225EC
:10779000A3F13002D1B2092910D9A3F14100C1B23D
:1077A000052903D8A3F13703D9B207E0A3F1610299
:1077B000D0B205281AD8A3F15703D9B24FEA071758
:1077C000FCB241EA040708F101082C4606E02C4609
:1077D00004E02C4602E02C4600E02C463046D84718
:1077E000FF2CBFD004F1FF35002CBCD1DDF804C064
:1077F0003846FFF757FF019B5A69D8F1010838BF97
:107800004FF0000882F8508003B0BDE8F08F00BF51
:1078100042F6B063C2F200031B684B634BB15A6877
:10782000824209D09B684B631BB15A688242F9D1EE
:1078300002E04FF01E0070474FF00000704700BF9D
:10784000884204D8884234BF0220002070474FF09D
:1078500001007047D0F80431D0F80021934214BFE2
:10786000C05C0020704700BFD0F80431FF2B14BF6C
:1078700001330023C0F80431704700BF10B4DCF8B6
:107880001420D16C0B46044658B14FEA016343EA19
:10789000116301F47F4043EA002301F47F0143EACE
:1078A0001123DCF8040030B199B24FEA134060F3C1
:1078B0000F0361F31F435CB94FEA036141EA1361AF
:1078C00003F47F4041EA002103F47F0341EA1323DC
:1078D000D36410BC704700BFDCF80030FA2B05D829
:1078E00040F67462C2F20002D05C70474FF00000B4
:1078F000704700BFDCF8003003F10103CCF8003022
:10790000DCF8140090F8512002F1010280F85120B7
:10791000704700BF70B404460846A1B199188C4264
:1079200011D22518AA420ED294423ABFC4EB0206E5
:10793000F6B20026A94205D20019821AD31AF1180C
:10794000C8B200E0304670BC704700BFF0B583B0ED
:1079500042F6B863C2F200034FF008021A7042F612
:10796000A060C2F2000004683CB3154642F6B86756
:10797000C2F200074FF0000621680B6873B10DF1E9
:1079800007000DF1060198479DF807009DF80610C5
:1079900032463B78FFF7BEFF4519EDB26468002C14
:1079A000EAD142F6B862C2F200021078A84204D2CC
:1079B00042F6B861C2F200010D7042F6B863C2F23D
:1079C00000034FF000025A7042F6C064C2F2000495
:1079D000246834B3154642F6B867C2F2000716466B
:1079E0002068036873B10DF107000DF10601984797
:1079F0009DF807009DF8061032467B78FFF78AFF56
:107A00004519EDB26468002CEAD142F6B861C2F2C1
:107A100000014A78AA4204D242F6B860C2F20000DD
:107A2000457042F6B863C2F200034FF0010199704D
:107A300042F61874C2F2000424683CB30D4642F6C4
:107A4000B867C2F200074FF000062268136873B1EE
:107A50000DF107000DF1060198479DF807009DF80C
:107A600006103246BB78FFF755FF4519EDB2646842
:107A7000002CEAD142F6B860C2F200008178A94237
:107A800004D242F6B862C2F20002957042F6B863C0
:107A9000C2F200034FF00000D87042F62074C2F228
:107AA0000004246834B3054642F6B867C2F2000702
:107AB000064621680A6872B10DF107000DF1060152
:107AC00090479DF807009DF806103246FB78FFF7B7
:107AD00021FF4519EDB26468002CEAD142F6B86383
:107AE000C2F20003D878A84204D242F6B861C2F2CA
:107AF0000001CD7003B0F0BD42F61473C2F2000372
:107B000019684AF20000C0F60200401A704700BF30
:107B1000034610B182688A4218D042F6B463C2F2BA
:107B20000003186860B182688A4203D10BE0836861
:107B30008B420AD040680028F9D14FF0000305E0DD
:107B40004FF0000302E0034600E00346184670478A
:107B500010B540F6B874C2F200044FF4117303FB81
:107B60000044D4F80811B1F1FF3F03D0D4F8042148
:107B700091420DD123689A6A4FF0FF019047002887
:107B800034D0D4F8080100F10100C4F8080110BD98
:107B900091422BD86318197942F6A462C2F200020E
:107BA00013787BB9FD290FD923689A6A4FF0FE013B
:107BB0009047D8B142F6A460C2F200004FF0010134
:107BC000017010BD6FEA01012268936AC9B298473B
:107BD00060B1D4F8080100F10100C4F8080142F6D0
:107BE000A461C2F200014FF000020A7010BD00BF94
:107BF00070B5064640F6B875C2F200054FF4117430
:107C000004FB00F42B194FF00101C3F80C112A59A1
:107C1000936998472859016A3046884770BD00BF6C
:107C200038B540F6B871C2F200014FF4117202FB90
:107C300000F28C18D4F80831D4F80451AB420DD0BE
:107C40008958E3188A6A1979904738B1D4F808013D
:107C5000FF2814BF01300020C4F8080138BD00BF60
:107C600038B540F6B874C2F200044FF4117202FB4A
:107C700000F2A318D3F80451D3F808118D4206D1AD
:107C80004FF00001C3F80C11A2589369984738BD12
:107C900010B440F6B873C2F200034FF4117202FB45
:107CA000003000F58870D0F80031FF2B14BF5A1C4B
:107CB0000022D0F80441A2421CBFC154C0F80021E8
:107CC00010BC7047F8B542F61474C2F20004246880
:107CD0008568C768466807FB05604518611911D2B9
:107CE000CE180B48864210D8012B04D1635D137067
:107CF0004FF00000F8BD10461A460CF06DFA4FF038
:107D00000000F8BD4FF01F00F8BD4FF01F00F8BD98
:107D100001A0020810B542F6BC63C2F200031A7853
:107D200040F6B870C2F200004FF4117404FB020474
:107D3000F8F736FD4FF0FF31C4F810124FF0000392
:107D4000C4F8183204F58874F8F734FD10BD00BF8C
:107D5000F8B506464FF00203037049F20000C0F682
:107D60000100C28B4FF6FF718A4221D03F4C404B3D
:107D7000A34222D203F110033E4DEF1A4FEA17122D
:107D80004FF6FF7502F1010002F001071C46D98B86
:107D9000A9424FD115E01C46D98BA94211D002F15E
:107DA000010203F110031C46D98BA94257D108E008
:107DB00049F20004C0F6010403E049F20004C0F6F1
:107DC00001044FF6FF7021464FF00D02FFF754FA01
:107DD0004FF6FF73984208BF0020E28982421BD011
:107DE000A4F1100549F20000C0F6010085421AD343
:107DF0004FF6FF7029464FF00D02FFF73DFA4FF6A0
:107E0000FF71884208BF002034F8024C84420AD136
:107E10002C464FF0010201E04FF00002607BFF288A
:107E200006D1327004E04FF0020333704FF00004CB
:107E30002046F8BD4FF0000202F1010203F11003E9
:107E40008242BED0002FA6D01C46D98BA942B8D002
:107E500002F1010203F1100382429CD1B1E702F169
:107E6000010203F11003824295D1AAE700980108AC
:107E7000009001080F98010870B5C0B005460E4685
:107E800020F0FF04684621464FF04002F8F7F0FB6F
:107E900000AB53FA85F031464FF010020CF09CF91C
:107EA000684621464FF48072FAF74AFC40B070BD34
:107EB00038B5054640F6B874C2F200044FF41173A9
:107EC00003FB0044D4F81C02FDF73CFB42F6BC6007
:107ED000C2F200000178A94206D142F6BC63C2F2A8
:107EE00000034FF0FF021A704FF00000C4F81C02AC
:107EF00038BD00BF10B54FF00000FBF737FE42F66B
:107F0000A063C2F200031C6834B12068016901B1AA
:107F100088476468002CF8D110BD00BF10B5044636
:107F2000072822D8032894BF4FF4FA73322303FBA7
:107F300001F142F65C63C2F2000303EBC000416052
:107F400059B1FDF7CDFE002808BF012042F65C6361
:107F5000C2F2000343F8340010BD42F65C61C2F285
:107F600000014FF0000241F8342010BD38B504463E
:107F700007284BD842F65C63C2F2000303EBC00053
:107F800045680DB342F65C61C2F2000151F834203D
:107F9000D2B1FDF7A5FE002808BF012042F65C63C0
:107FA000C2F2000353F83410401A85420BD242F655
:107FB0005C63C2F2000303EBC4024FF0000555609E
:107FC00043F8345000E02D1A05F104054CF6CD417C
:107FD000CCF6CC41A1FB05204FEA9003032C0AD834
:107FE00003F1630348F21F51C5F2EB11A1FB033209
:107FF0004FEA521038BD03F109014CF6CD42CCF6E0
:10800000CC42A2FB01304FEAD00038BD4FF0000057
:1080100038BD00BF70B506466446DCF814305D6AB2
:10802000FDF75EFE6169CA6A0AB9C86208E0801A93
:1080300005EB850506FB05F6B04224BF0020C862AB
:108040006369D96AD1F1010038BF002070BD00BF5B
:1080500010B540F6B873C2F200034FF4117404FB7C
:10806000003303F58873D3F80841002C5FD15AB16F
:108070004FF0FF31C3F8001141F6C903C2F200030B
:108080004FF00000187010BDD3F80021B2F1FF3F8F
:1080900006D1FF294BD14FF00002C3F8002110BDDB
:1080A000FF291ED141F6C901C2F200014FF00004C0
:1080B0000C70012A10D94FF00102C3F8082140F6D4
:1080C000B873C2F200034FF4117101FB0030D0F815
:1080D0001C02FCF7F5FF10BD4FF00000C3F80001D3
:1080E00010BDFE2907D141F6C903C2F200034FF0CB
:1080F0000101197010BD41F6C900C2F200000078FC
:1081000048B16FEA0101C9B241F6C900C2F20000EC
:108110004FF000040470FF2A05D8995402F10102BF
:10812000C3F8002110BD4FF0FF32C3F8002110BD8D
:1081300008B540F6B873C2F200034FF4117202FBA7
:108140000030D0F80811D0F8043100F10400994251
:108150000AD94FF00002C0F8002142F6D460C2F202
:1081600000004068FCF7ACFF08BD00BFF8B56546ED
:1081700040F6B473C2F200031C7804F00802D7B2D0
:1081800027B1DCF8146096F8516007E014F0110F85
:1081900006BFDCF8144094F85260002601EB80041E
:1081A00011F820304FEA9312012A08D0022A10D188
:1081B00011F82070C7F3C20303FB06F70BE06A69EE
:1081C00092F8513011F82070C7F3C20202FB03F796
:1081D00001E04FF0000711F8200000F0070104292A
:1081E00050D8DFE811F0940140003B002200050068
:1081F00042F61C71C2F200010B684AF20007C0F699
:108200000107FA1892F802E0D0784FEA006040EADD
:108210000E40527840EA0220FF5C03F104030B6039
:108220003843FFF7B9F868602CE042F61C72C2F2DE
:10823000000213684AF20000C0F60100C11891F86C
:1082400001C0C05C4FEA004040EA0C208978084336
:1082500003F1030313603F186F6013E0FFF750FA58
:10826000C2196A600EE042F61C73C2F2000318687D
:108270004AF20001C0F601010A5CBF186F6000F10C
:108280000100186063784FEA9310012807D0022894
:108290000ED16178C1F3C20202FB06F70AE06F69F2
:1082A00097F851306078C0F3C20101FB03F701E099
:1082B0004FF00007627802F00703042B50D8DFE884
:1082C00013F0260140003B002200050042F61C711D
:1082D000C2F200010B684AF20007C0F60107FA1863
:1082E00092F802E0D0784FEA006040EA0E405278FF
:1082F00040EA0220FF5C03F104030B603843FFF700
:108300004BF8A8602CE042F61C72C2F2000213681F
:108310004AF20000C0F60100C11891F801C0C05C2B
:108320004FEA004040EA0C208978084303F1030338
:1083300013603F18AF6013E0FFF7E2F9C219AA60BB
:108340000EE042F61C73C2F2000318684AF2000104
:10835000C0F601010A5CBF18AF6000F101001860AF
:10836000A3784FEA9310012807D002280ED1A178F4
:10837000C1F3C20202FB06F70AE06F6997F85130B9
:10838000A078C0F3C20101FB03F701E04FF0000742
:10839000A27802F00703042B4ED8DFE803F0B83EC2
:1083A0003920030042F61C71C2F200010B684AF248
:1083B0000007C0F60107FA1892F802E0D0784FEAF9
:1083C000006040EA0E40527840EA0220FA5C03F175
:1083D00004030B601043FEF7DFFFE8602CE042F679
:1083E0001C72C2F2000213684AF20000C0F60100DB
:1083F000C11891F801C0C05C4FEA004040EA0C206F
:108400008978084303F1030313603F18EF6013E01A
:10841000FFF776F9C219EA600EE042F61C73C2F269
:10842000000318684AF20001C0F601010A5CBF1897
:10843000EF6000F101001860E3784FEA9310012823
:1084400002D002280FD108E06E6996F85130E0782A
:10845000C0F3C20101FB03F607E0E178C1F3C202F9
:1084600002FB06F601E04FF00006E27802F0070397
:10847000042B4CD8DFE803F04B031318300042F60E
:108480001C73C2F2000318684AF20001C0F6010131
:108490000A5CB6182E6100F101001860F8BDFFF704
:1084A0002FF982192A61F8BD42F61C72C2F200024D
:1084B00013684AF20000C0F60100C1184C78C05C95
:1084C0004FEA004040EA04208978084303F103039F
:1084D000136036182E61F8BD42F61C71C2F200011D
:1084E0000B684AF20004C0F60104E2189678D078CE
:1084F0004FEA006040EA0640527840EA0220E25C1F
:1085000003F104030B601043FEF746FF2861F8BD3A
:1085100008B503281ED8DFE800F00209101748F25A
:108520006020C0F601000DF047FC08BD48F2642051
:10853000C0F601000DF040FC08BD48F27820C0F6FE
:1085400001000DF039FC08BD48F29020C0F6010092
:108550000DF032FC08BD00BF2DE9F8430546884602
:1085600016461F4642F6BC63C2F2000393F8009021
:1085700043F29040C2F20000016842F69C62C2F2EF
:1085800000021368994201D0FFF7C4FB072D6ED893
:108590001F2E6CD840F6B874C2F200044FF411706C
:1085A00000FB094442F6D460C2F200004FF0000123
:1085B000FCF726FB217965F34711072D14BF002531
:1085C0000125AA1962F304012171CBB22DB184F8FF
:1085D000058043444FF0020001E04FF0010006F136
:1085E000FF3E5FFA8EFE46B302463F1A0EF0010CC4
:1085F0003D5C04F1040635545B1902F101020EF1F1
:10860000FF31C9B2FF2934D114E0BD5C04F1040686
:10861000B5545B1902F1010201F1FF3101F0FF01D4
:10862000BD5CB5545B1902F1010201F1FF31C9B221
:10863000FF29EAD100F1010070442218137100F102
:108640000100C4F804014FF0FF33C4F80831216879
:108650000B6A42F6BC60C2F2000000789847FCF753
:10866000FDFC42F6D460C2F20000FCF7D7FBBDE887
:10867000F8834FFA8CF5002DC7D0BD5C04F10406D9
:10868000B5545B1902F1010201F1FF31C9B2FF29B2
:10869000BBD1CFE738B5054642F62064C2F20004EC
:1086A0002046FCF7BBFBF8F753FF2846FCF79EFE7D
:1086B00020464FF00001FCF7A3FA38BD10B586B094
:1086C0000DF10700FFF744FB044618B19DF8073091
:1086D00023B90FE049F20004C0F60104E2894FF625
:1086E000FF7082422BD049F60001C0F601018C4296
:1086F00009D32AE0304821464FF00D020BF016F95D
:10870000002848D0EAE74FF6FF7249F60000C0F6AD
:1087100001006FEA0403C118C1F3001104F1100451
:10872000E389934239D10AE004F110031C46D98948
:10873000914204D003F11004E389934239D149F600
:108740000002C0F60102944207D349F20004C0F6C9
:10875000010420462146F9F789FF02A816494FF087
:108760000D020BF039FD4FF0FF008DF815004FF6AC
:10877000FF7002A94FF00D02FEF77EFD4FF6FF716C
:10878000884212BFADF816000021ADF81610204641
:1087900002A9FFF771FB06B010BD8442D5D20029B3
:1087A000C2D004F11004E1899142C8D08442BBD305
:1087B000CBE78442B8D3C8E77A0E00202DE9F04F0A
:1087C00085B0884691461D46E2464FF00004264695
:1087D0004FF0020B2DE007462846C047034670B312
:1087E00024B9202822D0092802D11FE0012C05D16C
:1087F0002B2B0DD02D2B0DD05C4601E0022C01D18E
:108800002E2B09D0A3F13002D0B2092817D805E0E9
:108810005C4603E05C4601E04FF003040E2E05D8F1
:1088200004A98A1902F8103C06F101062846C84737
:108830003846FF28CFD000F1FF370028CCD1012CDB
:1088400012D98EB104ACA6194FF0000406F8104CF2
:10885000684621460BF0C4F8DAF81410C864DAF858
:10886000142082F8504005E0DAF814304FF001008F
:1088700083F8500005B0BDE8F08F00BF10B586B09A
:108880004AF20000C0F601003449F9F7EFFE002873
:108890004BD1334B334A9A421DD24AF20001C0F603
:1088A00001010B68B3F1FF3F42D102F104032E4AEC
:1088B000D01A20F00302991812F0040F3FD1184685
:1088C0008B420CD003F104021B68B3F1FF3F3ED092
:1088D0004FF0000031E04AF20000C0F601004AF219
:1088E0000003C0F60203984225D10DF10700FFF7FF
:1088F0002FFA0446B0B19DF80710022912D002A841
:1089000021464FF010020BF067FC9DF815006FF345
:1089100007008DF81500204602A9FFF7ADFA4FF0C9
:1089200001000AE04FF0010007E04FF0000004E012
:108930004FF0000001E04FF0000006B010BD1846F7
:1089400003F104030268B2F1FF3FB8D0C0E702F1BF
:1089500004031068B0F1FF3FB1D0B9E7FF9F0208F0
:1089600000A0020800A0010803A002082DE9F003FE
:108970000346002842D040F20022C0F6000292F8DE
:10898000468092F847C042F6B860C2F200004578CF
:1089900092F84870047842F6C466C2F20006306865
:1089A00096F8049076794FF000021A7083F80180EF
:1089B00083F802C0DA704FF0FB0C83F804C04FF06C
:1089C000060C83F805C09C71DD714FF004051D7223
:1089D0005D729F72DC721A734FEA10245C73987395
:1089E00083F80F901E745A744FF01D0098744FF066
:1089F0000202DA744FF0FE001875587529B142F67C
:108A0000B863C2F200031A680A60BDE8F003704759
:108A1000034628B142F6C462C2F200021068186030
:108A200042F6C461C2F200010879704770B505468C
:108A30000E4614464FF000002946FFF769F808B1CA
:108A4000F7F706FE42F6B463C2F200031A686260EA
:108A5000A56026601C6070BD08B539B142F6A06300
:108A6000C2F200031A68426018601EE042F6A0637A
:108A7000C2F200031B6883420FD1586842F6A0611E
:108A8000C2F20001086010E042685A6041605A6812
:108A90008242F9D013461BB907E033B14FF0000111
:108AA0005A688242F0D01346F5E7FEF74FFF08BD43
:108AB00008B539B142F6C063C2F200031A684260D9
:108AC00018601EE042F6C063C2F200031B688342D6
:108AD0000FD1586842F6C061C2F20001086010E090
:108AE00042685A6041605A688242F9D013461BB905
:108AF00007E033B14FF000015A688242F0D01346CC
:108B0000F5E7FEF723FF08BD08B539B142F6187343
:108B1000C2F200031A68426018601EE042F6187341
:108B2000C2F200031B6883420FD1586842F61871E5
:108B3000C2F20001086010E042685A6041605A6861
:108B40008242F9D013461BB907E033B14FF0000160
:108B50005A688242F0D01346F5E7FEF7F7FE08BDEB
:108B600008B539B142F62073C2F200031A684260B8
:108B700018601EE042F62073C2F200031B688342B5
:108B80000FD1586842F62071C2F20001086010E06F
:108B900042685A6041605A688242F9D013461BB954
:108BA00007E033B14FF000015A688242F0D013461B
:108BB000F5E7FEF7CBFE08BD42F6B063C2F2000354
:108BC0001A68826041601860704700BF70B582B05B
:108BD00006464FF000038DF807300D4601B10B70CB
:108BE00042F6A060C2F20000046874B121684B68CC
:108BF00043B130460DF107012A46984710B19DF860
:108C0000070011E06468002CF0D1072E03D830462D
:108C1000FAF7F0FF08E02DB14FF005022A704FF08F
:108C2000000001E04FF0000002B070BD70B582B0EE
:108C300006464FF000038DF807300D4601B10B706A
:108C400042F6A060C2F20000046874B121688B682B
:108C500043B130460DF107012A46984710B19DF8FF
:108C6000070019E06468002CF0D1072E0BD83046BD
:108C7000FAF7D6FF8DF8070010B13046FBF716F86B
:108C80009DF8070008E02DB14FF005022A704FF063
:108C9000000001E04FF0000002B070BD70B582B07E
:108CA00006464FF000038DF807300D4601B10B70FA
:108CB00042F6A060C2F20000046874B12168CB687B
:108CC00043B130460DF107012A46984710B19DF88F
:108CD000070011E06468002CF0D1072E03D830465D
:108CE000FAF76EFF08E02DB14FF005022A704FF041
:108CF000000001E04FF0000002B070BD70B582B01E
:108D000006464FF000038DF807300D4601B10B7099
:108D100042F6C060C2F20000046894B121688B681A
:108D20002BB130460DF107012A46984718B96468FF
:108D3000002CF3D105E09DF80700003018BF01209A
:108D400008E02DB14FF006022A704FF0000001E05C
:108D50004FF0000002B070BDF0B583B005460E467E
:108D60004FF000038DF8073042F6C060C2F20000F9
:108D700004681CB34FF000072168CA681AB128467E
:108D800031469047E8B923689B6833B128460DF116
:108D900006010DF10702984700E038469DF80710DC
:108DA00091B9646814B10028E6D000E070B128469B
:108DB000314606F02DF94FF0000009E04FF00600B3
:108DC00006E04FF0000003E0084601E04FF0060027
:108DD00003B0F0BD70B582B005460E464FF00003FB
:108DE0008DF8073012B11946FFF7B6FF42F6C060A2
:108DF000C2F20000046884B121684B6828463146FD
:108E00000DF10702984710B19DF8070007E064686C
:108E1000002CF1D14FF0060001E04FF0060002B047
:108E200070BD00BF08B54FF0000001464FF00102D1
:108E3000FFF7D0FF08BD00BF70B582B005460E46F3
:108E40004FF000038DF8073042F61870C2F20000B0
:108E500004689CB121684B68284669460DF10702F9
:108E6000984728B10EB1009830609DF8070014E0D3
:108E700064681CB19DF80720002AEBD045B956B1B3
:108E80004FF00000F8F7CCFE30604FF0000004E037
:108E90004FF00F0001E04FF0000002B070BD00BFC6
:108EA00070B582B005460E464FF000038DF80730CE
:108EB00042F62070C2F2000004689CB121684B6841
:108EC000284631460DF10702984710B19DF807007A
:108ED0000DE064684CB19DF80720002AEED04FF0F9
:108EE0000E0004E04FF00E0001E04FF00E0002B063
:108EF00070BD00BF70B582B005460E464FF000034E
:108F00008DF8073042F62070C2F200000468BCB150
:108F100021688B685BB1284669460DF107029847C6
:108F200028B10EB1009830609DF807000DE064682C
:108F30004CB19DF80720002AEAD04FF0060004E06B
:108F40004FF0060001E04FF0060002B070BD00BF18
:108F50002DE9F04F2DED048B8BB00746154691425D
:108F600054D289464FF0000B4FF000089FED868BDE
:108F70009FED879B6FEA0106B01800F00106CDF85F
:108F800004B0022F47D14BE0CDF804B0022F05D139
:108F90005FFA89F001A9FFF7ADFF04E05FFA89F0FD
:108FA00001A9FFF749FF04EB44030AAAD118A1F174
:108FB000200601F8209C01F81F8C019809F070FF31
:108FC00053EC182B0AF00AF953EC192B09F0C2FFE5
:108FD00009F02CFFB07004F101040A2C04D005F153
:108FE000FF3048450AD14CB104EB44044FF0070070
:108FF0003946E2B202ABFFF7AFFA444609F1010984
:109000004E46CDF804B0022F7DD182E00BB0BDEC0E
:10901000048BBDE8F08FC8B201A9FFF70DFF03E094
:10902000C8B201A9FFF766FF0AAC04F8209D84F8D6
:109030000180019809F034FF53EC182B0AF0CEF8A8
:1090400053EC192B09F086FF09F0F0FEA0704FF0E9
:10905000000404F1010405F1FF334B450DD10AE092
:1090600004EB44024FF007003946D2B202ABFFF7DF
:1090700073FA444601E0002CF2D109F101094D4593
:10908000C4D9002E80D0CDF804B0022F05D05FFAED
:1090900089F001A9FFF7D0FE04E05FFA89F001A989
:1090A000FFF728FF04EB44010AAE761806F8209D6E
:1090B00086F80180019809F0F3FE53EC182B0AF0B2
:1090C0008DF853EC192B09F045FF09F0AFFEB07095
:1090D00004F101040A2C0AD104EB44044FF0070008
:1090E0003946E2B202ABFFF737FA444605E005F134
:1090F000FF30484501D1002CEED109F101094D4561
:109100003FF642AF82E75FFA89F001A9FFF794FECC
:1091100004E05FFA89F001A9FFF7ECFE04EB4403D9
:109120000AAAD118A1F1200A01F8206C01F81F8CBD
:10913000019809F0B5FE53EC182B0AF04FF853ECE8
:10914000192B09F007FF09F071FE8AF8020004F1FB
:1091500001040A2C0AD104EB44044FF007003946FD
:10916000E2B202ABFFF7F8F9444605E005F1FF3043
:10917000B04201D1002CEED109F101094D453FF675
:1091800003AF43E7AFF300800000000000E06F4052
:10919000000000000000E03F2DE9F04F95B040F6E0
:1091A000C410FCF723F94FF002004FF0000142F623
:1091B000B863C2F20003DA78FFF7CAFE4FF0000B83
:1091C000DA46D9464FF001074CF6CD44CCF6CC44F4
:1091D00001944FF07D00FCF709F98DF82F90C846F7
:1091E0004E464C4613E045F0800504F10804E4B215
:1091F0000CABF05CA84202D00CA97554B84606F13D
:1092000001069DF82F50002D50D1202E4ED0204623
:109210000DF12F01FFF7DAFC051C18BF012504F141
:109220000100C0B20DF12F01FFF7D0FC10B145F0E5
:109230000205EDB204F10201C8B20DF12F01FFF7F2
:10924000C5FC08B145F0040504F10302D0B20DF1EC
:109250002F01FFF7BBFC08B145F0080504F104033A
:10926000D8B20DF12F01FFF7B1FC08B145F01005A0
:1092700004F10500C0B20DF12F01FFF7A7FC08B102
:1092800045F0200504F10601C8B20DF12F01FFF7EA
:109290009DFC08B145F0400504F10702D0B20DF184
:1092A0002F01FFF793FC00289DD19EE7B8F1000F36
:1092B00002D1BAF1000F0AD14FF002004946F2B2D2
:1092C0000CABFFF749F94FF03200FCF78FF842F68C
:1092D000B862C2F2000292788AB1019EA6FB0A43EC
:1092E0004FEA131404EB8400BAEB800F07D1384621
:1092F0004946FFF72DFE4FF03200FCF777F8BBF13F
:10930000000F40F09B8003A849464FF020020AF06E
:1093100087FF42F6B861C2F200018D78ADB34E46C8
:109320006FEA0902531903F0010009F0070407FA74
:1093300004F29DF80C1042EA01038DF80C3006F19E
:109340000106AE42C0F299801FE014AA02EBD603D8
:1093500006F0070407FA04F013F8441C40EA01027F
:1093600003F8442C06F1010614AC04EBD60006F019
:10937000070107FA01F210F8443C42EA030400F83E
:10938000444C06F10106AE42DFDB4FF007004FF020
:1093900011014FF01E0203ABFFF7DEF84FF0320071
:1093A000FCF724F803A849464FF020020AF038FFE2
:1093B00042F6B865C2F20005EE78A6B348466FEAF9
:1093C00009018A1902F0010309F0070407FA04F5FC
:1093D0009DF80C1045EA01028DF80C2000F1010007
:1093E000864236DC1FE014AD05EBD00200F0070426
:1093F00007FA04F312F8441C43EA010502F8445C3E
:1094000000F1010014AA02EBD00500F0070407FAEE
:1094100004F315F8441C43EA010205F8442C00F15A
:1094200001008642DFDC4FF007004FF012014FF0E1
:109430001E0203ABFFF790F84FF0060BBAF1000FD6
:1094400004D10BF1FF3B4FF0280AC2E60AF1FF3AC4
:10945000BFE6002BC7D014AB03EBD00500F0070428
:1094600007FA04F215F8441C42EA010305F8443CEB
:1094700000F101008642B6DCD5E700283FF465AF75
:1094800014A800EBD60206F0070407FA04F312F85A
:10949000441C43EA010002F8440C06F10106AE4206
:1094A000FFF653AF71E700BF2DE9F04F2DED028BB2
:1094B00087B008EE100A0C4617469946129E13997B
:1094C000B5EEC08AF1EE10FA54BF00250125A8467A
:1094D00004F1FF33D8B2082807D8092A05D8A246D4
:1094E00001F1FF32944205D808E001F1FF339C42BC
:1094F00040F2CD8001F1FF34E4B2C8E018EE100A6A
:109500000AF0A2F848B930464FF03F0122460AF06F
:1095100087FE4FF000013155C4E018EE100A0AF042
:10952000FFF806EE900AF2EE047AF4EEE76AF1EE46
:1095300010FA0DDB4FF00100B0EE677A00F1010088
:1095400067EE877AF4EEE76AF1EE10FAF6DA03E0F6
:109550004FF00100F2EE047A21464319A34200F3D2
:109560009680C0EB040EC5EB0E0202F1FF3E47F6FB
:10957000EC1AC0F6010ADFED9C4AF6EE003AB2EEB4
:10958000044AC0EB040CC5EB0C0303F0010BBEF165
:10959000000F00F38F808AE0BEF1000F04DDBE45AE
:1095A000B4BF72463A4601E04FF000025AF822304A
:1095B00003EE103AB8EE430A20EE027AB4EEE47AF3
:1095C000F1EE10FA48BF37EE237ABDEEC73A13EE3C
:1095D00010CABCFBF3FB06EE10BAB8EEC65AB4EEE6
:1095E000E75AF1EE10FA0DDB00F1010C87EE006A8C
:1095F00067EE847A0EF1FF3E6046BEF1000200F392
:10960000C380BEE013EE105AB5FBF3F403FB145411
:109610002CB916EE107A002F08BF4FF00008B9F1F0
:10962000000F07D0C8EB0103181A002A18BF013831
:10963000831A01E04FF0000301F10101B8F1000FBE
:1096400004D048F2B427C0F6010703E045F69C6752
:10965000C0F6010722B148F2B820C0F6010003E0CD
:1096600045F69C60C0F6010048F2CC25C0F6010525
:10967000009501978DED026A03900492059430469F
:1096800048F2BC22C0F601020AF094F90AE0304622
:10969000002D0CBF2B212D2122460AF0C1FD4FF0D9
:1096A0000000305507B0BDEC028BBDE8F08F4FF0E5
:1096B000000203E0BE45B4BF72463A465AF8223073
:1096C00000EE103AB8EE405A65EE260AF4EEE40ACF
:1096D000F1EE10FA48BF70EEA30ABDEEE03A13EEC9
:1096E00010CABCFBF3FC06EE10CAF8EEC65AF4EE44
:1096F000E75AF1EE10FA85DB00F1010080EE852AD1
:1097000067EE847A0EF1FF3E42199142BFDBBBF156
:10971000000F3FF441AFBEF1000F02DC4FF000023A
:1097200003E0BE45B4BF72463A465AF8223001EE15
:10973000103AF8EE411A21EE822AB4EEE42AF1EE54
:1097400010FA48BF32EE232ABDEEC23A13EE10BA29
:10975000BBFBF3FB06EE10BAF8EEC62AF4EEE72ADE
:10976000F1EE10FAFFF64EAF00F1010082EE212A71
:1097700067EE847A0EF1FF3E43199942BFF60CAFB3
:1097800085E74FF0000202E0BA42A8BF3A465AF815
:10979000223006EE903AF8EE660A20EE861AB4EE13
:1097A000E41AF1EE10FA48BF31EE231ABDEEC13AC9
:1097B00013EE10BABBFBF3FB06EE10BAF8EEC65A76
:1097C000F4EEE75AF1EE10FAFFF61CAF0CF10100CF
:1097D00081EE202A67EE847A0EF1FF3E4219914213
:1097E000BFF6DAAE53E700BF0000004BF8B5054600
:1097F0000F46F6F7D5FF064640F6B872C2F20002F1
:109800004FF4117303FB05F01418115811B18A6855
:109810002846904784F820724FF00005C4F8105293
:10982000C4F81452C4F80451C4F808513046F6F78D
:10983000C1FF04F5097029464FF00802F6F76AFFE8
:10984000F8BD00BF70B588B0054640F6B874C2F2E6
:1098500000044FF4117303FB004494F82002002825
:1098600047D042F6BC61C2F200010878FF2803D05D
:109870004FF00401FFF7BAFF28464FF00001FFF751
:10988000B5FF42F6BC66C2F20006357048F2D82039
:10989000C0F601004FF007014EF23172C0F600022F
:1098A000FBF766FDC4F81C02246830784FF0010213
:1098B00000924FF00002019247F65133C0F60003C8
:1098C000029348F23111C0F60001039148F25103AE
:1098D000C0F60003049347F6B161C0F6000105919C
:1098E000069264684FF416514FF00803A047FEF744
:1098F00011FA08B070BD00BF38B505F07DFB42F627
:10990000BD63C2F200034FF001021A704FF0000471
:109910002546E0B229462A46FFF75CFA40B904F131
:109920000104E0B229462A46FFF754FA00285BD02A
:1099300042F62071C2F200010C6834B12368DA6883
:1099400002B190476468002CF8D142F6B460C2F2CC
:10995000000004683CB121680B680BB1A06898470F
:109960006468002CF7D1FAF781FCFEF7C3FA40F6E1
:10997000B872C2F2000292F82002042806D028B180
:109980004FF000004FF00401FFF730FF40F6B871D0
:10999000C2F2000191F86434042B06D02BB14FF0D1
:1099A00001004FF00401FFF721FF40F6B872C2F248
:1099B000000292F8A806042806D028B14FF0020051
:1099C0004FF00401FFF712FF40F6B871C2F2000138
:1099D00091F8EC38042B06D02BB14FF003004FF078
:1099E0000401FFF703FF38BD04F10104B4F5807FE3
:1099F0008FD19DE72DE9F04F2DED0A8BABB01CAF59
:109A000026AC47F25C25C0F6010595E80F0084E816
:109A10000F00A76047F6D903C0F60003E3602046B5
:109A20002AA9F8F7F7FF22AE95E80F0086E80F00A5
:109A3000B76047F6F500C0F60000F06030462146FA
:109A4000F8F7E8FF4FF000041B9442F62060C2F2E2
:109A500000002146FBF7D4F842F6C461C2F20001CF
:109A60000C71FFF749FF08F0C9FC4FF00200FFF747
:109A7000E9FE42F61C72C2F2000215680DBB0CF042
:109A80008BF9F0B9F7F764FC10F0C20F19D14FF061
:109A90000300FEF73DFD4FF47A744FF0320528467F
:109AA000FBF7A4FCF7F754FD04F1FF342846FBF75D
:109AB0009DFCF7F74DFD013CF1D14FF00000FEF7A2
:109AC00027FD40F6B473C2F200034FF000041C609F
:109AD0004FF00100187041F6CC05C2F2000528468F
:109AE000214641F254520AF09BFB40F67460C2F2E8
:109AF000000021464FF480720AF092FB42F65C604F
:109B0000C2F2000021464FF040020AF089FB42F603
:109B1000FC60C2F2000021464FF016020AF080FB02
:109B200021954FF00A01696220462946FDF770FE33
:109B300042F65862C2F20002146042F6AC63C2F20E
:109B400000031C6042F61C75C2F200054FF03004A1
:109B50002C604AF20004C0F6010494F82F0000F1D2
:109B6000010094F82E1000EB0122101942F6147334
:109B7000C2F200031860FCF7B3F80A902868215C71
:109B8000FF2924D142F6C462C2F200024FF0010361
:109B9000137110604FF0FF00507142F6A861C2F2DD
:109BA00000014FF000020A6042F6BC63C2F20003FB
:109BB000187840F6B871C2F200014FF4117202FB3E
:109BC0000013D3F81C02FBF77BFA04F0E8BC05F0A5
:109BD000F1F94FF000060996B3463446DFEDBE8A30
:109BE0009FEDBE9ADFEDBEAA9FEDBE8ADFEDBE9A65
:109BF0009FEDBEAAFFE72CB94FF00000FEF74AFD2B
:109C00004FF0640404F1FF3440F6B477C2F2000769
:109C10003D7805F0F7026FF304123A7042F61C73B8
:109C2000C2F200031868089042F61C76C2F20006E1
:109C30004AF20007C0F6010740F6B478C2F2000805
:109C400047F61429C0F6010931687D5C01F1010174
:109C5000316098F8002012F0010F0DD10BF1010BCB
:109C6000BBF5807F08D142F6C460C2F200004FF01D
:109C70003602027104F059BC0DF1700C28464946B9
:109C8000FEF774FA47F2B853C0F6010353F82510F3
:109C900048F2202AC0F6010A41F00100004731686D
:109CA0007A5C0B9201F1010131600F2A04F23584D4
:109CB0000DF1700C10465146FEF758FA47F6F07356
:109CC000C0F601030B9853F82010E5E731687A5C81
:109CD0000B9201F101013160102A02D9154604F0FE
:109CE0001DBC0DF1700C0B9847F27451C0F60101C8
:109CF000FEF73CFA47F23043C0F601030B9853F8E5
:109D00002010C9E731687A5C0B9201F101013160E2
:109D10002F2A02D9154604F001BC0DF1700C0B98E6
:109D200047F27031C0F60101FEF720FA47F61463DE
:109D3000C0F601030B9853F82010ADE731687A5C48
:109D40000B9201F1010131603B2A02D9154604F062
:109D5000E5BB0DF1700C0B9848F23001C0F6010123
:109D6000FEF704FA47F28023C0F601030B9853F87C
:109D7000201091E731687A5C0B9201F101013160AA
:109D80003F2A02D9154604F0C9BB0DF1700C0B989F
:109D900048F22011C0F60101FEF7E8F947F27443DA
:109DA000C0F601030B9853F8201075E731687A5C10
:109DB0000B9201F101013160432A02D9154604F0EA
:109DC000ADBB0DF1700C0B9848F25831C0F6010193
:109DD000FEF7CCF947F6D463C0F601030B9853F8AD
:109DE000201059E7219E96F846700DF1700CFDF792
:109DF00071FC219D3B1895F8502002F001001918C4
:109E00001C9185F84710FF2994BF0021012185F896
:109E10005010F0E6219E96F846700DF1700CFDF79B
:109E200059FC3D181C95219B83F84750FF2D94BF8A
:109E30000025012583F85050DDE60DF1700CFDF78B
:109E400049FC30B1219A92F84710081C18BF012034
:109E500001E04FF00000219E86F84700CBE60DF1AF
:109E6000700CFDF737FC219F97F84750284087F882
:109E70004700C0E61D9BA3F1FB031C9314E11D9852
:109E8000A0F1FB001C909CE11D9AA2F1FB021C9228
:109E9000CDE11D99A1F1FB011C9169E21D9BA3F18C
:109EA000FB031C934FF002001B9001E21D9AA2F1EC
:109EB000FB021C921E991B912BE21D9BA3F1FB033D
:109EC0001C9325E11D98A0F1FB001C90A7E21D9AB0
:109ED000A2F1FB021C92E3E200000034FFFF7F4B83
:109EE000FFFF7FCB00000000FEFFFFCAFEFFFF4A1E
:109EF0001D9EA6F1FB061C961E9F1B9714E31D9941
:109F0000A1F1FB011C911E9B1B934FF000008DF8EB
:109F10006A00C2E31D9AA2F1FB021C921E991B91DA
:109F20004FF001038DF86A30B7E31D98A0F1FB00F4
:109F30001C9000F04EBC1D9DA5F1FB051C9500F08A
:109F4000A3BC9DF874004FF00101FEF705FF8DF8EA
:109F50006B0000283FF44FAE42F6C464C2F2000426
:109F6000207104F0E2BA1D9E1C964FF001038DF89B
:109F70006A301E46219A92F847100B4205D09DF890
:109F800070003146FEF7E8FE68B99DF86A304FEA86
:109F900043008DF86A001C9A02F101021C9210F035
:109FA000FE03E7D10CE09DF86A10012908D19DF865
:109FB0006B4042F6C460C2F20000047104F0B5BA0E
:109FC0000DF1700CFDF786FB15E69DF8740004F0AA
:109FD000E3FF10E60DF1700CFDF77CFB1C9042F6E0
:109FE0001C73C2F200031A681C9902EB410018604E
:109FF000FDF786FB1C9001F0CCBC1D9BFA2B08D909
:10A0000042F6C464C2F200044FF01300207104F061
:10A010008CBA40F67462C2F20002D15C1C91DEE799
:10A02000219B93F852201C92D9E7219991F8500076
:10A030001C90D4E74FF0000BDDE5219F97F84650C8
:10A040001B950DF1700CFDF745FB1C901B99FDF75E
:10A05000F7FB219E86F84700CDE5219F97F8470042
:10A0600097F84610FDF7ECFB87F85000C3E50DF1BB
:10A07000700CFDF757FB1E9B40F67462C2F20002A3
:10A08000D05C1D9920EA0105D554B4E542F6FC6088
:10A09000C2F200004FF000014FF015020AF0C0F8C4
:10A0A000A9E54FF000061C960DF1A80C1CF8386DC0
:10A0B000FDF710FB0146304606F0A8FD8DF86B0059
:10A0C00000283FF498AD42F6C464C2F20004207147
:10A0D00004F02BBA05F028FC8DE505F02DFC8DF879
:10A0E0006B0000283FF487AD42F6C463C2F2000360
:10A0F000187104F01ABA42F61477C2F200073A68EF
:10A100001D98101805F004FC75E54FF000011C9136
:10A110001C9B40F6B872C2F200024FF4117000FBB3
:10A12000032191F82022032A3FD140F6B876C2F2EB
:10A13000000600FB03F303F58877F119F31803F128
:10A1400004034FF00000D1F80021FE2A94BF551CF3
:10A150000025D1F80461B54214BF0025012565F33F
:10A160000000B24214BF0022012262F34100D3F882
:10A170000051FE2D94BF013500250DF1A80C4CF8BF
:10A18000385DD3F80471BD4214BF0025012565F385
:10A190008200D3F80811D1F1010338BF002363F323
:10A1A000C300C0B2FDF77EFA25E542F6C464C2F2F0
:10A1B00000044FF04803237104F0B7B94FF00000DA
:10A1C0001C901C9B40F6B872C2F200024FF4117151
:10A1D00001FB032090F82022032A1CD140F6B87618
:10A1E000C2F2000601FB0365D5F81072D5F814120F
:10A1F000781AB0F5807F88BF00F580701C901C9A9B
:10A20000FF2A84BFFF221C920DF1A80C1CF8380D08
:10A21000FDF748FAEFE442F6C464C2F200044FF0DE
:10A220004803237104F081B94FF000031C931C987C
:10A2300040F6B872C2F200024FF4117101FB002324
:10A2400093F82022032A24D140F6B876C2F2000601
:10A2500001FB006505F58877D7F80011D7F80431C0
:10A26000CA1AB2F5807F88BF02F580721C920DF188
:10A27000700CFDF72FFA8DF86A001C9EB04238BFB3
:10A280001C90D7F804011C9D2918CBB2C7F80431E3
:10A29000B1E442F6C464C2F200044FF048002071F9
:10A2A00004F043B94FF000021C924FF002001B90E3
:10A2B0001C9B40F6B872C2F200024FF4117101FB10
:10A2C000032090F82022032A15D140F6B877C2F275
:10A2D000000701FB03760DF1700C1B9847F6550142
:10A2E000C0F6000147F66902C0F6000206F5887361
:10A2F000FDF72AFA7FE442F6C464C2F200044FF08C
:10A300004803237104F011B94FF000011C911D980E
:10A310001B901C9B40F6B872C2F200024FF4117100
:10A3200001FB032090F82022032A15D140F6B875CE
:10A33000C2F2000501FB03570DF1700C1B9847F6A4
:10A340005501C0F6000147F66902C0F6000207F5A4
:10A350008873FEF733FA4EE442F6C464C2F2000496
:10A360004FF04803237104F0E0B84FF000011C9156
:10A370001C9840F6B872C2F200024FF4117303FB4E
:10A38000002191F82022032A3DD140F6B876C2F28E
:10A39000000603FB006505F588750DF1700CFDF7EF
:10A3A00099F98DF86A00D5F804111C914FF0000757
:10A3B0001B97D5F800710B468F4207D06A5C82422A
:10A3C00019D04FF001024FF0000E0CE04FF0FF00EB
:10A3D0001B9010E002F10101EE5C864202D11C9359
:10A3E0001B9208E00A46FF2B14BF01337346BB42A1
:10A3F000F0D11C93EAE70DF1700C9DF86C00FDF7AD
:10A4000051F9FFF7F8BB42F6C464C2F200044FF002
:10A410004800207104F089B84FF000031C931C9889
:10A4200040F6B872C2F200024FF4117101FB002332
:10A4300093F82022032A27D140F6B875C2F200050E
:10A4400001FB005707F58875D7F81462D7F810128A
:10A450008E4212D00DF1700CFDF73CF98019C7B295
:10A460001C970DF1700CE85DFDF71CF94FF000052D
:10A47000219E86F85050FFF7BEBB4FF00102219B92
:10A4800083F85020FFF7B7BB42F6C464C2F2000461
:10A490004FF04800207104F048B84FF000011C91C3
:10A4A0001C9B40F6B872C2F200024FF4117000FB20
:10A4B000032191F82022032A28D140F6B877C2F26E
:10A4C000000700FB037505F58876D6F80401D6F879
:10A4D0000011884213D00DF1700C305CFDF7E2F8EA
:10A4E000D6F80471FF2F14BF01370027C6F8047196
:10A4F0004FF00005219E86F85050FFF77CBB4FF0CF
:10A500000102219B83F85020FFF775BB42F6C4641B
:10A51000C2F200044FF04803237104F006B84FF074
:10A5200000001C901D991B9142F61472C2F20002A9
:10A53000D2F800801B9F08EB07064AF20003C0F622
:10A5400002039E4208D942F6C464C2F200044FF0EE
:10A550001F02227103F0E9BF1C98032808D942F6B4
:10A56000C460C2F200004FF03703037103F0DDBF97
:10A57000F1780C2908D942F6C464C2F200044FF005
:10A580003701217103F0D1BF40F6B875C2F2000562
:10A590004FF4117202FB005393F8200238B118F8FF
:10A5A000071021B10FE04846FEF774F805E04CF2C1
:10A5B0004F354FF09609DDF828A0FBF791FBCAEB69
:10A5C0000002AA42EFD918F80770032F3FF613AB29
:10A5D000DFE807F002080F169DF87000FFF732F968
:10A5E000FFF709BB9DF87000314606F029FBFFF725
:10A5F00002BB9DF87000314605F018F9FFF7FBBA71
:10A600009DF87050B77828464FF00301FFF7EEF839
:10A610004FF4117303FB05F040F6B871C2F200016C
:10A62000085800283FF4E7AA47F26C23C0F601035C
:10A6300007EB470703EB0708F67847F6B812C0F6B2
:10A64000010252F82610DA5D98F8013098F802708D
:10A6500000974FF00006019647F62147C0F6000725
:10A66000029747F66147C0F60007039747F6914700
:10A67000C0F60007049747F6B167C0F600070597D4
:10A68000069646682846B047FFF7B5BA4FF0000176
:10A690001C911D981B908DF86A101C9840F6B87399
:10A6A000C2F200034FF4117101FB003292F8203224
:10A6B000032B78D140F6B875C2F2000501FB0057B4
:10A6C00007F5887942F61476C2F2000632682199BD
:10A6D0008B6BD018D35CFF2B5CD080464FF001070A
:10A6E0004FF0000A0894CDF82CB0BB4698F8014012
:10A6F00004EB032642F61472C2F2000213689819A2
:10A70000D9F804111C919DF86A501DB19F5D00F1AC
:10A71000010000E0574600F1FF349DF86A602EB159
:10A7200077B9089C5D46DDF82CB005E062783AB94F
:10A73000089C5D46DDF82CB01C98C9F804012BE09C
:10A740001C9BD9F80001984218D014F8016F19F831
:10A7500003501B9939B9304609F0D0F8C6B22846E3
:10A7600009F0CCF8C5B2AE4208D11C9AFF2A14BF3A
:10A77000013252461C9207F1FF37CEE70BF1010B75
:10A7800018F8023FFF2BB1D1089CDDF82CB04FF038
:10A79000000501E04FF000050DF1700CE8B2FCF788
:10A7A00081FFFFF728BA42F6C464C2F200044FF0FA
:10A7B0004800207103F0B9BE4FF000031C931E9AAD
:10A7C0001B924FF001018DF86A1066E74FF000010F
:10A7D0001C911C9B40F6B872C2F200024FF411703B
:10A7E00000FB032191F82022032A31D140F6B876EC
:10A7F000C2F2000600FB036505F588770DF1700CC9
:10A80000FCF768FF8DF86A004FF000011C91D7F843
:10A810000431D7F80051AB4212D0FA5C82420FD11A
:10A820004FF00006FF2B14BF01333346AB4202D179
:10A83000C7F8043104E0F95C8142F3D0C7F8043171
:10A840000DF1700C4FF00000FCF72CFFFFF7D3B9AF
:10A8500042F6C464C2F200044FF04803237103F0CF
:10A8600064BEFBF73DFA0A9FC01B0DF1700C4CF261
:10A870004F3398428CBF00200120FCF713FFFFF7F5
:10A88000BAB94FF000001C901C9D40F6B872C2F29D
:10A8900000024FF4117606FB052191F82072032F78
:10A8A0007FF4A9A940F6B873C2F2000306FB053095
:10A8B00000F10405D0F80861D5F8002102F1010289
:10A8C000964238BF06F58076B11AFF2934BF0F468D
:10A8D000FF270DF1700CF8B2FCF7E4FEFFF78BB91F
:10A8E0001D9B40F67460C2F20000C55C05F1FF36A6
:10A8F000C654FFF780B91D9BFA2B08D942F6C464F1
:10A90000C2F200044FF01301217103F00EBE40F6B5
:10A910007461C2F20001CA5C02F1FF30C2B2CA54D3
:10A92000002A3FF468A91E9B1C9301F032B81D98C1
:10A93000FA2808D942F6C464C2F200044FF01300AA
:10A94000207103F0F2BD40F67463C2F200031A5C9A
:10A9500002F1FF31CAB21A54002A42F0FB83FFF71A
:10A960004AB91D9BFA2B08D942F6C464C2F200040E
:10A970004FF01303237103F0D8BD40F67461C2F2A7
:10A980000001CA5C02F1FF30C2B2CA54002A02F0D0
:10A99000E183FFF730B9219F97F8515005F1FF3659
:10A9A00087F85160FFF727B9219991F8470000F126
:10A9B000FF3281F84720FFF71EB9219BD86C08F0C1
:10A9C000AFFE219FF864FFF716B9219D95ED137A2C
:10A9D000D5ED127A37EE270A85ED130A219DE86C32
:10A9E00008F012FE30B14FF00206219D85F850604C
:10A9F000FFF701B9219FF86C08F016FE30B14FF057
:10AA00000101219B83F85010FFF7F5B84FF00002C9
:10AA1000219880F85020FFF7EEB89DF87400219936
:10AA200001F14C01FEF708FA8DF86B0000283FF4A5
:10AA3000E2A842F6C464C2F20004207103F075BDBE
:10AA40009DF874002199C96CFEF72AFA8DF86B0005
:10AA500000283FF4D0A842F6C462C2F2000210718E
:10AA600003F063BD219EF06C08F0DEFD20B9219853
:10AA7000806C08F0D9FD30B14FF00306219880F8C2
:10AA80005060FFF7B8B8219BD3ED13BA93ED12BA1B
:10AA90007BEECB0A10EE900A08F042FE0CEE100A94
:10AAA0001BEE900A1BEE101A08F0D4FD01464FF081
:10AAB0007E5008F0CFFD01EE100A61EE281AB4EEC8
:10AAC000E1CAF1EE10FA06D84FF00001219A82F89F
:10AAD0005010FFF790B8219F97ED132AD7ED122A57
:10AAE000B4EEE22AF1EE10FA05DD4FF0010587F829
:10AAF0005050FFF780B8B4EEE22AF1EE10FA4CBFE6
:10AB00000222032287F85020FFF775B8219B93EDAE
:10AB1000133AF7EE003A33EE634A83ED134A219875
:10AB2000C06C08F081FD30B14FF00305219981F828
:10AB30005050FFF760B8219A92ED13BA7BEE49BAF4
:10AB40001BEE900A08F0ECFD0BEE900A1BEE100ACB
:10AB500019EE101A08F07EFD01464FF07E5008F005
:10AB600079FD00EE100A60EE280AF4EEE0BAF1EE8C
:10AB700010FA1ED9219E96ED13BA3BEE091A11EE7A
:10AB8000100A08F0CDFD0BEE900A1BEE100A1AEE2B
:10AB9000901A08F05FFD01464FF07E5008F05AFD14
:10ABA00001EE900A21EEA82AF4EEC2BAF1EE10FAF4
:10ABB00006D84FF00406219B83F85060FFF71BB8BE
:10ABC000219BDD6C284608F0ABFD0BEE100A2846F1
:10ABD00018EE101A08F03EFD01464FF07E5008F0C6
:10ABE00039FD02EE900A22EEA83AB4EEC3BAF1EEB5
:10ABF00010FA06D84FF00000219A82F85000FEF7B4
:10AC0000FABF2199D1ED133AF4EEC83AF1EE10FAF9
:10AC100005DD4FF0010781F85070FEF7ECBFF4EE50
:10AC2000C83AF1EE10FA4CBF0222032281F85020FC
:10AC3000FEF7E1BF219FD7ED124A97ED135AC4EEFC
:10AC4000855AC7ED135AC9E62199C86C08F0D8FC9B
:10AC5000002840F09C86FEF7CEBF219AD66C304685
:10AC600008F05EFD0BEE100A304618EE101A08F0E0
:10AC7000F1FC01464FF07E5008F0ECFC06EE100AA5
:10AC800066EE286AB4EEE6BAF1EE10FA00F37F86BB
:10AC9000FEF7B1BF2198C06C08F0B2FC002800F0AC
:10ACA0007686FEF7A8BF219B93ED137AD3ED127A37
:10ACB000B4EEE77AF1EE10FA80F26986FEF79BBFF8
:10ACC000219991ED130AD1ED120AB4EEE00AF1EEEA
:10ACD00010FA00F35C86FEF78EBF219A92ED131AEC
:10ACE000D2ED121AB4EEE11AF1EE10FA40F24F86EC
:10ACF000FEF781BF219890ED132AD0ED122AB4EE11
:10AD0000E22AF1EE10FA00F14286FEF774BF219EAE
:10AD1000F66C304608F004FD0BEE100A304618EED3
:10AD2000101A08F097FC01464FF07E5008F092FC94
:10AD300003EE100A63EE283AB4EEE3BAF1EE10FA2D
:10AD400040F22586FEF757BF219DE86CFCF7FAFA22
:10AD5000E8640DF1700C4FF00000FCF78FFDFEF77A
:10AD60004ABF1D9B102B08D942F6C464C2F20004EE
:10AD70004FF01203237103F0D8BB219FF86C08F049
:10AD80003FFC38B9219AD2ED134AB6EE005A34EEA0
:10AD900085BA06E0219991ED13BAB6EE004A3BEE72
:10ADA00044BA1BEE100A08F02BFC88B9B4EECABAFC
:10ADB000F1EE10FA04DC1BEE100A08F025FC38B1A5
:10ADC0004FF00100219E86F850006FF000402CE00B
:10ADD0001BEE100A08F014FC88B1B4EEE9BAF1EEEB
:10ADE00010FA04D41BEE100A08F00EFC38B14FF034
:10ADF0000101219A82F850104FF0004015E01BEE3F
:10AE0000100A08F011FC38B14FF00207219B83F8BB
:10AE100050704FF0000008E0BDEECBBA1BEE100AF8
:10AE20004FF00006219D85F850604FEA006545EA25
:10AE3000106700F47F4347EA032100F47F0241EAF0
:10AE4000122042F6FC66C2F200061D9D7051FEF70C
:10AE5000D2BE1D99102908D942F6C464C2F200047A
:10AE60004FF01203237103F060BB42F6FC67C2F29D
:10AE700000077A584FEA026040EA126602F47F4502
:10AE800046EA052302F47F0143EA112705EE907A92
:10AE9000B8EE656A219880ED136AB4EECA6AF1EEE5
:10AEA00010FA04DCB4EEE96AF1EE10FA05D54FF0C1
:10AEB000010680F85060FEF79EBE4FF0000280F859
:10AEC0005020FEF798BE0DF1700C4FF00100FCF71A
:10AED000D5FC219DE86CFCF75FFA2199C864FEF768
:10AEE0008ABE219FD7ED136AB7EE007A76EE877A95
:10AEF000C7ED137A13E6219FF86C08F095FB50B16B
:10AF0000219D4FF0000185F847104FF0040785F8A8
:10AF10005070FEF770BE219890ED134AB4EEC84A07
:10AF2000F1EE10FA23DB9FEDD56AB4EEC64AF1EEDE
:10AF300010FA0FD5FCEEC46A16EE902A0DF1700CD3
:10AF4000D0B2FCF7AFFB4FF00006219B83F85060B6
:10AF5000FEF751BE0DF1700C4FF0FF00FCF7A2FBA5
:10AF60004FF00207219880F85070FEF744BEB4EE0F
:10AF7000C84AF1EE10FA7EF53EAEDFEDC14AB4EEFE
:10AF8000E44AF1EE10FA11DDB1EE445AFCEEC55A76
:10AF900015EE903A0DF1700CD8B2FCF783FB4FF030
:10AFA0000105219981F85050FEF725BE0DF1700C76
:10AFB0004FF0FF00FCF776FB4FF00302219E86F86E
:10AFC0005020FEF718BE1D98F92808D942F6C4642F
:10AFD000C2F200044FF01300207103F0A6BA219AC8
:10AFE00092ED137AFDEEC77A17EE906A33B21C9396
:10AFF0009DB2C6F3072141EA052740F67462C2F20A
:10B0000000021752FEF7F7BD1D9AF92A08D942F639
:10B01000C464C2F200044FF01302227103F085BA37
:10B02000219E96ED130AFCEEC00A10EE903A9DB2F6
:10B030001C954FEA152141EA052740F67460C2F2DB
:10B0400000008752FEF7D7BD1D9E219B9E64FEF730
:10B05000D2BD1D9D2199CD64FEF7CDBD0DF1700CC3
:10B06000FCF738FB01EE100AF8EE411A219FC7EDFC
:10B07000131AFEF7C0BD1D98F92808D942F6C4641A
:10B08000C2F200044FF01300207103F04EBA40F6F4
:10B090007462C2F20002165A4FEA162343EA0625EA
:10B0A000A9B202EE101AF8EE422A219FC7ED132A28
:10B0B000FEF7A1BD1D9BF92B08D942F6C464C2F26C
:10B0C00000044FF01303237103F02FBA40F67462AB
:10B0D000C2F20002D65A4FEA162545EA06218FB27F
:10B0E00003EE107AF8EE433A2198C0ED133AFEF7DA
:10B0F00082BD1D98072808D942F6C461C2F200013A
:10B100004FF00800087103F010BAFCF72FFF04EEAF
:10B11000100AF8EE444A219AC2ED134AFEF76BBDBD
:10B12000219E96ED135AD6ED125A25EE256A86ED2C
:10B13000136A53E4219DD5ED136AB1EE667A85ED6D
:10B14000137AFEF758BD4FF000004FF001010A4698
:10B15000FDF740FE219F97ED130AF1EE047A60EEB1
:10B16000270A4FF000030093019342F62470C2F2C5
:10B170000000BCEEE01A11EE101A4FF0FF0248F684
:10B180002563C0F60003FAF775FDFEF734BD1D997F
:10B19000F72908D942F6C464C2F200044FF0130044
:10B1A000207103F0C2B940F67462C2F20002505836
:10B1B000FCF7F2F8219EB064FEF71DBD1D9BF72B36
:10B1C00008D942F6C461C2F200014FF013020A71BD
:10B1D00003F0ABB940F67465C2F20005E858FCF71D
:10B1E000DBF8219FF864FEF706BD1D98072808D9F3
:10B1F00042F6C464C2F200044FF00801217103F06A
:10B2000094B9219ED6ED131AF4EEC81AF1EE10FA95
:10B210000DDBF4EEC91AF1EE10FA08D8BCEEE12A03
:10B220008DED1C2A4FF0000586F850501FE0F4EE1B
:10B23000C91AF1EE10FA07DD6FF07F401C904FF055
:10B24000010386F8503012E04FF000031C9311EE1A
:10B25000900A08F0D5F928B14FF00201219A82F83E
:10B26000501004E04FF00305219F87F850501D98BF
:10B270001C99FCF753FEFEF7BEBC00BF00008043E4
:10B28000000080C3219EF06C08F0CEF900287EF407
:10B29000B2AC219FD7ED132AF4EEC82AF1EE10FAD2
:10B2A00004DD4FF07E50F864FEF7A5BCF4EEC82A2A
:10B2B000F1EE10FA7EF59FAC4FF00002CBF68072F3
:10B2C000FA64FEF798BC219B9D6ACDB1FAF708FDA0
:10B2D000219EB76AC7F1040210184CF6CD43CCF694
:10B2E000CC43A3FB00154FEA9501776AB1FBF7F257
:10B2F00003EE102AF8EE433AC6ED133AFEF77BBC94
:10B300004FF6FF71C7F67F71D964FEF774BC1D9EBE
:10B31000F72E08D942F6C464C2F200044FF01301BC
:10B32000217103F002B92198C06CFCF70BF840F6CC
:10B330007463C2F200039851FEF75DBC219E96ED46
:10B34000124AD6ED134A34EE645A86ED135AFFF7CB
:10B3500045BB219FFA6C1C92B86CF864BA64FEF786
:10B360004ABC2199C86C08F05FF930B14FF0030571
:10B37000219F87F85050FEF73EBC219BD86C08F007
:10B3800043F930B14FF00406219B83F85060FEF77B
:10B3900032BC219EF56C284608F0C2F90BEE100A6B
:10B3A000284618EE101A08F055F901464FF07E5065
:10B3B00008F050F905EE900A25EEA86AB4EEC6BA78
:10B3C000F1EE10FA06D84FF00000219981F85000F4
:10B3D000FEF711BC219FD7ED136AF4EEC86AF1EEB7
:10B3E00010FA05DD4FF0010287F85020FEF703BC8C
:10B3F000F4EEC86AF1EE10FA4CBF0222032287F87D
:10B400005020FEF7F8BB219AD2ED13BA92ED12BA92
:10B410003BEECBCA1CEE100A08F082F90CEE100AC3
:10B420001BEE900A1BEE101A08F014F901464FF0BB
:10B430007E5008F00FF907EE100A27EE280AB4EE46
:10B44000C0CAF1EE10FA0DF1700C8CBF0020012083
:10B45000FCF728F9FEF7CFBB2198C66C304608F000
:10B460005FF90BEE100A304618EE101A08F0F2F8E9
:10B4700001464FF07E5008F0EDF807EE900A67EEB7
:10B48000A80AB4EEE0BAF1EE10FA0DF1700C8CBF20
:10B4900000200120FCF706F9FEF7ADBB219991EDE4
:10B4A000131AD1ED121AB4EEE11AF1EE10FA0DF101
:10B4B000700CB4BF00200120FCF7F4F8FEF79BBB32
:10B4C000219B93ED132AB5EEC02AF1EE10FA0DF18F
:10B4D000700CB4BF00200120FCF7E4F8FEF78BBB32
:10B4E000219DD5ED132A95ED123AF4EEC32AF1EE23
:10B4F00010FA0DF1700CD4BF00200120FCF7D2F837
:10B50000FEF779BB219FD7ED133A97ED124AF4EE7F
:10B51000C43AF1EE10FA0DF1700C8CBF002001203E
:10B52000FCF7C0F8FEF767BB219AD2ED134A92ED03
:10B53000125AF4EEC54AF1EE10FA0DF1700C54BF38
:10B5400000200120FCF7AEF8FEF755BB2198D0EDA6
:10B55000135AF5EEC05AF1EE10FA0DF1700C54BF0B
:10B5600000200120FCF79EF8FEF745BB219ED6ED9A
:10B5700013BA96ED12BA3BEECB6A16EE100A08F03B
:10B58000CFF80CEE100A1BEE900A1BEE101A08F012
:10B5900061F801464FF07E5008F05CF806EE900A24
:10B5A00026EEA87AB4EEC7CAF1EE10FA0DF1700CCF
:10B5B000D4BF00200120FCF775F8FEF71CBB2199D1
:10B5C000CD6C284608F0ACF80BEE100A284618EEB1
:10B5D000101A08F03FF801464FF07E5008F03AF894
:10B5E00000EE100A60EE287AB4EEE7BAF1EE10FA37
:10B5F0000DF1700CD4BF00200120FCF753F8FEF7CA
:10B60000FABA1D9BF82B08D942F6C464C2F20004B2
:10B610004FF01303237102F088BFFAF761FB219FFB
:10B6200000F104004CF6CD42CCF6CC42A2FB001057
:10B630004FEA9006796AB6FBF1F51D9B40F67462FD
:10B64000C2F20002D1184878D65C4FEA064343EABA
:10B6500000208A7840EA02011B916D1A25F07F468E
:10B660001C9600EE906AB8EE601A87ED131AFEF78A
:10B67000C2BA219FF86CB864FEF7BDBA219A92F85D
:10B680005110002940F08381FEF7B5BA219B93F851
:10B690005100002800F07B81FEF7ADBA1D99FA2910
:10B6A00008D942F6C464C2F200044FF013012171BC
:10B6B00002F03BBF40F67462C2F20002535C002B02
:10B6C0007EF499AA1E981C9063E11D9BFA2B08D961
:10B6D00042F6C464C2F200044FF01303237102F077
:10B6E00024BF40F67462C2F20002D05C00283EF42F
:10B6F00082AA1E991C914CE142F6C460C2F200007D
:10B700004FF00102027102F010BF1D99132908D9F0
:10B7100042F6C464C2F200044FF01203237102F037
:10B7200004BF42F6FC63C2F20003585C1E9A10424A
:10B730007EF461AA1F991C912BE11D98132808D94A
:10B7400042F6C464C2F200044FF01202227102F009
:10B75000ECBE42F6FC62C2F20002115C1E9B194272
:10B760003EF449AA1F981C9013E11D99FA2908D9A3
:10B7700042F6C464C2F200044FF01301217102F0DA
:10B78000D4BE40F67463C2F20003585C00287EF415
:10B7900032AA1E9A1C922DE11D9BFA2B08D942F663
:10B7A000C464C2F200044FF01303237102F0BDBE63
:10B7B00040F67460C2F20000C25C002A3EF41BAA8C
:10B7C0001E991C9116E11D98FA2808D942F6C46406
:10B7D000C2F200044FF01302227102F0A6BE40F63E
:10B7E0007462C2F20002115C1E9B99427EF603AAAB
:10B7F0001F981C90CDE01D99FA2908D942F6C4641F
:10B80000C2F200044FF01303237102F08EBE40F623
:10B810007463C2F20003585C1E9A9042FEF4EBA9D6
:10B820001F991C91B5E01D98FA2808D942F6C46406
:10B83000C2F200044FF01302227102F076BE40F60D
:10B840007462C2F20002115C1E9B99427EF4D3A97D
:10B850001F981C909DE01D99FA2908D942F6C464EE
:10B86000C2F200044FF01303237102F05EBE40F6F3
:10B870007463C2F20003585C1E9A90423EF4BBA966
:10B880001F991C9185E01D98FA2808D942F6C464D6
:10B89000C2F200044FF01302227102F046BE40F6DD
:10B8A0007462C2F20002115C1E9B99423EF6A3A98B
:10B8B0001F981C906DE01D99FA2908D942F6C464BE
:10B8C000C2F200044FF01303237102F02EBE40F6C3
:10B8D0007463C2F20003585C1E9A9042BEF48BA9B6
:10B8E0001F991C9155E0219890F847201D998A4294
:10B8F0007EF481A91E9B1C937CE0219890F8472040
:10B900001D998A423EF477A91E9B1C9372E02198F0
:10B9100090F847201D998A427EF66DA91E9B1C93C4
:10B9200068E0219890F847201D998A42FEF463A9A7
:10B930001E9B1C935EE0219890F847201D998A4237
:10B94000BEF459A91E9B1C9354E0219890F84720FF
:10B950001D998A423EF64FA91E9B1C934AE09DF812
:10B9600074000DF16B01FDF761F98DF86A009DF827
:10B970006B1031B142F6C464C2F20004217102F0CE
:10B98000D4BD00283EF437A91E981C9001E01D9AF2
:10B990001C921C984AF20003C0F6010393F82E2073
:10B9A00093F82F1041EA0223834208D242F6C4647E
:10B9B000C2F200044FF00900207102F0B6BD42F659
:10B9C0001C76C2F200063060FEF715B90DF1700C5E
:10B9D000FBF780FE1C900028D9D0FEF70CB90DF1C2
:10B9E000700CFBF777FE1C900028D0D1FEF703B94E
:10B9F0001D9B1C93219A136A052B08D942F6C46437
:10BA0000C2F200044FF00A03237102F08EBD03F16D
:10BA1000020042F61C71C2F20001096842F82010CF
:10BA200003F10103219A1362B3E70DF1700CFBF7E8
:10BA300051FE1C900028DBD0FEF7DDB80DF1700C34
:10BA4000FBF748FE1C900028D2D1FEF7D4B80DF1C8
:10BA5000700CFBF73FFE1C901D9988427EF4CBA82A
:10BA60001E981C9095E70DF1700CFBF733FE1C90AF
:10BA70001D9A90423EF4BFA81E9B1C9389E70DF1CE
:10BA8000700CFBF727FE1C901D9988427EF6B3A828
:10BA90001E981C907DE70DF1700CFBF71BFE1C90AF
:10BAA0001D9A9042FEF4A7A81E9B1C9371E70DF10E
:10BAB000700CFBF70FFE1C901D998842BEF49BA8EA
:10BAC0001E981C9065E70DF1700CFBF703FE1C90AF
:10BAD0001D9A90423EF68FA81E9B1C9359E79DF835
:10BAE00074000DF16B01FDF771F88DF86A009DF897
:10BAF0006B1031B142F6C464C2F20004217102F04D
:10BB000014BD00283EF477A81E981C9041E79DF8CC
:10BB100074000DF16B01FDF759F88DF86A009DF87E
:10BB20006B3033B142F6C461C2F200010B7102F016
:10BB3000FCBC00287EF45FA81E9A1C9229E70DF138
:10BB4000700CFBF7EFFD40F67460C2F200001E9B24
:10BB5000C25C1D990A423EF44EA81F981C9018E73B
:10BB60000DF1700CFBF7DEFD40F67462C2F20002CC
:10BB70001E9BD15C1D9801427EF43DA81F9A1C9229
:10BB800007E70DF1700CFBF7CDFD40F67461C2F2D2
:10BB900000011E9BC85C1D9A10427EF42CA81F99C0
:10BBA0001C9127E70DF1700CFBF7BCFD40F67460AB
:10BBB000C2F200001E9BC25C1D990A423EF41BA803
:10BBC0001F981C9016E798F8005045F0080088F878
:10BBD0000000FEF739B80DF1700CFBF77BFD8DF816
:10BBE0006A00219991F851201D9BD1181C911E9A31
:10BBF000C2F1FB03994208D942F6C464C2F20004C0
:10BC00004FF01303237102F090BC4FF000061B9617
:10BC10001E9FE7B11C9940F67465C2F200056A5C8C
:10BC2000824232D007F1FF3240F67463C2F2000361
:10BC30005B1840F67466C2F20006C6F10105C1F158
:10BC40000107BE1B12F0010F18D002F0CCBC4FF060
:10BC5000FF001B9019E013F8019F02F1FF3E4845D9
:10BC600003D11C911B971E920FE07246E918F7183A
:10BC700013F801CF604542F0C284F2E7E918F718E3
:10BC8000002AE8D11C911E92E1E70DF1700C9DF89D
:10BC90006C00FBF707FDFDF7AEBF0DF1700CFBF775
:10BCA00019FD42F64861C2F2000108704FF001022E
:10BCB0001C920C9194E0219890F851101D9BCA1889
:10BCC0001C92F92A08D942F6C464C2F200044FF06B
:10BCD0001300207102F029BC1E981B900DF1700C0E
:10BCE00026AD45F0010122AE46F001024FF00003FF
:10BCF000FBF72AFDFDF77FBF219991F851201D9B8D
:10BD0000D0181C90FA2808D942F6C464C2F2000484
:10BD10004FF01301217102F008BC1F9F1E98B8421A
:10BD200028BF38461B900DF1700C26AD45F001017F
:10BD300022AE46F001024FF00003FCF73FFDFDF795
:10BD40005ABF0DF1700CFBF7C5FC034642F648667E
:10BD5000C2F2000630464FF0100148F2E822C0F669
:10BD6000010207F027FE1C900C9639E01E9A1C92E7
:10BD70001F9B1B934FF000000C9031E04FF0FF3100
:10BD80001C910C912CE0219EF06C9DF878109DF890
:10BD90007C2042F64866C2F2000600964FF010037F
:10BDA00001934FF00103FDF77FFB4FF0FF321C9230
:10BDB0000C9615E02198C06C9DF878109DF87C20B9
:10BDC00042F64866C2F2000600964FF01003019357
:10BDD0004FF00003FDF768FB4FF0FF311C910C960C
:10BDE0001D9B03F10500C1B20B91A3F1FB02032AD5
:10BDF00023D840F6B873C2F200034FF411700B99C8
:10BE000000FB013292F82032032B08D042F6C460C6
:10BE1000C2F200004FF04804047102F086BB40F605
:10BE2000B876C2F200064FF411770B9807FB006753
:10BE300007F104074FF0000605E0219F97F85160D5
:10BE4000F6184FF00007DDF870A0BAF1FF3F11D1EE
:10BE50004FF0FF0A4FF00009C84642F6C461C2F233
:10BE600000010F9140F67462C2F200020D920E952D
:10BE70000C9D05E0BAF1000FECD14FF000095CE039
:10BE80001D9BA3F1FB03032B10D8D7F80061FF2EF5
:10BE900014BF01364646D7F80401864206D1404613
:10BEA000FCF7F8FBD7F804118E42F8D0B5F1FF3F4C
:10BEB00010D1219850F8341F0A68D2F800C04946C2
:10BEC00010AA4FF00103E0470F9B187158B10E9D67
:10BED00002F02BBB25B115F809308DF8403002E097
:10BEE0001B9A8DF840201C98B0F1FF3F02D19DF8BD
:10BEF000401011B31D9AA2F1FB02032A07D8D7F80C
:10BF000000319DF84020FA54C7F8006111E0FA2E84
:10BF100009D90E9D42F6C464C2F200044FF0130129
:10BF2000217102F002BB9DF840300D98835506F157
:10BF3000010609F10109D145A2D31D9EA6F1FB0618
:10BF4000032E04D80B98FBF753FEFDF754BE219F38
:10BF500097F8515009EB050E87F851E0FDF74BBEFD
:10BF60001D9AA2F1FB00032859D802F10502D7B2AD
:10BF700040F6B871C2F200014FF4117202FB0713D0
:10BF800093F82002032808D042F6C464C2F20004E9
:10BF90004FF04803237102F0C8BA40F6B876C2F2F7
:10BFA00000064FF4117505FB076505F104051E99A0
:10BFB00001F1FF321E9269B34FF0000842F61C797E
:10BFC000C2F200094AF2000AC0F6010AD5F800617F
:10BFD000FF2E14BF01364646D5F804319E4206D1E5
:10BFE0004046FCF757FBD5F804018642F8D0D9F853
:10BFF0000030D5F800211AF80310A95403F1010309
:10C00000C9F80030C5F800611E9E06F1FF301E9091
:10C01000002EDBD13846FBF7EBFDFDF7ECBD1E9B98
:10C020001C93219991F8510082181B92C3F1FB06D1
:10C03000B24208D942F6C464C2F200044FF01300C1
:10C04000207102F072BAC71881F851701C9A02F17F
:10C05000FF351C95002A3DF4CEAD42F61C76C2F2A7
:10C06000000636681B9F40F67463C2F20003D919BC
:10C070004AF20000C0F6010030184FF0000305F04E
:10C08000010810F803E001F803E003F10103934213
:10C0900042F09A820DE010F8039001F8039003F14A
:10C0A000010310F8038001F8038003F101039342B8
:10C0B000F1D1E819A91901F1010142F61C72C2F28D
:10C0C000000211604FF0FF331C9300F101001B9040
:10C0D000FDF791BD4FF000028DF86A20219890F88D
:10C0E00051201D9BD1181C911E9A1B92C2F1FB037B
:10C0F000994208D942F6C464C2F200044FF0130218
:10C10000227102F012BA40F67467C2F2000707EB20
:10C1100001099DF87CA042F61475C2F200052E6854
:10C12000806B3118335CFF2B52D088464FF00107EB
:10C1300008970B9498F8014004EB032342F614751A
:10C14000C2F200052E68F0184FF000011C919DF816
:10C150006A20002A02F00D82F75C00F1010002F073
:10C160000ABA9DF86A5015B15FB90B9C02E060787D
:10C1700038B90B9C219E96F851001D1886F8515035
:10C1800029E014F8015F19F803A046B9284607F022
:10C19000B5FBC5B2504607F0B1FB5FFA80FA5545D2
:10C1A00008D11C9B03F101031C9307F1FF371B9976
:10C1B0009942D6D2B246089A02F10102089218F8C2
:10C1C000023FFF2BB6D10B9C4FF00007089702E00F
:10C1D0004FF0000208920DF1700C0899C8B2FBF7FD
:10C1E00061FAFDF708BD4FF001018DF86A1075E79F
:10C1F0000DF1700CFBF76EFA034642F64866C2F288
:10C20000000630464FF0100148F2F022C0F601025D
:10C2100007F0D0FB1C900C96E2E50DF1700CFBF7DB
:10C2200059FA034642F64866C2F2000630464FF01D
:10C23000100148F2F822C0F6010207F0BBFB1C9087
:10C240000C96CDE50DF1700CFBF744FA034642F66F
:10C250004866C2F2000630464FF0100148F2FC2258
:10C26000C0F6010207F0A6FB1C900C96B8E50DF194
:10C27000700CFBF72FFA034642F64866C2F200063E
:10C2800030464FF0100148F20432C0F6010207F0C8
:10C2900091FB1C900C96A3E5219991F8513003F184
:10C2A000010381F85130FDF7A6BC1D9E40F6746273
:10C2B000C2F20002975D07F101079755FDF79BBC9D
:10C2C000219D95F8470000F1010085F84700FDF732
:10C2D00092BC9DF874000DF16B01FCF777FC0DF139
:10C2E000700CFBF7DFF99DF86B1000293DF483AC6F
:10C2F00042F6C464C2F20004217102F016B99DF83E
:10C3000074000DF16B01FCF7C9FC0DF1700CFBF72B
:10C31000C9F99DF86B30002B3DF46DAC42F6C46258
:10C32000C2F20002137102F000B91D981C904FF088
:10C3300000011B914FF001038DF86A309DF87000E9
:10C340000DF16B01FCF742FC9DF86B1099B920B11F
:10C350009DF86A201B9810431B909DF86A304FEAA5
:10C3600043018DF86A101C9A02F101021C9211F02F
:10C37000FE0FE3D10AE09DF86A00012806D142F6DB
:10C38000C464C2F20004217102F0CFB80DF1700C48
:10C390009DF86C00FBF786F9FDF72DBC1D9B1C93E7
:10C3A0004FF000011B914FF001028DF86A209DF8BB
:10C3B00070000DF16B01FCF771FC9DF86B309BB9BF
:10C3C00020B19DF86A001B9901431B919DF86A20DA
:10C3D0004FEA42038DF86A301C9800F101001C906E
:10C3E00013F0FE0FE3D10AE09DF86A10012906D18F
:10C3F00042F6C464C2F20004237102F096B80DF153
:10C40000700C9DF86C00FBF74DF9FDF7F4BB9DF83F
:10C4100074000DF16B01FCF709FC8DF86A009DF8C2
:10C420006B3033B142F6C462C2F20002137102F003
:10C430007CB80DF1700CFBF735F9FDF7DCBB1D98EE
:10C440001C904FF000011B914FF001038DF86A30F2
:10C45000219A92F8470003420ED09DF870000DF12A
:10C460006B01FCF7E3FB9DF86B309BB920B19DF8A5
:10C470006A101B9A0A431B929DF86A004FEA400318
:10C480008DF86A301C9901F101011C9113F0FE0333
:10C49000DED10AE09DF86A20012A06D142F6C46482
:10C4A000C2F20004237102F040B81B9E219F87F85E
:10C4B0004760FDF7A0BB9DF874000DF16B01FCF720
:10C4C0001DFC0DF1700CFBF7EDF89DF86B000028DA
:10C4D0003DF491AB42F6C461C2F20001087102F072
:10C4E00024B81D9B1C93D8B20DF16B01FCF706FC20
:10C4F0001B909DF86B0030B142F6C464C2F2000498
:10C50000207102F012B84FF001058DF86A501C9AA4
:10C5100051191C91C8B20DF16B01FCF7EFFB9DF8AE
:10C520006A6000FA06F01B9F07431B9706F101069D
:10C530008DF86A601C9901F101011C91F3B2072B7F
:10C54000E8D90DF1700C9DF86C00FBF7ABF8FDF726
:10C5500052BB0DF1700C219890F85100FBF7A2F836
:10C56000FDF749BBFDF747BB42F6BD65C2F20005CA
:10C570004FF001022A70FDF73EBB42F6BD66C2F2E3
:10C5800000064FF000073770FDF735BB21984FF0DC
:10C5900000014FF0540207F043FE4FF000012191DB
:10C5A00042F65863C2F200031C6804F1FF301860C1
:10C5B00001F017BF42F65863C2F2000318683F2823
:10C5C00008D942F6C464C2F200044FF0300222716E
:10C5D00001F0ABBF4FF001051C9541F6CC06C2F24D
:10C5E0000006B76D002F41F0D18705E0D2F8AC10FE
:10C5F000002949D11C9301E04FF001031D9F41F632
:10C60000CC05C2F200054FF0540606FB03F3EA180E
:10C61000EF5057601E9982F852104FF00A00506296
:10C62000104600F13400219901F134014FF010025D
:10C6300007F0D2FD1C9B06FB035000F1440021993A
:10C6400001F144014FF0040207F0C6FD1C9F06FBF8
:10C65000075000F14800219901F148014FF008020C
:10C6600007F0BAFD219A92F851101C9806FB00556C
:10C6700085F8511042F65866C2F20006336803F19D
:10C6800001033360FDF7B7BA03F101052B4602F150
:10C690005402D2F8AC00002841F08687AAE71C9328
:10C6A000FDF7A9BA219A92F852101E9182E70DF176
:10C6B000700CFBF70FF81E907CE71D9F219981F805
:10C6C0005170FDF798BA0DF1700C9DF87400FAF7EF
:10C6D000E9FFFDF790BA2198836A002B3DF48BAAFD
:10C6E000F9F7FEFA21998A6A801A496A1D9B01FBB3
:10C6F00003F303EB83029042BDF47DAA1E981C90C5
:10C70000FFF747B9F9F7ECFA219DA862FDF773BA74
:10C7100042F6FC61C2F200014A7D1E995318152BA6
:10C7200008D942F6C461C2F200014FF012030B7146
:10C7300001F0FBBE1D9BC2F1FB00834208DD42F607
:10C74000C464C2F200044FF01302227101F0EDBE86
:10C7500042F6FC66C2F20006701840F67467C2F238
:10C760000007F91807F038FDFDF745BA98F80050B2
:10C7700045F0100088F80000FDF766BA219E96F893
:10C780004770002F0CBFFF22002286F84720FDF7DC
:10C7900032BA219991F847306FEA030581F8475082
:10C7A000FDF729BA0DF1700CFAF7BCFF1E9E40F69A
:10C7B0007467C2F20007B85D1D9A4240BA55FDF792
:10C7C0001ABA2199886B1D9B1A181C9292E1219923
:10C7D000C86B8B6BC2181C928CE12199086C40B914
:10C7E00042F6C464C2F200044FF02003237101F04A
:10C7F0009CBE00F1FF350D64FDF7FDB9219A116C67
:10C8000001F10101116400297DF4F5A942F6C4602B
:10C81000C2F200004FF02004047101F086BE219B9B
:10C820005A6B1168486840B942F6C464C2F2000409
:10C830004FF01E01217101F078BE0DF1700CFAF776
:10C8400049FF1C90219850F8346F33685E681D9939
:10C850001CAA4FF00103B04742F6C462C2F20002C4
:10C86000107100283DF4C7A901F05FBE0DF1700CF6
:10C87000FAF730FF1C902BE10DF1700CFAF72AFF4C
:10C88000219FF863FDF7B7B90DF1700CFAF722FF9D
:10C89000219D2864FDF7AFB9219850F8346F3368B3
:10C8A0001E681D991CAA4FF00103B04742F6C462EE
:10C8B000C2F200021071002841F037860DF1A80C79
:10C8C0001CF8380DFAF7EEFEFDF795B92198416B8B
:10C8D0000DF1700C0879FAF7E5FEFDF78CB90DF152
:10C8E000700C219F97F83C00FAF7DCFEFDF783B946
:10C8F000219B1A6CFF2A08D942F6C464C2F20004D4
:10C900004FF02000207101F010BE0DF1700CD0B27C
:10C91000FAF7C8FEFDF76FB9219D6E6B31688F681D
:10C92000B84701EE900AB8EE612A219B83ED132AE5
:10C93000FDF761B9219AD2ED0E2AB8EE623A82ED86
:10C94000133AFDF758B92198D0ED103AB8EE634A82
:10C9500080ED134AFDF74FB92199D1ED134ABCEE92
:10C96000E45A8DED1C5AC5E0219BD3ED135A9FED7F
:10C97000C26AF4EEC65AF1EE10FA08DB42F6C4645D
:10C98000C2F200044FF02002227101F0CEBDFCEE95
:10C99000E56AC3ED106AFDF72EB9219850F8346F9F
:10C9A00031680E681D991CAA4FF00403B04742F687
:10C9B000C463C2F200031871002841F0B6851C98C8
:10C9C000FAF7EAFC219DA864FDF715B9219850F803
:10C9D000342F166836681D991CAA4FF00403B0471F
:10C9E00042F6C461C2F200010871002841F09D8541
:10C9F0001C98FAF7D1FC219FF864FDF7FCB8219848
:10CA0000436B1A68516841B942F6C464C2F200042B
:10CA10004FF01E00207101F088BDC06CFAF792FC47
:10CA20001C90219850F8346F33685E681D991CAAD9
:10CA30004FF00403B04742F6C462C2F20002107124
:10CA400000283DF4D8A801F070BD1D9A2198C36B51
:10CA5000C3F1FB018A4208D942F6C464C2F2000461
:10CA60004FF01300207101F060BD50F8347F3E6834
:10CA700036684FF0000140F67467C2F20007BA183A
:10CA8000B04742F6C463C2F20003187100283DF4B7
:10CA9000B2A801F04ABD219850F8342F11680E68F1
:10CAA0001D991BAA4FF00403B04742F6C463C2F2BB
:10CAB00000031871002841F038851B9882B2C0F33A
:10CAC000072141EA022398B21C9013E01D9A1C92A0
:10CAD0001C982199FAF79CFE8DF86B0000283DF414
:10CAE0008AA842F6C464C2F20004207101F01DBDA0
:10CAF0001D991C912198426B11688B6898471C996D
:10CB0000884208D242F6C464C2F200044FF01F000B
:10CB1000207101F00ABD219DA963FDF76CB81D9D30
:10CB2000219FFD63FDF767B81D9E219B1E64FDF7E5
:10CB300062B82198826B1D99531A1C93DAE71E9AEA
:10CB40002198C36B9918152908D942F6C464C2F21A
:10CB500000044FF01200207101F0E7BC42F6FC67C0
:10CB6000C2F200077B7550F8346F31680E681D996A
:10CB7000BA18B04742F6C463C2F200031871002825
:10CB80003DF439A801F0D1BC2198426B1668766853
:10CB900046B942F6C461C2F200014FF01E020A71AA
:10CBA00001F0C3BC1D9AC36BC3F1FB018A4208D9D3
:10CBB00042F6C464C2F200044FF01300207101F089
:10CBC000B4BC00F134004FF0000140F67467C2F2CB
:10CBD0000007BA18B04742F6C463C2F200031871E6
:10CBE00000283DF408A801F0A0BCF7F74DFC002890
:10CBF0007DF401A81D9B1C93FEF7CBBEF7F744FC08
:10CC000000283CF4F8AF1D981C90FEF7C2BE1D9999
:10CC1000072908D942F6C464C2F200044FF00502A5
:10CC2000227101F082BCC8B24FF00001F7F7EAFBB5
:10CC300007EE100AB8EE470A219F87ED130AFCF7AA
:10CC4000DABF1D9B072B08D942F6C460C2F2000070
:10CC50004FF00501017101F068BCD8B24FF001013D
:10CC6000F7F7D0FB07EE900AF8EE670A219DC5EDB5
:10CC7000130AFCF7C0BF00BF000080471D9A072AB7
:10CC800008D942F6C464C2F200044FF005032371D0
:10CC900001F04BBCD0B24FF00001F7F723FBFCF7DB
:10CCA000AABF1D98072808D942F6C461C2F2000144
:10CCB0004FF005020A7101F038BCC0B24FF001011B
:10CCC000F7F710FBFCF797BF1D9B072B08D942F61F
:10CCD000C464C2F200044FF00500207101F025BCCD
:10CCE000D8B24FF00001F7F74DFBFCF784BF1D9958
:10CCF000072908D942F6C463C2F200034FF00502C7
:10CD00001A7101F012BCC8B24FF00101F7F73AFBFB
:10CD1000FCF771BF9DF87400F4F754FA00287CF416
:10CD20006AAF42F6C464C2F200044FF028002071DA
:10CD300001F0FBBB9DF874001CA9F4F765FA40B93B
:10CD400042F6C461C2F200014FF028030B7101F0FA
:10CD5000ECBB9DED1C1AF8EE411A219EC6ED131A8C
:10CD6000FCF749BF219A92ED132A9DF87400FCEE5E
:10CD7000C22A12EE901AF4F76BFA00287CF43BAF4B
:10CD800042F6C464C2F200044FF02800207101F0A2
:10CD9000CCBBFCF730BF0DF1700CFAF79BFC30B93F
:10CDA000219F97F847502E1C18BF012601E04FF035
:10CDB0000106219981F84760FCF71DBF9DF874605A
:10CDC0000DF1700CFAF786FC014630464FF0010277
:10CDD000FCF700F88DF86B0000283CF40CAF42F62D
:10CDE000C463C2F20003187101F09FBB0DF1700C17
:10CDF000FAF770FC01468DF86A009DF87400FBF7A5
:10CE0000ABFF8DF86B0000283CF4F5AE42F6C4622F
:10CE1000C2F20002107101F088BB1D981C904FF007
:10CE200001038DF86A301E46219A92F847100B4292
:10CE300008D092F846109DF8700019403246FBF772
:10CE4000C9FF68B99DF86A304FEA43008DF86A005F
:10CE50001C9A02F101021C9210F0FE03E4D10CE0D6
:10CE60009DF86A10012908D19DF86B4042F6C46014
:10CE7000C2F20000047101F058BB0DF1700CFAF71A
:10CE800029FC0DF1700CFAF725FCFCF7B4BE9DF8F7
:10CE900074004FF001010A46FBF79CFF8DF86B0010
:10CEA00000283CF4A8AE42F6C462C2F2000210713F
:10CEB00001F03BBB9DF874004FF000014FF0010200
:10CEC000FBF788FF8DF86B0000283CF494AE42F627
:10CED000C463C2F20003187101F027BB0DF1700C9E
:10CEE000FAF7F8FB219F97F84750284387F8470047
:10CEF000FCF781BE1D980DF1A80C4CF8380DFBF71E
:10CF000089F800287CF477AE42F61C76C2F200065F
:10CF10000899316001F087BA10A8FAF719FF0146A5
:10CF200040B19DF84000022804D0CE484FF00D02D9
:10CF300007F052F90DF1700C9DF84000FAF7B2FBC2
:10CF4000FCF759BEFBF7BAFBFCF755BE0DF1700CB0
:10CF5000FAF7C0FBFCF74FBE1D9E142E08D942F60F
:10CF6000C464C2F200044FF01203237101F0DDBA71
:10CF70000DF1700CFAF7AEFB42F6FC62C2F2000251
:10CF80009055FCF738BE0DF1700CFAF7A3FB42F692
:10CF9000FC67C2F200077875FCF72DBE0DF1700C2E
:10CFA000219D95F84700FAF77DFBFCF724BE1D99FB
:10CFB000142908D942F6C460C2F200004FF01202F0
:10CFC000027101F0B2BA0DF1700C42F6FC66C2F2C9
:10CFD0000006705CFAF766FBFCF70DBE0DF1700CF5
:10CFE00042F6FC63C2F20003587DFAF75BFBFCF7E4
:10CFF00002BE1D9E102E08D942F6C464C2F200047F
:10D000004FF01201217101F090BA219FB86CFAF72C
:10D0100099F942F6FC65C2F20005A851FCF7EBBD98
:10D020001D98FA2808D942F6C463C2F200034FF0F3
:10D0300013021A7101F079BA0DF1700C40F67466A2
:10D04000C2F20006305CFAF72DFBFCF7D4BD0DF1FF
:10D05000700CFAF767FB40F67467C2F200071E9D7A
:10D06000795D1D9801420DF1700C0CBF0020FF206E
:10D07000FAF718FBFCF7BFBD1D9BF92B08D942F648
:10D08000C461C2F200014FF013020A7101F04DBAFF
:10D0900040F67462C2F20002D15A1C9100293CF49D
:10D0A000AAADFEF776BC1D9BFA2B08D942F6C464E4
:10D0B000C2F200044FF01302227101F036BA40F6BA
:10D0C0007460C2F20000C15C002943D1FCF793BD3B
:10D0D0001D9BFA2B08D942F6C464C2F200044FF03B
:10D0E0001302227101F021BA40F67460C2F200000E
:10D0F000C15C79B3FCF77FBD0DF1700CFAF7EAFA69
:10D100001C9038BBFCF777BD0DF1700CFAF70AFBE9
:10D1100040F67460C2F200001E9BC15C1D9A114271
:10D1200018D0FCF768BD0DF1700CFAF7FBFA40F669
:10D130007460C2F200001E9BC15C1D9A114209D1AD
:10D14000FCF759BD0DF1700CFAF7C4FA1C900028D9
:10D150007CF451AD2198036A43B942F6C464C2F22B
:10D1600000044FF00301217101F0DFB903F1FF3535
:10D17000056203F1010350F8236042F61C77C2F206
:10D1800000073E60FCF737BD219F97F847504FEAF4
:10D19000D51646EA450087F84700FCF72CBD219BD1
:10D1A00093F847204FEA520141EAC21783F84770CB
:10D1B000FCF721BDFAF79EFEFCF71DBD42F6CC65DB
:10D1C000C2F20005EE784FF0010000FA06F02B796C
:10D1D00023EA00032B71FCF70EBD42F6C464C2F2D1
:10D1E00000044FF00102227101F09FB942F6CC61B8
:10D1F000C2F20001CF7847B942F6CC60C2F200001B
:10D200004FF00603C370FCF7F6BC07F1FF3542F69A
:10D21000CC66C2F20006F570FCF7EDBC42F6CC62BB
:10D22000C2F20002117801F1FF37FDB215701679D4
:10D23000FF2E0BD1632D7CF6DEAC42F6CC61C2F240
:10D2400000014FF063020A70FCF7D5BC172D7CF685
:10D25000D2AC42F6CC60C2F200004FF0170303706C
:10D26000FCF7C9BC7A0E002042F6CC67C2F2000778
:10D270007D7805F1FF36F0B278703B79FF2B0BD14A
:10D2800000287CF4B8AC42F6CC67C2F200074FF03D
:10D290000C057D70FCF7AFBC3B287CF6ACAC42F6CD
:10D2A000CC61C2F200014FF03B024A70FCF7A3BC14
:10D2B00042F6C464C2F200044FF00100207101F094
:10D2C00034B942F6C463C2F200034FF00101197190
:10D2D00001F02BB942F6C464C2F200044FF001021F
:10D2E000227101F022B942F6C460C2F200004FF090
:10D2F0000103037101F019B942F6CC66C2F20006CF
:10D30000F778052F08D942F6CC61C2F200014FF040
:10D310000002CA70FCF76FBC07F1010742F6CC654A
:10D32000C2F20005EF70FCF766BC42F6CC60C2F2B8
:10D330000000037803F10103DEB206700779FF2FC6
:10D340000BD1632E7CF657AC42F6CC60C2F20000E3
:10D350004FF000020270FCF74EBC172E7CF64BAC6F
:10D3600042F6CC65C2F200054FF000012970FCF7CF
:10D3700042BC42F6CC66C2F20006737803F10103A8
:10D38000DFB277703579FF2D0BD10C2F7CF633ACE3
:10D3900042F6CC66C2F200064FF001027270FCF752
:10D3A0002ABC3B2F7CF627AC42F6CC61C2F20001CE
:10D3B0004FF000004870FCF71EBC42F6C464C2F295
:10D3C00000044FF00103237101F0AFB842F6CC67BF
:10D3D000C2F20007FD784FF0010101FA05F138793A
:10D3E00081EA00063E71FCF706BC0DF1700CFAF7FD
:10D3F00071F942F6CC62C2F200021071FCF7FBBB7D
:10D400000DF1700CFAF766F9062842F6CC63C2F209
:10D41000000392BFD8700027DF70FCF7ECBB0DF162
:10D42000700CFAF757F942F6CC65C2F20005287085
:10D43000FCF7E1BB0DF1700CFAF74CF942F6CC6148
:10D44000C2F200014870FCF7D6BB0DF1700CFAF780
:10D4500041F942F6CC66C2F20006B070FCF7CBBBD5
:10D460000DF1700C42F6CC60C2F200000079FAF7C0
:10D4700019F9FCF7C0BB0DF1700C42F6CC62C2F298
:10D480000002D078FAF70EF9FCF7B5BB0DF1700C7D
:10D4900042F6CC63C2F200031878FAF703F9FCF7FE
:10D4A000AABB0DF1700C42F6CC67C2F20007787887
:10D4B000FAF7F8F8FCF79FBB0DF1700C42F6CC655B
:10D4C000C2F20005A878FAF7EDF8FCF794BB42F633
:10D4D000C464C2F200044FF00101217101F025B8CB
:10D4E0001D9A0F2A08D942F6C464C2F200044FF014
:10D4F0002700207101F019B840F67476C2F20006D8
:10D5000006EB820042F6CC63C2F2000316F82270EA
:10D510001F7045785D704FF000019970D970827866
:10D520001A71FCF768BB42F6C463C2F200034FF005
:10D530000101197100F0F9BF42F6CC66C2F2000693
:10D54000F7784FF0010505FA07F5327945EA020050
:10D550003071FCF750BB42F6C464C2F200044FF0D5
:10D560000103237100F0E1BF42F6C461C2F2000181
:10D570004FF001020A7100F0D8BF4FF00006139679
:10D5800012961196199642F6CC67C2F200073D78C2
:10D5900005F164051695787800F1FF331593B97895
:10D5A000149111A806F03EFC179A1AB102F1FF3748
:10D5B000FEB201E04FF0060642F6CC65C2F200056D
:10D5C000EE70FCF718BB1D9A0F2A08D942F6C46406
:10D5D000C2F200044FF02702227100F0A6BF40F60D
:10D5E0007470C2F2000000EB820142F6CC63C2F21A
:10D5F00000031E7800F822605F784F701D798D70EF
:10D60000FCF7F9BA42F6C460C2F200004FF0010123
:10D61000017100F08ABF0DF1700C219B93F850004E
:10D62000FAF740F8FCF7E7BA40F6B474C2F2000427
:10D63000227812F0010F08D142F6C460C2F2000055
:10D640004FF03001017100F070BF42F65860C2F235
:10D650000000016841B942F6C464C2F200044FF010
:10D660003102227100F061BF40F6B473C2F20003D0
:10D670001C7804F0FE0242F00400187042F6AC611F
:10D68000C2F200014FF000030B6000F0AABE40F6AA
:10D69000B473C2F200031C7814F0010F08D142F6F3
:10D6A000C460C2F200004FF03002027100F03DBFD2
:10D6B00042F65862C2F20002106840B942F6C463F2
:10D6C000C2F200034FF034041C7100F02EBF40F68C
:10D6D000B471C2F200010B7803F0FE0444F00202C0
:10D6E0000A7042F6AC60C2F200004FF00001016027
:10D6F00000F077BE219E96F846700DF1700CF9F798
:10D70000E9FF219D391A95F8503003F001000A1AFB
:10D710001C9285F84720FF2A94BF0022012285F839
:10D720005020FCF768BA1D9BFA2B08D942F6C46456
:10D73000C2F200044FF01301217100F0F6BE40F672
:10D740007466C2F200061E9FF754FCF754BA4FF0FD
:10D7500000051C951AE04FF001001C9016E04FF0F8
:10D7600002021C9212E04FF003031C930EE04FF0F4
:10D7700004061C960AE04FF005071C9706E04FF0E0
:10D7800006011C9102E04FF007051C951D991B91A5
:10D790001C98FAF7C3FBFCF72EBA0DF1700CF9F7E1
:10D7A000C1FF1E9B40F67462C2F20002D05C1D9E57
:10D7B0000643D654FCF71FBA1D9B132B08D942F61B
:10D7C000C464C2F200044FF01202227100F0ADBE38
:10D7D00042F6FC67C2F200071E99F954FCF70BBA37
:10D7E00042F6FC65C2F200051D986875FCF703BAA5
:10D7F00043F23C23C2F20003196841B942F6C46007
:10D80000C2F200004FF00102027100F08EBE4E68BD
:10D810001D981E994FF001020DF16A03B0478DF873
:10D820006B009DF86A20D2F1010138BF0021219BD5
:10D8300083F8501000283CF4DEA942F6C464C2F21A
:10D840000004207100F071BE43F23C21C2F20001DD
:10D850000B6843B942F6C460C2F200004FF0010108
:10D86000017100F062BE1A681D981E9990478DF8EC
:10D870006B0000283CF4BFA942F6C464C2F2000465
:10D88000207100F052BE43F23C23C2F200031A683A
:10D8900042B942F6C460C2F200004FF001010171CA
:10D8A00000F043BE56681D981E994FF000020DF11E
:10D8B0006A03B0478DF86B009DF86A10D1F1010240
:10D8C00038BF0022219B83F8502000283CF493A904
:10D8D00042F6C464C2F20004207100F026BE09982A
:10D8E0001E99FAF715F9099040B942F6C463C2F2DD
:10D8F00000034FF01700187100F017BE099A136863
:10D900005B6943B942F6C461C2F200014FF01502EF
:10D910000A7100F00ABE099880689DF8741042F6FA
:10D92000FC62C2F2000298478DF86B0000283CF4BC
:10D9300062A942F6C464C2F20004207100F0F5BD91
:10D9400009981E99FAF7E4F8099040B942F6C463C1
:10D95000C2F200034FF017021A7100F0E6BD099FF2
:10D9600039688F6947B942F6C460C2F200004FF0CF
:10D970001501017100F0D9BD42F6FC66C2F2000645
:10D98000099A90689DF8741032460DF16A03B84701
:10D990008DF86B009DF86A30337000283CF42BA999
:10D9A00042F6C464C2F20004207100F0BEBD0998C2
:10D9B0001E99FAF7ADF809901D997F2909D1061C27
:10D9C00018BF012642F6FC65C2F200052E70FCF776
:10D9D00012B9099840B942F6C463C2F200034FF08D
:10D9E0001700187100F0A1BD099B1A68536843B96C
:10D9F00042F6C461C2F200014FF015020A7100F054
:10DA000094BD09988068C9B242F6FC62C2F2000275
:10DA100098478DF86B0000283CF4EDA842F6C464EA
:10DA2000C2F20004207100F080BD09981E99FAF737
:10DA30006FF8099040B942F6C463C2F200034FF098
:10DA400017021A7100F071BD099F39688F6847B9D4
:10DA500042F6C460C2F200004FF01501017100F0FF
:10DA600064BD42F6FC66C2F20006099A90689DF811
:10DA7000741032780DF16A03B8478DF86B009DF889
:10DA80006A30337000283CF4B6A842F6C464C2F28F
:10DA90000004207100F049BD09981E99FAF738F882
:10DAA000099040B942F6C461C2F200014FF0170379
:10DAB0000B7100F03ABD099F3868C76847B942F654
:10DAC000C460C2F200004FF01502027100F02DBDDB
:10DAD00042F6FC66C2F20006099988689DF8741047
:10DAE00032460DF16A03B8478DF86B009DF86A3035
:10DAF000337000283CF47FA842F6C464C2F20004EC
:10DB0000207100F012BD09981E99FAF701F80990EA
:10DB100040B942F6C460C2F200004FF01702027131
:10DB200000F003BD099F3868076947B942F6C46130
:10DB3000C2F200014FF015030B7100F0F6BC099E14
:10DB4000D6F808809DF8749042F6FC66C2F2000692
:10DB50003068F9F721FC0246404649460DF16A0358
:10DB6000B8478DF86B009DF86A20327000283CF4AD
:10DB700042A842F6C464C2F20004207100F0D5BC91
:10DB800009981E99F9F7C4FF099040B942F6C46399
:10DB9000C2F200034FF01700187100F0C6BC0999DB
:10DBA0000B68DB6943B942F6C461C2F200014FF071
:10DBB00015020A7100F0B9BC099880689DF87410CC
:10DBC00042F6FC62C2F2000298478DF86B00002812
:10DBD0003CF411A842F6C464C2F20004207100F0C3
:10DBE000A4BC09981E99F9F793FF099040B942F631
:10DBF000C463C2F200034FF01700187100F095BC27
:10DC000009990A68136A43B942F6C461C2F2000175
:10DC10004FF015020A7100F088BC099880689DF8E1
:10DC2000741042F6FC62C2F2000298478DF86B0055
:10DC300000283BF4E0AF42F6C464C2F20004207155
:10DC400000F073BC09981E99F9F762FF099040B97A
:10DC500042F6C461C2F200014FF017030B7100F0ED
:10DC600064BC09990A68536A43B942F6C460C2F2B7
:10DC700000004FF01502027100F057BC099880684F
:10DC80009DF8741010AA98478DF86B001098F9F75A
:10DC900059FB42F6FC61C2F2000108609DF86B304E
:10DCA000002B3BF4A8AF42F6C464C2F20004237117
:10DCB00000F03BBC1D98072808D942F6C464C2F2A4
:10DCC00000044FF00801217100F02FBC42F65C65A2
:10DCD000C2F2000555F83070002F7BF48CAFF7F7D7
:10DCE000FFFF002808BF012042F65C66C2F2000672
:10DCF0001D9A46F83200FBF77EBF1D9B072B08D903
:10DD000042F6C464C2F200044FF00803237100F02D
:10DD10000CBC42F65C60C2F2000050F83350002D9B
:10DD20003BF469AFF7F7DCFF1D9F42F65C66C2F279
:10DD3000000656F83720811A1C9106EBC703586875
:10DD400081428CBF0020C1EB00001B9042F65C6555
:10DD5000C2F2000505EBC7061B9A72604FF0000186
:10DD600045F83710FBF747BF1D9EFA2E07D942F63C
:10DD7000C460C2F200004FF013020271D5E30DF14E
:10DD8000700CF9F7A7FC40F67467C2F20007B855AB
:10DD9000FBF731BF0DF1700CF9F7C4FC0DF1700CFD
:10DDA000F9F798FC1C9050B11E9D40F67462C2F2C7
:10DDB0000002505D1D9E06435655FBF71CBF1E9D7D
:10DDC00040F67466C2F20006735D1D9923EA0107EE
:10DDD0007755FBF710BF1D9B1E9AD118C9B242F6AA
:10DDE000FC60C2F200004175142907D942F6C464F0
:10DDF000C2F200044FF01203237196E342F61C773F
:10DE0000C2F200073D6842F6FC66C2F20006F01856
:10DE10004AF20003C0F60103E91806F0DDF93A689A
:10DE20001E9950183860FBF7E6BE1D9AF82A07D9EC
:10DE300042F6C464C2F200044FF01300207174E390
:10DE4000F7F74EFF00F104004CF6CD47CCF6CC4777
:10DE5000A7FB00154FEA95062199486AB6FBF0F337
:10DE60001C931D9A40F67467C2F200074FEA1345EF
:10DE7000BD54BE184FEA13217170B370FBF7BBBEDF
:10DE80001D9BF82B07D942F6C464C2F200044FF080
:10DE90001301217149E3F7F723FF00F104004CF669
:10DEA000CD42CCF6CC42A2FB00274FEA9705219E3B
:10DEB000716AB5FBF1F01D9B40F67467C2F2000772
:10DEC000FA185578FE5C4FEA064141EA0527937837
:10DED00047EA03021B92801A20F07F451C950DF142
:10DEE000700C1E9885422CBF00200120F9F7DAFB48
:10DEF000FBF781BE219E96F846700DF1700CF9F784
:10DF0000E9FB3A1A1C92219B83F84720FF2A94BF11
:10DF10000022012283F85020FBF76DBE1D98F928DE
:10DF200007D942F6C460C2F200004FF0130202713A
:10DF3000FBE242F61C71C2F200010B6840F674620B
:10DF4000C2F200021352FFF705B9219B93F8475024
:10DF50001C9593F8466083F8476083F84650FBF7BA
:10DF60004ABE1D98072807D942F6C464C2F20004CD
:10DF70004FF008012171D8E2F9F7F8FF0DF1A80C74
:10DF80004CF8380D003018BF0120F9F78BFBFBF778
:10DF900032BE219F97F8470097F846200DF1700C8C
:10DFA000904214BF00200120F9F77CFBFBF723BE51
:10DFB000219B93F8470093F846500DF1700C401BDD
:10DFC00018BF0120F9F76EFBFBF715BE219E96F8EE
:10DFD000470096F846100DF1700C88422CBF0020C7
:10DFE0000120F9F75FFBFBF706BE219F97F847007A
:10DFF00097F846200DF1700C904294BF002001204C
:10E00000F9F750FBFBF7F7BD219B93F8470093F816
:10E0100046500DF1700CA8428CBF00200120F9F78A
:10E0200041FBFBF7E8BD219E96F8470096F84610A5
:10E030000DF1700C884234BF00200120F9F732FB4B
:10E04000FBF7D9BD1D98102807D942F6C464C2F267
:10E0500000044FF01203237167E242F6FC67C2F23C
:10E0600000073858F9F798F9219AD064FBF7C3BD37
:10E070001D99102907D942F6C460C2F200004FF082
:10E080001202027151E242F6FC65C2F200056858C4
:10E09000F9F782F9219EB064FBF7ADBD42F6FC634F
:10E0A000C2F200035A7D1D9BD118152907D942F6EB
:10E0B000C463C2F200034FF01201197135E21E99D8
:10E0C000C2F1FB00814207DD42F6C464C2F20004E3
:10E0D0004FF01302227128E240F67467C2F2000783
:10E0E000781842F6FC65C2F20005E91806F074F8EB
:10E0F000FBF781BD42F6C460C2F200004FF001049C
:10E10000047112E20DF1700CF9F70CFB40F6746625
:10E11000C2F200061E9FF55D1D9A15423BF46BADE1
:10E1200042F61C73C2F20003089919607BE10DF1FD
:10E13000700CF9F7F7FA40F67460C2F200001E9E08
:10E14000875D1D9D2F427BF456AD42F61C73C2F2D3
:10E150000003089A1A6066E19DF874000DF16B01E6
:10E16000FAF734FD8DF86A009DF86B1029B142F67C
:10E17000C464C2F200042171D7E100283BF43BAD36
:10E1800042F61C70C2F20000089E06604BE19DF84A
:10E1900074000DF16B01FAF719FDD0F1010338BFDE
:10E1A00000238DF86A309DF86B302BB142F6C464C1
:10E1B000C2F200042371B8E1219FFD6A15B98DF800
:10E1C0006A5002E09DF86A0060B90DF1700C1E986B
:10E1D000F9F720FF30B942F61C73C2F20003089A27
:10E1E0001A6020E10DF1700C9DF86A00F9F75AFAF7
:10E1F0004FF000062199CE62FBF7FDBC9DF874003C
:10E200000DF16B01FAF7E2FC8DF86A009DF86B10D6
:10E2100029B142F6C462C2F20002117185E1002800
:10E220007BF4E9AC42F61C77C2F20007089D3D6022
:10E23000F9E09DF874000DF16B01FAF7F7FC8DF829
:10E240006A009DF86B302BB142F6C464C2F2000440
:10E2500023716AE100287BF4CEAC42F61C70C2F256
:10E260000000089E0660DEE09DF874000DF16B0171
:10E27000FAF7DCFC011C18BF01218DF86A1092E747
:10E280009DF874000DF16B01FAF7A0FC021C18BF99
:10E2900001228DF86A2086E71D9E102E07D942F6CE
:10E2A000C463C2F200034FF012021A713DE12198DB
:10E2B000C06CF9F747F842F6FC61C2F200018851E0
:10E2C000FBF799BC0DF1700CF9F704FA219E96F852
:10E2D0004770D7F1010538BF0025002814BF284634
:10E2E00085F0010086F84700FBF785BC0DF1700C46
:10E2F000F9F7F0F9219991F84730584081F8470033
:10E30000FBF779BC0DF1700CF9F7E4F9219A82F86A
:10E310005100FBF770BC04F0F1FC0DF1A80C4CF8B7
:10E32000380DFF2828BFFF20C0B2F9F7BBF9FBF773
:10E3300062BC04F0D9FC0DF1A80C4CF8380DFF2894
:10E3400028BFFF20C0B2F9F7ADF9FBF754BC04F0C9
:10E35000DFFC0DF1A80C4CF8380DFF2828BFFF207A
:10E36000C0B2F9F79FF9FBF746BC04F0B3FC0DF11E
:10E37000700C00280CBFFF200020F9F793F9FBF781
:10E380003ABC42F61470C2F2000001681D9BC81826
:10E3900004F006F88DF86B0000283BF42CAC42F634
:10E3A000C464C2F200042071BFE01D9803F0B6FF00
:10E3B000FBF721BC0DF1700CF9F78CF903F0A8FF05
:10E3C000FBF719BC42F61476C2F2000637681D9DB1
:10E3D000781903F0BFFFFBF70EBC03F0A3FFFBF7B8
:10E3E0000ABC40F6B472C2F20002107810F0010FBD
:10E3F00007D042F6C461C2F200014FF0320008714A
:10E4000093E042F65861C2F200010B68B3B900F024
:10E410000204E2B292B142F6C464C2F200044FF0C8
:10E420003503237181E040F6B477C2F200073D78EE
:10E4300015F0010F18BF00247BF4DDAB219E2EB137
:10E4400042F61C77C2F200073D68756042F6AC6088
:10E45000C2F2000001683F2900F2948001F101013D
:10E460001B911C9111B94FF001041B9441F6CC068D
:10E47000C2F200064FF0540540F6B474C2F2000434
:10E4800042F65867C2F200071C9B05FB036221920B
:10E490009BB9217801F00400C1B209B9386840B9CC
:10E4A000217841F001006FF382002070506840B184
:10E4B00015E04FF001021C92E6E7506878B9402B56
:10E4C00002D003F1010301E04FF000031C931B9AFB
:10E4D0009342D9D14FF00000FAF7DCF8D4E742F6C6
:10E4E000AC66C2F20006336042F61C75C2F200054B
:10E4F00028604FF0000B5C46FBF77DBB219F3E6A16
:10E5000046F000453D63FBF776BB4FF00002219BD0
:10E510001A63FBF770BBFBF76EBB0B9D42F6C4643E
:10E52000C2F200044FF00101217142F6C463C2F24D
:10E530000003089C1C605D71F3F70AF8F3F708F814
:10E54000219D296A79B14FF000001C90219A136A2D
:10E550004BB1F2F7FDFF1C9C04F101041C94219DBA
:10E56000296AA142F5D84FF00000FAF793F8FBF7BB
:10E5700078BA4FF0000700F1FF344FF00003564621
:10E58000FDF7EFBD4FF000031C936CE74FF0020363
:10E590001C9341F6CC02C2F20002FEF727B82BB062
:10E5A000BDEC0A8BBDE8F08F05F10103D2F80061E4
:10E5B000002E3EF41FA805F1020302F1A802412B30
:10E5C0007EF414A8FEF76BB8B8F1000F3DF463AD0C
:10E5D00010F803C001F803C003F1010393427DF476
:10E5E0005AADFDF766BDE918F71813F801CF02F12F
:10E5F000FF3E60453DF435AB7246FDF73FBB0EF183
:10E60000FF32FDF73BBB00BF38B5054642F69C64C0
:10E61000C2F200042068F6F795FF4FF00003236074
:10E620008DB148F20830C0F601004FF0070149F6FD
:10E63000F512C0F60002F6F79BFE42F6A862C2F29F
:10E640000002106038BD42F6A864C2F200042068DF
:10E65000F6F778FF4FF000002060FBF74DF903F06C
:10E66000CDFE42F6BC61C2F200010878FF2803D05B
:10E670004FF00401FBF7BAF838BD00BF70B542F6A1
:10E68000D460C2F2000048F21831C0F60101F6F77A
:10E690009FFA42F6BC63C2F200034FF0FF021A7009
:10E6A00040F6B874C2F200044FF0040684F8206209
:10E6B0004FF00005C4F81C522846F6F773FC2060A2
:10E6C00084F86464C4F860544FF00100F6F76AFC03
:10E6D000C4F8440284F8A866C4F8A4564FF00200B7
:10E6E000F6F760FCC4F8880484F8EC68C4F8E858CD
:10E6F0004FF00300F6F756FCC4F8CC0642F6206053
:10E70000C2F2000048F22431C0F60101F6F760FAC7
:10E7100040F2CC10C2F200002946FAF74DFAF9F7A0
:10E7200015F94FF00100FFF76FFF70BD000000000A
:10E730002DE9F04F2DED028B8FB04FF0000842F61F
:10E74000A867C2F2000742F69C63C2F2000303937B
:10E7500042F6BC6BC2F2000B40F6B876C2F200067D
:10E760009FEDBD8B39684FF0FF3041B9F2F7F0FEF5
:10E77000386800280CBFFA204FF0FF30FFE7F6F7AB
:10E7800035FE28B1B8F1320F09D808F1010806E0CA
:10E79000B8F1330F0CBF4FF034084FF000083A685F
:10E7A000C2B9F2F7D5FEB8F1320F0CD1039C206844
:10E7B000F6F7C8FE4FF00005039B1D604FF0020006
:10E7C000F9F7A6FE06E0B8F1340F03D14FF00100CF
:10E7D000F9F79EFE9BF800104FF4117000FB0162E8
:10E7E000D2F81842002CBDD04FF4117505FB01F38F
:10E7F00003F5887406EB0409315DE0290CD199F822
:10E8000001000E2808D14FF6FF704946D9F80021C3
:10E81000F8F732FD10B355E2325D02F01F0509EB47
:10E8200005035A78294605F0010019F80550521BD6
:10E8300001F1FF33002940F062820BE019F8030078
:10E84000151A03F1FF3119F80120AA1A01F1FF335B
:10E850000029F3D112F0FF0F40F03482335D4FEA0C
:10E860005310072800F22682DFE810F00800240287
:10E8700024023500A400240288001A01335D09F146
:10E88000010513F01F0000F01D8209F1020905F1D6
:10E89000020500F1FF3255FA82F402944FF00005B0
:10E8A0004FF0010A15E019F8011CE8B22140524668
:10E8B000FAF790FA002840F0058205F101054FEAC9
:10E8C0004404FF2CEFD909F101090299894500F0B0
:10E8D000F9815446E7E799F80140386860B1F6F7E6
:10E8E00031FE4FF000003860FBF706F84FF00100F2
:10E8F000F9F70EFEF2F72CFE03990B686BB948F29C
:10E900002C30C0F601004FF0070149F29912C0F611
:10E910000002F6F72DFD039D286005A84FF00001C9
:10E92000FAF724F87CB9F7F7DBF9C1B201F1FF334C
:10E93000DDB2FD2D41F6C800C2F2000092BF0170A9
:10E940000122027009E041F6C800C2F2000002781C
:10E9500002FB04F404EB1424047041F6C804C2F270
:10E96000000421780EAB03F8241D4FF003004FF094
:10E9700000014FF01602F9F7EFFDF3E60DF1130079
:10E98000F9F7E6F901469DF813508DF81450012D62
:10E9900006D828B10DF115004FF00D0205F01CFC52
:10E9A0004FF006004FF000014FF00E0205ABF9F7F3
:10E9B000D3FDD7E69BF800304FF4117101FB03F44F
:10E9C00099F80100032868D8DFE800F00222344AF1
:10E9D0004FF00100FFF718FE4FF000050EAB03F8F3
:10E9E000255D4FF0040029464FF00102F9F7B4FD10
:10E9F00032599BF800004FF0010400940195D2F8C1
:10EA00000CC04FF416512A464FF00803E04756E178
:10EA10004FF0000142F6C463C2F2000319714FF0D7
:10EA200001040EAB03F8254D4FF004002246F9F720
:10EA300093FD44E1F9F742FE0EAB4FF0020103F8FB
:10EA4000251D4FF004004FF000014FF00102F9F7CF
:10EA500083FD4FF0010432E10000000000E06F4050
:10EA60000EAB4FF0120203F8252D4FF004004FF0CB
:10EA700000014FF00102F9F76FFD35599BF80000D6
:10EA80004FF0010400944FF000020192ED684FF442
:10EA900016414FF00803A84711E14FF000040EE1C2
:10EAA00099F80150A5F102050C2D00F20681DFE86E
:10EAB00015F00D0067007E0004010401040104014B
:10EAC000040104010401040104019D00315DC1F34E
:10EAD0000400C5B2012D00F0F58009F1050509F12A
:10EAE000080400EBC00200EB420303EBC30101F199
:10EAF0005401C8B200EB4002A418C5EB040CACF101
:10EB0000030E0EF0010A99F8029015F8010C04F0BA
:10EB100009F953EC182B04F017FC04F0DDF9014659
:10EB20004846FAF7BDF905F10305A54240F0CD804E
:10EB3000C8E015F8039C15F8010C04F0F3F853EC49
:10EB4000182B04F001FC04F0C7F901464846FAF717
:10EB5000A7F905F1030515F803AC15F8010C04F04D
:10EB6000E1F853EC182B04F0EFFB04F0B5F9014683
:10EB70005046FAF795F905F10305A542D9D1A1E070
:10EB800099F80250305DC0F30402A2F10302D2B240
:10EB900009F10301AC18FF2CC4BF6A42D2B240F69F
:10EBA0007463C2F20003581905F016FB8AE099F865
:10EBB000022099F803500EAC04F8242D0DF1150035
:10EBC00040F67461C2F200018918202D34BF2A4634
:10EBD000202205F001FB05F101034FF007004FF083
:10EBE0000301DAB22346F9F7B7FCBBE599F8024016
:10EBF00074B999F8031059B903F000FC48F23C309D
:10EC0000C0F6010007F0D8F8F9F738FE002848D020
:10EC100099F8022099F8033048F24C30C0F6010010
:10EC200043EA022107F0C8F899F803A0494611F811
:10EC3000020F4AF20005C0F6010505EB002540F67B
:10EC40007464C2F2000404EB0A0001F102014FF007
:10EC5000800205F0C1FA4FF68071CFF6FF71CAEB62
:10EC60000102D3B2E018E9184FF0800205F0B4FABF
:10EC7000204629464FF48072F3F762FDA0B9204682
:10EC800029464FF4807204F051FE80B94FF0010024
:10EC90004FF000010A460B46F9F75EFC4FF0010405
:10ECA0000DE04FF000040AE04FF0000407E04FF0E1
:10ECB000000404E04FF0000401E04FF00004002CD9
:10ECC0007FF450ADF9F726F84CE5BAF1000F3FF4A8
:10ECD00030AF15F803AC15F8010C04F023F853EC31
:10ECE000182B04F031FB04F0F7F801465046FAF710
:10ECF000D7F805F10305A5427FF41BAFE2E7002832
:10ED00003FF49CAD19F80310521A03F1FF33B3F12D
:10ED1000FF3F7FF493AD9DE5704700BF42F6497316
:10ED2000C2F200031A78027042F64870C2F2000084
:10ED300003780B70704700BF42F64973C2F20003BC
:10ED40001B78834225D842F64872C2F2000212783C
:10ED50009A18904220DAC01A4FEA50034FF001028D
:10ED600002FA03F310F0010F09D042F65470C2F218
:10ED70000000026813400B704FF00100704742F62C
:10ED80004C70C2F20000026813400B704FF001009B
:10ED900070474FF0000070474FF00000704700BF11
:10EDA00010B542F64973C2F200031B7883427AD849
:10EDB00042F64872C2F2000212789A18904275DA4E
:10EDC000C31A03F0FE0442F65870C2F20000027843
:10EDD000A418E4B24FEA53024FF0010000FA02F225
:10EDE00013F0010F12D041B142F65470C2F200008C
:10EDF000016842EA010303601AE042F65470C2F26D
:10EE00000000036823EA0203036011E041B142F607
:10EE10004C70C2F20000036842EA0301016007E09F
:10EE200042F64C73C2F20003196821EA020119602C
:10EE300042F64C70C2F2000001680A4224D042F649
:10EE40005473C2F20003186802420ED020464FF0FD
:10EE50000001F2F79FF904F10102D0B24FF0010175
:10EE6000F2F798F94FF0010010BD20464FF0010174
:10EE7000F2F790F904F10101C8B24FF00001F2F786
:10EE800089F94FF0010010BD20464FF00001F2F764
:10EE900081F904F10102D0B24FF00001F2F77AF9E2
:10EEA0004FF0010010BD4FF0000010BD4FF000000A
:10EEB00010BD00BF08B542F65873C2F200031870C7
:10EEC00042F65073C2F20003197042F64973C2F25F
:10EED00000031A70091A01F10101C8B242F6487222
:10EEE000C2F200021070412801D9F1F7B1FB40F2E3
:10EEF000D810C2F200004FF00101F9F7D9FD08BDAA
:10EF00002DE9F84342F65973C2F2000318784FEA2C
:10EF1000400111F0FF0405D042F65972C2F200021E
:10EF2000147006E042F65975C2F200054FF0010672
:10EF30002E7042F67C77C2F20007387842F6597399
:10EF4000C2F20003197808420CBF4FF000094FF0DD
:10EF500001094FF000052C464FF0010742F65C76A0
:10EF6000C2F20006A84604F01F0207FA02F0AB59ED
:10EF7000184204D0204649464246F9F72BFF04F1D7
:10EF80000104E4B214F01F0FEDD105F10405202DAA
:10EF9000E9D1BDE8F88300BF42F67C73C2F20003FA
:10EFA000187042F65970C2F200004FF00102027070
:10EFB000704700BF00B583B042F65C70C2F200003B
:10EFC0004FF000014FF00802F1F7A4FB4FF00003EF
:10EFD00000934FF00100019042F68070C2F20000F1
:10EFE0004FF47A714FF006024EF60173C0F600033B
:10EFF000F6F740FE03B000BD08B542F68070C2F2DD
:10F000000000F6F791FD4FF0CC00FFF7C5FF08BDFB
:10F0100089B14FEA501242F65C73C2F2000300F06D
:10F020001F004FF0010101FA00F053F822100843CD
:10F0300043F8220011E04FEA501242F65C73C2F22C
:10F04000000300F01F004FF0010101FA00F053F837
:10F05000221021EA000143F822104FF0000070470F
:10F0600008B54FF4404048F27C41C0F6010142F639
:10F07000A472C2F20002F9F7D9FC08BD70B51546BA
:10F0800081B9537D8BB14FF000042646285D31468F
:10F09000F5F7BEFA04F10104687DA042F6D84FF0FE
:10F0A000000070BD4FF0140070BD4FF0000070BD47
:10F0B00008B54FF00C004FF00001F5F7A9FA08BDB4
:10F0C00010B586B0F1B942F6B073C2F200031978F8
:10F0D00042F6B170C2F20000037802AC00944FF027
:10F0E0001000019010461A464FF00103FAF7DCF9C0
:10F0F00048F27840C0F60100214606F05DFE4FF070
:10F10000000001E04FF0140006B010BD08B5012961
:10F1100008D148F26020C0F6010006F04DFE4FF025
:10F12000000008BD4FF0140008BD00BF08B511B1C4
:10F13000012916D106E050781178F5F721FB4FF040
:10F14000000008BD117842F6B070C2F200000170F4
:10F15000527842F6B173C2F200031A704FF0000009
:10F1600008BD4FF0140008BD08B505292AD8DFE80E
:10F1700001F0030B1529291F1046F5F7D7FA0028CF
:10F180000CBF1620002008BD48F20430C0F6010074
:10F19000114606F011FE4FF0000008BD48F2FC20B9
:10F1A000C0F60100114606F007FE4FF0000008BD52
:10F1B00048F2E820C0F60100114606F0FDFD4FF0D0
:10F1C000000008BD4FF0140008BD00BF037B13B959
:10F1D000437B13B90EE0994208D301F1FF318A183D
:10F1E000437B9A428CBF0020012001E04FF00000D9
:10F1F000C0B270474FF00100704700BF70B4447A4E
:10F2000024B14FF0320606FB04F610E0C57847F64D
:10F21000B814C0F6010454F82550B5F5964F9DBFBB
:10F2200049F26466B6FBF5F606EB86060826847A94
:10F2300024B14FF0320505FB04F501E041F28835B9
:10F24000C07A18B1FF2808BF012001E04FF001008B
:10F2500001B10E6002B1156003B1186070BC704757
:10F2600040F6B873C2F200034FF4117202FB003093
:10F270004FF00001C0F810124FF6FF73C0F82C32A7
:10F28000C0F81812704700BFF8B505460E4640F6A4
:10F29000B874C2F200044FF4117303FB0044D4F8B5
:10F2A000240200EB5007F6F71BFDD4F82812421A8F
:10F2B000974202D9B81AF6F799F823689A6928464E
:10F2C0004FF00101904740F6B870C2F200004FF4D1
:10F2D000117101FB05014FF6FF7001F10401324687
:10F2E000F7F7CAFFA31918714FEA10225A7106F1F5
:10F2F0000206C4F804614FF00000C4F80801216858
:10F300000B6A28469847F5F7A9FE2846FFF7A8FF9D
:10F31000F8BD00BF38B504460D460368F92B08D880
:10F3200040F67460C2F20000185A03F10203236031
:10F330003DE0A3F57A72FA2A0AD840F67461C2F267
:10F3400000018A5C4FEA022003F1010323602EE0F2
:10F35000A3F5FA60262811D84FF0000001460246B6
:10F36000F5F71EFA2368A3F5FA6281184978805CE4
:10F3700040EA012003F10203236018E0A3F6B8314C
:10F380007C290DD803F10042A2F6B83040F6746132
:10F39000C2F2000131F8100003F10103236006E01E
:10F3A00055B14FF001032B704FF0000038BD2DB167
:10F3B0004FF000032B7038BD4FF0000038BD00BF88
:10F3C00030B583B004460D4602A840F8084D6846A3
:10F3D0000DF10701FFF79EFF9DF8073083B904F197
:10F3E000FF34651902A941F8085D68460DF107016F
:10F3F000FFF790FF9DF80720101C18BF012001E0C7
:10F400004FF0010003B030BD2DE9F0410D46174625
:10F410001E4640F6B871C2F200014FF4117404FBAD
:10F420000010D0F83002037BFF2B02D1427BFF2A71
:10F4300056D02C68F92C15D821464FF00202FFF760
:10F44000C5FE002850D0002E52D140F67460C2F2A2
:10F45000000027522B6803F102032B604FF00100DC
:10F46000BDE8F081A4F57A78B8F1FA0F18D84146D2
:10F470004FF00102FFF7AAFE00283DD0002E3FD139
:10F480004FEA172740F67462C2F2000202F80870D1
:10F49000296801F1010129604FF00100BDE8F08108
:10F4A000A4F6B8317C292FD804F10044A4F6B8346E
:10F4B0004FEA44014FF00202FFF788FE002827D0F0
:10F4C000002E29D140F67460C2F2000020F81470BA
:10F4D0002B6803F101032B604FF00100BDE8F081C0
:10F4E0004FF00000BDE8F0814FF00000BDE8F08172
:10F4F0004FF00100BDE8F0814FF00000BDE8F08161
:10F500004FF00100BDE8F0814FF00000BDE8F08150
:10F510004FF00000BDE8F0814FF00100BDE8F08140
:10F5200030B583B040F6B874C2F200044FF41175E0
:10F5300005FB0040D0F83002B1F57A7F1BD3A1F56E
:10F540007A7163B1837B13B9C37B13B907E0994226
:10F5500023D38A1802F1FF32C07B824220D8C8B27E
:10F560000DF10701F9F7CAFB9DF80710D1F1010071
:10F5700038BF002019E04FEAD10402F107024FEA38
:10F58000D20523B121462A46FFF720FE58B128199B
:10F59000FA288CBF0020012007E04FF0000004E0B3
:10F5A0004FF0000001E04FF0000003B030BD00BF9D
:10F5B00008B5B0F57A7F21D279B14FEAD00340F691
:10F5C0007462C2F2000200F007004FF0010101FA7C
:10F5D00000F0D15C0843D05408BD4FEAD00340F698
:10F5E0007462C2F2000200F007004FF0010101FA5C
:10F5F00000F0D15C21EA0000D05408BD00F11800F1
:10F60000C0B24FF00102F9F7E5FB08BD10B540F6B6
:10F61000B874C2F200044FF4117303FB0044D4F831
:10F620001C02F5F78FFF4FF00000C4F81C0210BD5C
:10F6300038B54FF4117101FB00F140F6B872C2F217
:10F6400000028C18D4F80831D4F80451AB420BD026
:10F650008958E3188A6A1979904728B1D4F80801C3
:10F6600000F10100C4F8080138BD00BF08B540F63C
:10F67000B873C2F200034FF4117202FB0031D1F8EB
:10F68000082101F10401D1F800319A420BD140F672
:10F69000B871C2F200014FF4117202FB0010D0F8F1
:10F6A0001C02F5F70DFD08BD70B582B005468DF85A
:10F6B000071040F6B874C2F200044FF4117303FB54
:10F6C0000044D4F81802002850D11AB12846FFF798
:10F6D000C7FD4BE0F6F704FBD4F82812431AC4F830
:10F6E0002802D4F81002D4F82422934204D800F15E
:10F6F0000103B3F5807F04D12846FFF7B1FD4FF039
:10F700000103D4F81012621802A911F8010D82F851
:10F710001001C4F81032B4F82C024FF00102F7F7D0
:10F72000ABFDC4F82C0208BB04F5887694F82032AF
:10F73000012B03D1304601F0F3FA38B994F82012C6
:10F74000022913D1304600F013F978B14FF00102CD
:10F75000C4F8182240F6B870C2F200004FF41173DA
:10F7600003FB0505D5F81C02F5F7AAFC02B070BD35
:10F7700010B542F6B373C2F200031B78032B47D8CF
:10F7800040F6B872C2F200024FF4117101FB03237C
:10F7900040F62C02C2F2000252E8001F01F1010102
:10F7A00042E80014012CF7D018B14FF00100C3F863
:10F7B0003C0242F6B274C2F200044FF00101217023
:10F7C000D3F840221AB1D3F81C02F5F779FC40F6C1
:10F7D0002C03C2F2000353E8002FA2F1010243E818
:10F7E0000024012CF7D053E8002FB2F1004F0DD1C7
:10F7F0004FF0000243E80024012CF4D04EF60450F0
:10F80000CEF20000016841F080510160BFF32F8FFC
:10F8100010BD00BF10B542F6B373C2F200034FF043
:10F8200004041C70FFF7F2FE10BD00BF2DE9F04F7D
:10F8300089B005460E4691F8029009EB490947F256
:10F840006C28C0F6010809EB08074FF4117B0BFB8D
:10F8500000FB40F6B87AC2F2000A0BEB0A044FF044
:10F860000201F9F7C3FF42F6B373C2F200031D7041
:10F87000C4F83062304604F5097104F50D7204F5E0
:10F880000E73FFF7BBFC2846FFF7EAFCF6F728FAF1
:10F89000C4F828024FF00100009048F2A440C0F6DE
:10F8A00001004FF004014FF69932C0F600022B46DA
:10F8B000F5F752FDC4F81C025BF80A40F27847F6EF
:10F8C000B811C0F6010151F8221019F808207B7810
:10F8D000BE7800964FF0000001904FF23166C0F6FE
:10F8E000000602964FF26D66C0F6000603964FF2D0
:10F8F000A966C0F6000604964FF61506C0F6000687
:10F900000596069064682846A04709B0BDE8F08FC8
:10F9100008B542F6B473C2F2000318604FF001005C
:10F92000FFF726FF08BD00BF42F6B273C2F2000324
:10F930004FF000021A70704708B542F6B473C2F275
:10F940000003186868B142F6B371C2F200010A7888
:10F95000032A09D84FF00000FFF70AFF4FF000001C
:10F9600008BD4FF0480008BD4FF0480008BD00BF7B
:10F9700010B4D0F80031032B20D94278102A20D8B7
:10F9800090F901404FF0010101FA04F448F26002DD
:10F9900061F31F4214420CD114F00E0F11D0052B4D
:10F9A00012D9807800F10500834214BF00200120A5
:10F9B0000CE0082B14BF0020012007E04FF00000EE
:10F9C00004E04FF0010001E04FF0000010BC704770
:10F9D000072814D840B24FF0010303FA00F111F0E8
:10F9E0000A0F0FD111F0050F03D111F0F00F03D161
:10F9F00005E04FF0010070474FF0040070474FF0F2
:10FA0000000070474FF00200704700BF2DE9F04F33
:10FA100083B005460E4617461C464FF000000146CF
:10FA20000246F4F7BDFE83463846FFF7D1FF804615
:10FA3000002800F0A980042805D04FF00100002E16
:10FA400000F0A78003E016F0010FF6D09FE0A7F1C9
:10FA5000040A40F67463C2F200030193BAF1030F83
:10FA600004D8019AA858F7F797FC8146072F00F2AF
:10FA70008280DFE807F0042416364C5E676FB5F528
:10FA8000FA6F08D90BEB0502A2F5FA6108784FEA84
:10FA9000002323806FE00199685C4FEA00232380F4
:10FAA00069E0B5F5FA6F06D90BEB0502A2F5FA612C
:10FAB0000B7823805FE0019BE85C20805BE0B5F57C
:10FAC000FA6F0AD9A5F5FA618B449BF801009BF8FF
:10FAD000003043EA002222804DE001982A5A228019
:10FAE00049E0B5F5FA6F0AD9A5F5FA639B449BF88E
:10FAF00000009BF8012042EA002121803BE0019BAD
:10FB0000E85A4FEA102242EA0021218033E04FEA0E
:10FB100019434FEA132040EA0321234623F8021B2E
:10FB20001FFA89F24FEA122040EA022161801C4646
:10FB300021E0C9F30F41224622F8021BA4F80290EB
:10FB4000144618E0234623F8029BC9F30F40608057
:10FB50001C4610E01FFA89F04FEA102141EA00220A
:10FB6000234623F8022B4FEA19404FEA102141EABD
:10FB7000002262801C46454404F10204013E7FF4E9
:10FB80006DAF4FF0010004E04FF0000001E04FF0D6
:10FB9000000003B0BDE8F08F2DE9F04F8BB05FFAA5
:10FBA00080FB40F6B873C2F200034FF4117404FBFB
:10FBB0000B344FF000054FF4117000FB0BF1019175
:10FBC00001F5887640F6B872C2F200020392B718C7
:10FBD00004970BE02668B36958464FF00001984738
:10FBE0004FF00100C4F84002F5F738FA42F6B2735C
:10FBF000C2F2000318780028ECD042F6B471C2F2C9
:10FC000000010E68002EE5D04FF00002C4F840223B
:10FC1000DDF80CA0DDF8109060E3D4F83C0240B1B0
:10FC20004FF00005C4F83C5242F6B471C2F2000134
:10FC30000D682E78062E00F0A4800CD8032E1CD060
:10FC400003D8002E00F0AB811AE0042E42D0052E1E
:10FC500040F0A58167E0802E00F07F8106D80F2E4E
:10FC600000F0C080102E40F09A812DE1812E00F02E
:10FC70008D81822E40F093817EE14FF008062BE0CB
:10FC80002A79B5F8057002F1FF33B3F5FA6F19D28E
:10FC90004FEA172040EA072113FA81F6B6F5FB6F09
:10FCA00013D2019F07EB0A0101F104036878087180
:10FCB0002E785E706F885F804FEA02229A804FF044
:10FCC000060104E04FF0FF3101E04FF0FF314FF04B
:10FCD00007065FE14FF007062F79B5F8051007F129
:10FCE000FF327C2A19D84FEA112040EA012312FA88
:10FCF00083F1FA2914D8DDF8048008EB0A0202F136
:10FD0000040368781071297859706A885A804FEA1C
:10FD100007279F804FF006013CE14FF0FF3139E1AA
:10FD20004FF0FF3136E1A9884FEA112343EA012061
:10FD300087B24FEAD702FA2A1ED8019E06EB0A03C1
:10FD400003F10401687818712E784E706B884B802F
:10FD500007F007074FF0010000FA07F040F674665D
:10FD6000C2F20006B25C0240002A14BFFF23002347
:10FD70008B804FF0060101E04FF0FF314FF0060697
:10FD800008E1A879FFF724FEAB88024610B34FEADA
:10FD9000132141EA032080B200F1FF37BE18FA2E8A
:10FDA0001BD8DDF804C00CEB0A0202F104036978E9
:10FDB00011712F785F706E885E804FF00101AA7913
:10FDC00003F10403FFF722FE002814BF06214FF0C1
:10FDD000FF3104E04FF0FF3101E04FF0FF314FF011
:10FDE0000706D7E02A791646B5F8053002F1FF304C
:10FDF000B0F5F66F60D24FEA132141EA0327B9B29A
:10FE00004FEAD1031818FA2859D8019F07EB0A08BE
:10FE100008F1040C687888F804002F788CF80170D9
:10FE20006888ACF802004FEA0227ACF8047002F1CF
:10FE300007004FEAD0078CF8067008F10B00002A83
:10FE400035D001F007014FF0010202FA01F70797E0
:10FE500040F67467C2F20007964606F1FF31114082
:10FE600005910292002A00F0C182BBE2A846029EE0
:10FE700001E0A846029E012A04BF00250570FD5C32
:10FE80000D4202D00578154305704FEA41018029E3
:10FE900084BF013371464FEA4202802A84BF013099
:10FEA000724606F1FF35012A40F0E082DBE29CF861
:10FEB000061001F1070104E04FF0FF3101E04FF0BF
:10FEC000FF314FF0070665E0E879FFF781FD2979FA
:10FED000B5F8056001F1FF337A2B2DD878B34FEADE
:10FEE000162242EA0627BAB202F1FF3601FB00638E
:10FEF000FA2B05D9A2F5FA67262F23D8022824D891
:10FF0000019800EB0A0303F104066F781F7128784B
:10FF100058716F88DF804FEA012018814FEA41074E
:10FF20009F721046EA7903F10B03FFF76FFD78B17A
:10FF3000B17901F107010DE04FF0FF310AE04FF018
:10FF4000FF3107E04FF0FF3104E04FF0FF3101E0F7
:10FF50004FF0FF314FF008061CE0B5F801104FEAF2
:10FF6000112242EA012042F61473C2F200031F6814
:10FF700017FA80F6771BBAE16B784FF0320000FB7E
:10FF800003F0F5F733FA4FF00207B0E16FF001012B
:10FF90004FF00106AE19B1F1FF3F0ED100E02E4641
:10FFA0004FF0000342F6B472C2F20002136042F650
:10FFB000B277C2F200073B708FE1002940F38381E2
:10FFC0005846FFF761F92068826958464FF00001F2
:10FFD000904794F83872002F00F07F8107F1FF3EC0
:10FFE0000EF00108D4F83402F5F700FA002840F0CA
:10FFF000DA8106E0D4F83402F5F7F8F9002840F089
:020000040801F1
:10000000568199F800006B78984240F0668199F823
:10001000012029788A4240F0608142F62060C2F2D5
:1000200000004FF00001F4F7EBFD2F7807F1FF30EF
:10003000032800F23581DFE800F00202595995F8F3
:1000400004E099F802700EF10702B7EBD20F40F00E
:100050002781B5F805504FEA152040EA05239FB2E5
:1000600007F007024FF0010101FA02F14FEAD7034E
:10007000BEF1000F00F014814FF0010040F67462F1
:10008000C2F2000207460EF1FF3C0CEA000C4FF0F2
:10009000000599F8038018EA000F00F02A812FE18B
:1000A00009EB050898F803C01CEA000F12F803805A
:1000B00014BF41EA080828EA010802F803804FEA61
:1000C0004000802884BF013538464FEA410180292D
:1000D00084BF013339460EF1FF3E09EB050C9CF855
:1000E000038018EA000F00F0408145E199F80220F2
:1000F0002B79B2EB430F40F0D380E979072900F266
:10010000CF8095F907704FF0010000FA07F313F064
:100110000A0F16D113F0050F03D113F0F00F09D118
:10012000BEE04FF0020ECDF808E04FF00108CDF828
:1001300014800CE04FF0040CCDF808C0CDF814C0CA
:1001400005E04FF0020CCDF808C0CDF814C0B5F8AA
:1001500005004FEA102343EA00211FFA81F8002A24
:1001600000F09E804FF0000740F67462C2F2000279
:100170000792CDF820B00994DDF818B01446E8795C
:1001800007287AD8DFE800F004140D1D28445362D4
:1001900009EB4700B0F803204FEA122308F80430B7
:1001A0006BE009EB4703B3F8031008F8041064E0B0
:1001B00009EB4700C278037942EA032128F80410CA
:1001C0005BE009EB4703B3F803104FEA112242EA60
:1001D000012028F8040050E009EB4703B3F80310AE
:1001E00007F101074FEA112242EA012060F31F4B99
:1001F00009EB4703B3F803104FEA112242EA01204A
:1002000060F30F0B5846F7F79DF848F8040034E008
:1002100009EB4703B3F8031061F31F4B07F1010724
:1002200009EB4702B2F8030060F30F0BEAE709EBB2
:100230004703B3F8031061F30F0B07F1010709EB54
:100240004702B2F8030060F31F4BDBE709EB4703FB
:10025000B3F8031007F101074FEA112242EA012027
:1002600060F30F0B09EB4703B3F803104FEA1122B9
:1002700042EA012060F31F4BC4E70599884407F167
:10028000010799F802200298131AD9B289F80210CE
:1002900000297FF474AF099CCDF818B0DDF820B0C8
:1002A00042F62060C2F20000F4F7B8FD15E007F155
:1002B000FF3202F0FF07D4F83402F5F797F8002870
:1002C00040F089809DE611F1020F06D142F6B27529
:1002D000C2F200054FF000032B70354642F6B277AC
:1002E000C2F200073B78002B7FF497AC7EE4EE1956
:1002F000F3E712F8038028EA010802F8038005E01A
:1003000012F8038041EA080802F803804FEA40002F
:100310004FEA4101802984BF01333946BEF1010E05
:10032000BED0BCF1000F3FF4BBAE09EB050C9CF84E
:10033000038018EA000F12F803C00CBF2CEA010C6E
:1003400041EA0C0C02F803C04FEA4000802884BF49
:10035000013538464FEA4101802984BF01333946CF
:10036000BEF1010E7FF49CAE9AE712F803C02CEAAE
:10037000010802F8038005E012F803C041EA0C0806
:1003800002F803804FEA4000802884BF01353846D8
:100390004FEA4101802984BF01333946BEF1010E85
:1003A0007FF47EAE7CE707F1FF3111F0FF0794D0B8
:1003B0004FFA88F3002B3FF41DAED4F83402F5F762
:1003C00015F800283FF41DAE07F1FF3010F0FF07CD
:1003D0007FF410AE81E707F1FF3111F0FF077FF4E2
:1003E00009AE7AE74FF0000288F80B20FA5C079913
:1003F0000A4205D098F80B2002990A4388F80B208E
:1004000007994FEA4101802984BF01337146DDF825
:1004100008804FEA4802013E02963FF448AD059E2F
:10042000002E3FF423AD012A04BF0026067017F802
:10043000038018EA010F04D0067842EA060880F823
:1004400000804FEA4101802984BF013371464FEAA1
:100450004202802A84BF01307246029E013E02960B
:100460007FF407AD23E54FF000060670FE5C0E42F8
:1004700002D00678164306704FEA4101802984BFF6
:10048000013371464FEA4202802A84BF013072462E
:100490006E1E7FF4F0AC454609E500BF38B540F666
:1004A000B875C2F200054FF4117404FB005505F154
:1004B0000404297162F07F026A71AB714FF003018D
:1004C000FEF7E2FE38BD00BF2DE9F04F89B05FFABC
:1004D00080FA40F6B873C2F200034FF4117404FBC3
:1004E0000A344FF4117000FB0AF1029101F588758E
:1004F00040F6B872C2F20002039205EB020B2668C6
:10050000B76950464FF00001B847F4F7A7FDD4F89B
:100510001002D4F814329842F1D094F81011D4F8A3
:100520003452A94240F00A8342F62060C2F2000031
:100530004FF00001F4F764FB94F8112102F1FF364B
:100540000F2E00F2EE82DFE816F010009E000F0181
:10055000EC027801C801EC02EC02EC02EC02EC02C5
:10056000EC02EC02EC02FB016B02BBF80260BBF890
:1005700004504FEA152343EA052087B207F1FF3202
:10058000B2F5FA6F09D350469BF800109BF8012092
:100590004FF00303FFF782FFCAE24FEA162141EA58
:1005A0000626B5B2504629463A464FF00003FEF7FC
:1005B000B7FF48B950469BF800109BF801204FF058
:1005C0000203FFF76BFFB3E2029B0398191801F1D6
:1005D000040201929BF800600E719BF801300198B3
:1005E00043704FF00008002F44D006E04FF00106A2
:1005F0004FF0000905F101050BE04FF000084FF046
:100600000106C14640F67461C2F2000105910494EE
:100610000C4640F2E73295420CD84FEAD500225CF6
:1006200005F0070342FA03F111F0010F0ED049EA79
:1006300006090BE005F11803D8B207A9F8F75EFB2D
:100640009DF81C1011B908B149EA060907F1FF37F6
:100650004FEA4606802E03D8002F00F08B82C9E7B0
:10066000019A02EB080383F8039008F10108002FB8
:10067000BCD1049C019981F80280504608F1030125
:10068000FEF702FE54E2BBF80250BBF804204FEA2A
:10069000122646EA0227BEB206F1FF31B1F5FA6F23
:1006A00009D350469BF800109BF801204FF003033C
:1006B000FFF7F4FE3CE24FEA152343EA052085B23A
:1006C000E8B207A9F8F782FA9DF81C204AB1504613
:1006D0009BF800109BF801204FF00203FFF7DEFEAD
:1006E00026E2029F03997B1803F1040001909BF816
:1006F00000201A719BF80170477056B3AFB24FF0EB
:1007000000084FF00105C14605E04FF001054FF02C
:10071000000907F10107F8B207A9F8F757FA9DF8A1
:100720001C1011B908B149EA050906F1FF364FEA74
:100730004505802D03D8002E00F02582E9E7019AB7
:1007400002EB080181F8039008F10108002EDCD1CA
:1007500001E04FF00008019F87F80280504608F141
:100760000301FEF791FDE3E1BBF802304FEA1326E7
:1007700046EA032080B20790BBF804704FEA1722C4
:1007800042EA0725AEB206F1FF317C2909D950466D
:100790009BF800109BF801204FF00303FFF77EFE4B
:1007A000C6E13146FEF70CFE48B150469BF80010FA
:1007B0009BF801204FF00203FFF770FEB8E1029BA7
:1007C00003981D1805F104079BF800202A719BF877
:1007D000011079703EB34FF0000806F1FF3303F0CB
:1007E000010907A84146FEF795FDA7F803004FF061
:1007F0000105AE4240F0CF8115E007A84146FEF763
:1008000089FD07EB4501A1F8030005F1010507A8E3
:100810004146FEF77FFD07EB4503A3F8030005F112
:100820000105AE42E9D14FEA4600C1B2B970504667
:1008300001F10301FEF728FD7AE1BBF80220BBF8C5
:1008400004504FEA152646EA0527BDB265B1B5F555
:100850007F4F09D050469BF800109BF801204FF0C5
:100860000303FFF71BFE63E14FEA122141EA022373
:100870009EB2504631464FF001021346FEF750FE3D
:1008800048B950469BF800109BF801204FF0020336
:10089000FFF704FE4CE10298039900EB0109304692
:1008A000B5F57F4F14BF00210121FEF781FE9BF8B3
:1008B000002089F804209BF8017089F80570BBF8C6
:1008C0000250A9F80650BBF80410A9F808105046C9
:1008D0004FF00601FEF7D8FC2AE1BBF802604FEAB0
:1008E000162747EA06218BB208A941F8043D504675
:1008F000BBF804204FF00003FEF786FD48B95046D0
:100900009BF800109BF801204FF00203FFF7C6FD93
:100910000EE10298039A851805F104069BF8007011
:100920002F719BF801107170BBF802307380BBF817
:100930000400B08050464FF00601FEF7A5FCF7E03A
:10094000BBF80200BBF804704FEA172646EA0722FC
:1009500095B205F1FF31B1F5FA6F06D29BF806307A
:1009600005F10707B3EBD70F09D050469BF80010ED
:100970009BF801204FF00303FFF790FDD8E04FEA0A
:10098000102646EA00201FFA80F8504641462A46C3
:100990004FF00103FEF7C4FD18B1002D40F0D280E6
:1009A00027E050469BF800109BF801204FF002030F
:1009B000FFF774FDBCE00BEB0700C179304629401E
:1009C000FEF7F6FD4FEA4505802D84BF0137454609
:1009D00006F1010630460BEB0702D1792940FEF7FC
:1009E000E7FD4FEA4505802D00F2F780F8E04E451F
:1009F000E1D1029D03982A1802F104069BF80070C9
:100A000017719BF801107170BBF802307380BBF84E
:100A10000450B58050464FF00601FEF735FC87E0E4
:100A2000BBF802704FEA172242EA072083B206930E
:100A3000BBF804504FEA152141EA0526B5B25F190B
:100A400007F1FF32079205F1FF307C2809D95046A3
:100A50009BF800109BF801204FF00303FFF71EFDE9
:100A600066E0504606A94FF000024FF00103FEF782
:100A7000CBFC50B1504607A94FF000024FF00103E4
:100A8000FEF7C2FC08B155B934E050469BF800109F
:100A90009BF801204FF00203FFF700FD48E04FF004
:100AA000000705F1FF3808F00109504606A9BBF818
:100AB00007203B46FEF7A8FC4FF00106B54240F088
:100AC000928017E00BEB4602504606A9B2F80720C9
:100AD0003B46FEF799FC06F101060BEB4603504638
:100AE00006A9B3F807203B46FEF78EFC06F1010687
:100AF000B542E7D1029D03982F1807F104069BF831
:100B000000203A719BF801107170BBF802307380BD
:100B1000BBF80450B58050464FF00601FEF7B4FB19
:100B200006E0504694F810114FF00103FFF7B6FCB1
:100B300042F62060C2F20000F4F770F95046FEF76A
:100B40008FFBDCE49BF80720404602F00101FEF732
:100B50002FFD08F1010608EB05094FF002054FF0E3
:100B600000074FF00108C6EB090111F0010F3FF437
:100B70003EAF22E0049C019D05EB080080F8039045
:100B800008F1010876E5019B03EB080080F803906B
:100B900008F10108DFE5B9F1000F3FF42EAE07A818
:100BA0004146FEF7B7FB07EB4502A2F8030005F14B
:100BB0000105AE427FF421AE35E60BEB0703D97990
:100BC00030462940FEF7F4FC4FEA4505802D84BFEE
:100BD0000137454606F1010609E707F101074546D9
:100BE00006F1010603E7B9F1000F3FF46BAF0BEB21
:100BF0004603504606A9B3F807203B46FEF704FC1F
:100C000006F10106B5427FF45DAF73E740F6B873B5
:100C1000C2F200034FF4117202FB003393F820324A
:100C2000012B0AD140F6B873C2F2000302FB003078
:100C3000C0F834124FF0000070474FF03700704793
:100C40002DE9F04F89B004460D4691F8029009EB6A
:100C5000490947F26C28C0F6010809EB08074FF470
:100C6000117B0BFB00FB40F6B87AC2F2000A0BEBDB
:100C70000A064FF00101F8F7B9FDC6F830522846D0
:100C800006F509714FF000021346FEF7B7FA204649
:100C90006978FFF7BBFF2046FEF7E2FAF5F720F888
:100CA000C6F828024FF00103009348F2B440C0F6A2
:100CB00001004FF0040140F2C942C0F60102234690
:100CC000F4F74AFBC6F81C025BF80A60EA7847F6BC
:100CD000B810C0F6010050F8221019F808207B78EF
:100CE000BD7800954FF0000001904FF23165C0F6DD
:100CF000000502954FF26D65C0F6000503954FF2B1
:100D0000A965C0F6000504954FF20D65C0F6000513
:100D10000595069075682046A84709B0BDE8F08F94
:100D2000D0F80031032B2BD94278102A2BD890F918
:100D300001204FF0010101FA02F212F06E0F06D10C
:100D400012F4803F12D112F4004F05D11BE0082BA2
:100D500014BF002001207047092B17D9807900F1BA
:100D60000900834214BF002001207047092B10D9CD
:100D7000807900F10900834214BF002001207047F0
:100D80004FF0000070474FF0010070474FF0000037
:100D900070474FF00000704742F6F573C2F200034F
:100DA0001A78027042F6EC70C2F2000003780B7001
:100DB000704700BF42F6F573C2F200031A78831A37
:100DC00012D442F6EC70C2F20000027893420EDABE
:100DD0004FF0010000FA03F342F6F072C2F2000293
:100DE000126813400B7070474FF0000070474FF0CF
:100DF0000000704708B52DED028BB0EE408A42F638
:100E0000F473C2F20003187888B94FF00000F0F7CD
:100E100007FF07EE900A88EE278AB7EE000AB4EEC5
:100E2000408AF1EE10FAD8BFB0EE480AFFE7BDECF9
:100E3000028B08BD08B543F22003C2F20003197803
:100E40004018C0B210EE101AF0F79CFC08BD00BFAD
:100E500010B542F6F573C2F200031A78841A4DD425
:100E600042F6EC70C2F2000003789C4249DA4FF07F
:100E7000010303FA04F3E1B142F6F071C2F200019A
:100E80000A68134240D142F6E071C2F200010868DC
:100E900018430860134342F6F072C2F20002136076
:100EA00042F6F873C2F2000393ED000AFFF7A2FFC7
:100EB0001EE042F6F071C2F200010A68134226D029
:100EC0006FEA030342F6E071C2F2000108681840BD
:100ED000086042F6E471C2F2000108681840086038
:100EE000134042F6F072C2F2000213609FED090A4D
:100EF0002046FFF79FFF4FF0010010BD4FF00000AC
:100F000010BD4FF0000010BD4FF0010010BD4FF0BC
:100F1000010010BD0000000070B52DED028B42F6FF
:100F2000E473C2F200031C68C4B142F6B870C2F2A6
:100F3000000090ED008A4FF000054FF001062642B8
:100F400004D02846B0EE480AFFF774FF4FEA460681
:100F500005F101052846264214D00FE042F6E07361
:100F6000C2F200031A6842F6E471C2F200010A609C
:100F70004FF000001860BDEC028B70BDB0EE480A67
:100F8000FFF758FF4FEA460605F10105202DD6D19F
:100F9000E4E700BF000000002DE9F8432DED028BCF
:100FA00042F6E873C2F2000393ED000AFFF722FF56
:100FB000B0EE408A42F6B870C2F20000D0ED007A7E
:100FC00037EEC00A10EE100A02F0AAFB01F068FF2B
:100FD00023A3D3E9002302F0F7FA00283CD142F61C
:100FE000B871C2F2000181ED008A42F6F072C2F2DD
:100FF0000002136883B342F6EC70C2F2000001787D
:1010000051B34FF001044FF0000542F6F077C2F201
:10101000000742F6E479C2F2000942F6E078C2F233
:10102000000842F6EC76C2F200063A6814420CD090
:10103000D9F80000D8F8003040EA03010C4204D18E
:101040002846B0EE480AFFF7F5FE05F101054FEA24
:1010500044043278AA42E8DCBDEC028BBDE8F88398
:101060007B14AE47E17A943F70B582B005461646D0
:101070009DF8184042F6F472C2F20002107042F677
:10108000F870C2F20000016042F6E871C2F200019D
:101090000E60A34243F22002C2F2000292BF13701C
:1010A00014701C4642F6F573C2F200039DF81C0052
:1010B000187043F22001C2F200010A78C2F1010364
:1010C000E418E4B242F6EC70C2F200000470202C86
:1010D00001D9EFF7BDFA40F2E010C2F200004FF084
:1010E0000101F7F7E5FC4FF0000100914FF001021C
:1010F000019242F6BC70C2F200004FF0FA014FF0CC
:10110000060240F61973C0F60103F4F7B3FDBDB94A
:101110004FF0000400944FF00100019042F6FC7083
:10112000C2F2000040F6C4114FF0060240F6997377
:10113000C0F60103F4F79EFD2046FFF72DFF04E003
:1011400042F6B873C2F200031E6002B070BD00BF69
:1011500043F22403C2F200031A7802705878087030
:10116000704700BF43F22403C2F200031B7883429E
:101170001AD843F22402C2F2000252789A1890421E
:1011800015DAC01AC3B24FEAD30243F23800C2F2F2
:101190000000825C03F0070342FA03F000F0010252
:1011A0000A704FF0010070474FF0000070474FF099
:1011B0000000704770B443F22403C2F200031B78AE
:1011C00083424DD843F22402C2F2000252789A18A8
:1011D000904248DAC01AC0B200F007054FF001048F
:1011E00004FA05F540F62C02C2F2000252E8003F74
:1011F00003F1010342E80036012EF7D043F2380331
:10120000C2F2000303EBD00393F8200028420CBF86
:1012100000200120087093F8201021EA050583F8CA
:10122000205052E8003FA3F1010342E80035012DB0
:10123000F7D052E8003FB3F1004F0DD14FF000035B
:1012400042E80035012DF4D04EF60450CEF20000F5
:10125000016841F080510160BFF32F8F204604E008
:101260004FF0000001E04FF0000070BC704700BF7D
:1012700043F22403C2F200031A790270587908700D
:10128000704700BF43F22403C2F200039A78027051
:10129000D8780870704700BF10B443F22403C2F23C
:1012A00000039B78834237D843F22402C2F2000243
:1012B000D2789A18904232DAC01AC3B24FEAD304F5
:1012C00003F007004FF0010202FA00F359B143F2B4
:1012D0003801C2F20001081990F8402043EA0201E7
:1012E00080F840100AE043F23801C2F20001081908
:1012F00090F8402022EA030280F8402043F23800B0
:10130000C2F20000021992F8601021EA030382F889
:1013100060304FF0010004E04FF0000001E04FF0BA
:10132000000010BC704700BF43F22403C2F2000368
:101330009B7883421BD843F22402C2F20002D27887
:101340009A18904216DAC01AC3B243F23802C2F2B7
:10135000000202EBD30090F8402003F0070342FAAA
:1013600003F000F001020A704FF0010070474FF0E7
:10137000000070474FF00000704700BF10B443F208
:101380002403C2F200039B78834237D843F224023D
:10139000C2F20002D2789A18904232DAC01AC3B26E
:1013A0004FEAD30403F007004FF0010202FA00F302
:1013B00059B143F23801C2F20001081990F86020D7
:1013C00043EA020180F860100AE043F23801C2F2F9
:1013D0000001081990F8602022EA030280F86020DA
:1013E00043F23800C2F20000021992F8401021EADC
:1013F000030382F840304FF0010004E04FF000009A
:1014000001E04FF0000010BC704700BF43F224031E
:10141000C2F200039A790270D8790870704700BF51
:10142000827802F107024FEAE2014FEA410202F13B
:101430000102037902EB8301407A0818704700BF6C
:1014400070B401F0070400EBD10000F1FF31C4F1EA
:10145000080611F8010F40FA04F00CB9C0B204E01C
:101460004D7805FA06F52843C0B2082B08D8C3F119
:1014700008034FF0FF0141FA03F31840107005E034
:1014800002F8010BA3F10803DBB2E2E770BC70477E
:101490002DE9F00F9DF82070044618B948F2F84481
:1014A000C0F6010402F0070C66464FF0FF0000FA98
:1014B0000CF5E8B201EBD20101F1FF31CCF10809E2
:1014C00048F2F848C0F601084A786FB9082B09D8E5
:1014D0004FF0010000FA03F000F1FF3505FA06F5C0
:1014E00005F0FF0022EA0002C5B294F800A00AFA53
:1014F00006FA05EA0A0A4AEA020201F101018A46ED
:101500000A70BCF1000F0DD04B450BDD4A7807B9CE
:10151000024094F800B04BFA09FB2BEA05052A4378
:101520008AF80120082B06D9444518BF0134A3F1DD
:101530000803DBB2C8E7BDE8F00F704708B5044800
:101540004FF000014FF0400202F06AFE08BD00BFFC
:10155000D831002008B504484FF000014FF02002B8
:1015600002F05EFE08BD00BF5830002010B54FF0FD
:10157000000443F23003C2F200031C6043F238005F
:10158000C2F2000021464FF4007202F049FE43F21D
:101590002400C2F2000021464FF0080202F040FE93
:1015A00010BD00BF10B50C4643F22403C2F2000385
:1015B0009979814217D843F22402C2F20002D3790A
:1015C000CA18904212DA401AC1B201F1680143F21E
:1015D0003803C2F2000353F82100F5F7DDFE206066
:1015E0004FF0010010BD4FF0000010BD4FF00000A3
:1015F00010BD00BF10B50C4643F22403C2F2000335
:101600001979814217D843F22402C2F200025379B9
:10161000CA18904212DA401AC1B201F1280143F20D
:101620003803C2F2000353F82100F5F7B5FE20603D
:101630004FF0010010BD4FF0000010BD4FF0000052
:1016400010BD00BF38B5054643F22403C2F20003C3
:101650009C79844217D843F22400C2F20000C27978
:10166000A3189D4212DA0846F5F76CFE2C1BE4B273
:1016700004F1680443F23801C2F2000141F8240089
:101680004FF0010038BD4FF0000038BD4FF00000B2
:1016900038BD00BF2DE9F0418AB00446FFF766FF70
:1016A00002A84FF000014FF0200202F0B9FD4FF008
:1016B000000001A9F7F75AF943F22403C2F200032C
:1016C0009DF804201A709DF8050098709DF806108A
:1016D00019719DF807509D714FF000064FF00108F9
:1016E00043F23007C2F200071D464AE06078FF2847
:1016F00045D14FEA531203F01F0108FA01F338688D
:1017000008B93C6008E0D8B20DF1280C0CEB82015E
:1017100051F8201C08422FD106F101060AA800EB5F
:101720008202DBB252F8201C43EA010042F8200C8E
:101730002046FFF775FE402871D8E37803F10702D1
:101740004FEAE2014FEA410000F10100627900EB4B
:101750008200E1794218402A64D8A078697842185A
:101760006A70E8781B18EB7021796A7988186871BB
:101770006179EB79CA18EA7104F10A0401E004F115
:1017800005042378FF2BB1D1102E4ED843F2240448
:10179000C2F200046279402A4AD843F22400C2F21D
:1017A0000000C179102946D843F22403C2F2000395
:1017B0005C783CB140F20020C2F200004FF0010121
:1017C000F7F74AF943F22402C2F20002D07838B1A6
:1017D00040F2F810C2F200004FF00101F7F768F98B
:1017E00043F22401C2F200014B793BB140F2E81010
:1017F000C2F200004FF00101F7F786F943F224042A
:10180000C2F20004E279DAB140F2F010C2F2000054
:101810004FF00101F7F7A4F94FF0000412E04FF088
:1018200045040AE04FF0430407E04FF0460404E0AB
:101830004FF00F0401E04FF00E04FFF797FE01E0B8
:101840004FF0000420460AB0BDE8F08108B540F230
:101850000020C2F200004FF00001F7F7FDF840F25F
:10186000F810C2F200004FF00001F7F721F940F242
:10187000E810C2F200004FF00001F7F745F940F21E
:10188000F010C2F200004FF00001F7F769F908BD4F
:101890002DE9F843044643F23003C2F2000318680E
:1018A00084421AD14FF0000543F22106C2F200062D
:1018B000357043F22D03C2F200031D7043F2340071
:1018C000C2F20000057043F22206C2F20006357033
:1018D00043F22C03C2F200031D70E57805F1070501
:1018E0004FEAE505E8B2667900EB860303F10103F0
:1018F000C018C6B296423ED843F23808C2F2000879
:1019000043F22102C2F20002177808EB070393F8B2
:10191000E0010F4607F8010B43F23401C2F2000167
:1019200091F8009008F1400049463A46E378FFF705
:1019300087FDEDB27F1908F1600049463A46E37829
:10194000FFF77EFD7A196379BBB143F22C05C2F231
:101950000005297808EB81004FF000031946C518EF
:10196000D5F8A051D55001F1010103F104036579C7
:101970008D42F4D801E04FF000063046BDE8F88310
:101980002DE9F04782B0044617461E4600296FD164
:10199000FFF746FDC5B2B5426CD1A3783E78002E64
:1019A00055D043F22102C2F20002117843F238000E
:1019B000C2F20000421892F8E011B14247D003F1A0
:1019C00007054FEAE50507F1010743F22D00C2F2D2
:1019D000000090F8009043F2380AC2F2000A4FF07B
:1019E00000020092384651464A46FFF751FD5FFA21
:1019F00085F84744A3784FF00101009138460AF179
:101A000020014A46FFF744FD47442379B3B143F22E
:101A10002200C2F2000001780AEB810C4FF00003B3
:101A20001A46F9580CEB0300C0F8A01002F10102AD
:101A300003F1040321799142F3D801E04FF0000251
:101A400005EB42054FEA450202F10102D5B243F22D
:101A50002103C2F20003187843F23801C2F20001F8
:101A60000B1883F8E0614FF0000283F8F02145E0A5
:101A70004FF0000543F22100C2F20000037843F268
:101A80003801C2F20001CA1892F8F001FF2835D0DF
:101A900000F10100C2B243F23801C2F20001CB18DA
:101AA00083F8F021082A29D143F22D06C2F200065C
:101AB00037788846A3784FF00006009630463A46BD
:101AC000FFF7E6FCA3780096304608F120013A467D
:101AD000FFF7DEFC217989B143F22200C2F2000057
:101AE000037803F1270308EB83023346304642F8BC
:101AF000040F03F1010321799942F8D843F221033D
:101B0000C2F200031A7802F101021A7043F22D00AA
:101B1000C2F200000178A378CA18027043F23400C0
:101B2000C2F200000178E378CA18027043F2220082
:101B3000C2F2000001782379CA18027043F22C0027
:101B4000C2F2000001786379CA180270284602B018
:101B5000BDE8F08730B40C18FA2C2BD869B343F2E7
:101B60003823C2F20003196840F67462C2F2000220
:101B7000051B6FEA050303F001050B181B796FEADB
:101B80000303835400F101039C421AD10FE0C818EB
:101B900000796FEA0000985403F10103C818007936
:101BA0006FEA0000985403F101039C42EFD14FF01B
:101BB000000004E04FF01A0001E04FF0000030BCDC
:101BC0007047002DE3D0C81800796FEA00009854E0
:101BD00003F101039C42DAD1E9E700BF10B50368C5
:101BE000B3F1FF3F1FD04AF20002C0F6010290425B
:101BF0001FD211466FEA0003D218C2F3002200F58B
:101C000080700368B3F1FF3F1DD10CE000F58073D5
:101C100018461A68B2F1FF3F05D003F580700368DB
:101C2000B3F1FF3F1CD14AF20001C0F60101884226
:101C300008D349F60004C0F6010420460A49F0F72B
:101C400015FD204610BD8842F3D2002ADED000F5F3
:101C500080700268B2F1FF3FE5D08842D6D3E8E752
:101C60008842D3D3E5E700BFFF9F01082DE9F0418B
